:020000040800F2
:1028000048AE0020C12A0008197F0108D12701081D
:102810001D4E01083D4D0008490702080000000058
:1028200000000000000000000000000045A80108B2
:1028300069780008000000001D8C0108D92A0008F2
:10284000DB2A0008DB2A0008DB2A0008DB2A000854
:10285000DB2A0008DB2A0008DB2A0008DB2A000844
:10286000DB2A0008DB2A0008DB2A0008E5760008DE
:10287000DB2A0008DB2A0008DB2A0008DB2A000824
:10288000DB2A0008DB2A00081D2D0008DB2A0008CF
:10289000DB2A0008DB2A0008DB2A0008DB2A000804
:1028A000DB2A0008B1DB0108DB2A0008DB2A00086C
:1028B000CDDD0108DB2A0008DB2A0008DB2A00083E
:1028C000DB2A0008DB2A0008DB2A0008DB2A0008D4
:1028D000DB2A0008DB2A0008DB2A0008B105020811
:1028E000DB2A0008DB2A0008DB2A0008DB2A0008B4
:1028F000DB2A0008DB2A00080000000000000000BE
:10290000000000000000000000000000DB2A0008BA
:10291000DB2A0008DB2A0008DB2A0008DB2A000883
:10292000DB2A0008DB2A0008DB2A0008DB2A000873
:10293000DB2A00080000000000000000DB2A00087D
:10294000DB2A0008DB2A0008DB2A0008DB2A000853
:10295000DB2A0008DB2A0008000000001D06020830
:10296000DB2A0008DB2A000800000000000000004D
:102970000000000000000000000000000000000057
:1029800000000000DB2A0008DB2A0008DB2A000820
:102990000000000000000000000000000000000037
:1029A0000000000000000000000000000000000027
:1029B0000000000000000000DB2A0008000000000A
:1029C0000000000000000000000000000000000007
:1029D000000000000000000000000000DB2A0008EA
:1029E00000F002F800F05CF80AA090E8000C8244C5
:1029F0008344AAF10107DA4501D100F051F8AFF2A2
:102A0000090EBAE80F0013F0010F18BFFB1A43F0CC
:102A100001031847505C0200705C02000A444FF04A
:102A2000000C10F8013B13F0070408BF10F8014B2D
:102A30001D1108BF10F8015B641E05D010F8016B72
:102A4000641E01F8016BF9D113F0080F1EBF10F8D6
:102A5000014BAD1C0C1B09D16D1E58BF01F801CBF9
:102A6000FAD505E014F8016B01F8016B6D1EF9D57C
:102A70009142D6D370470000002300240025002691
:102A8000103A28BF78C1FBD8520728BF30C148BFD1
:102A90000B6070471FB51FF0DCFA1FBD10B510BDED
:102AA00000F001F91146FFF7F5FF1EF05FFC00F0A2
:102AB0001FF903B4FFF7F2FF03BC00F027F9000091
:102AC0000948804709480047FEE7FEE7FEE7FEE7C2
:102AD000FEE7FEE7FEE7FEE7FEE7FEE704480549FE
:102AE000054A064B704700002DDA0108E12900086D
:102AF00048A8002048AE002048AA002048AA00208C
:102B000053EA020C00F069802DE9F04B4FF000060B
:102B1000002B1FBFB3FA83F503FA05F424FA05F678
:102B20005E4012BF1643B2FA82F502FA05F4C5F10F
:102B300020051EBF22FA05FC44EA0C04203556EAA3
:102B4000044C4FEA144418BF641C4FF000084FF0C7
:102B50000009904271EB030C39D3002919BFB1FA77
:102B600081F701FA07F6B0FA80F700FA07F6C7F125
:102B700020071EBF20FA07FC46EA0C062037B6FBEA
:102B8000F4FCA7EB0507103F07F01F0BCBF1200665
:102B90000CFA0BFB2CFA06F644BFB3460026202F96
:102BA000A4BF5E464FF0000B5BEA060C08BF4FF077
:102BB000010B19EB0B09ABFB027C48EB0608C01BB1
:102BC00006FB02CC0BFB03CC71EB0C01C1E70B46FF
:102BD000024641464846BDE8F08B13B54FF0000071
:102BE0004FF00001AFF30080BDE81C40704710B506
:102BF000203AC0F00B80B1E81850203AA0E81850F5
:102C0000B1E81850A0E81850BFF4F5AF5FEA027CB5
:102C100024BFB1E81850A0E8185044BF18C918C024
:102C2000BDE810405FEA827C24BF51F8043B40F8C5
:102C3000043B08BF7047D20728BF31F8023B48BFAA
:102C400011F8012B28BF20F8023B48BF00F8012BE8
:102C500070474FF0000200B513469446964620395F
:102C600022BFA0E80C50A0E80C50B1F12001BFF445
:102C7000F7AF090728BFA0E80C5048BF0CC05DF8AB
:102C800004EB890028BF40F8042B08BF704748BFF9
:102C900020F8022B11F0804F18BF00F8012B70476D
:102CA000704770477047754600F02CF8AE46050037
:102CB0006946534620F00700854618B020B5FFF757
:102CC0000DFFBDE820404FF000064FF000074FF029
:102CD00000084FF0000B21F00701AC46ACE8C0093A
:102CE000ACE8C009ACE8C009ACE8C0098D46704743
:102CF00010B50446AFF300802046BDE81040FFF752
:102D0000D8BE000000487047E8A7002001491820FD
:102D1000ABBEFEE7260002007047000010B5202180
:102D20000D481DF057FE40B120210B481DF04FFE0D
:102D30000A480068401C09490860012106481DF046
:102D400049FE40B1012104481DF041FE04480068DD
:102D5000401C0349086010BD00200140A408002069
:102D6000A00800201CB501A81DF01EFE02208DF851
:102D7000040000208DF8050001A81DF0FFFD684645
:102D80001DF0D7FD01208DF8000000208DF8010016
:102D90008DF8020001208DF80300694627481DF0D8
:102DA000AFFD002125481DF0D6FE04230122142189
:102DB00022481DF022FE0022072120481DF0BDFE02
:102DC00001211E481DF0F4FD01211C481DF0F5FDF8
:102DD00000224FF4807119481DF0D7FE14211748C6
:102DE0001DF0CEFE164915481DF0BAFE01229106CF
:102DF00012481DF0F7FD0122402110481DF0F2FDA0
:102E000001210E481DF0DEFD00BF40210B481DF0E2
:102E1000E1FD0028F9D009481DF092FD00BF0748E8
:102E20001DF094FD0028FAD104481DF098FD00BF64
:102E300002481DF09AFD0028FAD11CBD0020014077
:102E4000000280005A20014908607047B80F002036
:102E50000020044908800449087004490880044996
:102E600008607047C00F0020C20F0020C40F002070
:102E7000BC0F002001460020302905DB392903DC86
:102E8000A1F13002D0B20EE0412905DB462903DC76
:102E9000A1F13702D0B206E0612904DB662902DC29
:102EA000A1F15702D0B2704710B502460B4600217F
:102EB00007E05078147840EA04200144921C981EE0
:102EC00083B2012BF5DC13B1107801EB002102E095
:102ED00088B200EB1141080C0028F9D188B24FF6F6
:102EE000FF74604010BD00002DE9F0410546002749
:102EF00005EB45004E4A02EB0011302300224D48FD
:102F000003F0F4F94C4890F8670001281FD14948B4
:102F1000D0F805004749C1F80900084600780121AA
:102F2000B1EB901F4FD14348807B01094148007CA1
:102F300061F307103F4908740846B0F80D00B1F876
:102F40000F1060F30B013B48A0F80F103BE03A482C
:102F500090F86700022836D13648D0F80570D0F8CE
:102F600009003449C1F805000846C0F80970007826
:102F70000121B1EB901F26D12E48807B04092D48FA
:102F8000007C01092B48807B61F307102949887375
:102F90000846007C64F3071008740846B0F80D007A
:102FA000C0F30B060846B0F80F00B1F80D1060F33F
:102FB0000B012048A0F80D10B0F80F0066F30B00CD
:102FC0001C49A1F80F001B481C4908600968897852
:102FD00001F03F000FF03CFA1949086017480068FB
:102FE00017F05CFF1748007830B1002015490870D1
:102FF0004FF480401449886210480068C078C0F3DC
:103000004110012805D11148007820F004000F4933
:1030100008700A480068C078C0F34110022805D142
:103020000A48007820F0080008490870BDE8F081DF
:10303000EA2D00204A2E0020BB2900203C0B002056
:10304000C00B00204F0C0020000002406F0B00203E
:1030500010B515F02DFE1CF0FDFB1CF0F9FE10BDA7
:10306000F0B585B00024EBA30FCB01AD0FC5002652
:1030700000270EF04BF90546112D05D10120E94935
:1030800008704003E84988610A2D1ED14FF40050B2
:10309000E54988610120E54908700520E44981F887
:1030A000E90011F097FC11F041FC0220E1490860B1
:1030B000C82004F048FC0220DE491039086003E013
:1030C00016F02EFB16F048FBFAE70F2D0FD14FF448
:1030D0008040D54988614FF47A301DF017FB4FF4DA
:1030E000FA7004F030FC4FF48040CF4988620FF052
:1030F00099FD1EF0C9FBD04908800FF0BFF90DF013
:103100002BFD0DF00DFF0DF0ABFC002210214FF454
:1031100056200FF0E1F8C9490880012280214FF4C0
:1031200057200FF0D9F8C6490880032280214FF4B8
:1031300067200FF0D1F8C3490880022280214FF4A4
:103140005E200FF0C9F8C049088004F0EBFE0020B3
:103150001AF0CCFB01201AF0C9FBBC494878FFF7F4
:10316000C3FEBA484078BA490870BA4800780228C5
:1031700014D10020802302460821009010F0DCFAD0
:1031800000201023B4A208210090032005F060FC69
:10319000012000F0E1FE00F059FE38E1AD48007872
:1031A00004280FD10020802302460821009010F04F
:1031B000C3FA00201023ADA208210090032005F0DF
:1031C00047FC24E10B2D67D1A049497801EB41016F
:1031D000AB4A02EB011030230022AA4903F093F816
:1031E0009A494878FFF780FE9848407898490870D7
:1031F000002004F0F3F90220A34948700020802346
:1032000002460821009010F097FA002010239FA298
:1032100001460090022005F01BFC3CE00321601CED
:1032200015F086F9032309229D4901A803F05EF8F1
:103230000321E01C15F07CF903230D22984901A815
:1032400003F054F80020102301AA01460090042046
:1032500005F0FEFB264606EB46004FF4804101EBED
:103260000016894981F83840912231468648393024
:103270001EF0DAFA012003F005FFE01CD22190FBDA
:10328000F1F201FB120084B20A2004F05CFB4FF45F
:1032900000506549C862C1E7102D71D16B4949786A
:1032A00001EB4101764A02EB0110302300227549FF
:1032B00003F029F865494878FFF716FE634840781F
:1032C00063490870002004F089F900208023024639
:1032D0000821009010F030FA0020102371A201465E
:1032E0000090022005F0B4FB0823002272A101A87F
:1032F00002F0FCFFFF207349087032E0714800784B
:10330000FF282ED0704890F838400321601C15F03B
:103310000FF903230922624901A802F0E7FF032104
:10332000E01C15F005F903230D225D4901A802F008
:10333000DDFF0020102301AA01460090042005F0C3
:1033400087FB04EB4401614A02EB01109023002249
:103350005D49393102F0CAFFFF205A490870781CD4
:10336000C7B2462FCADB0DF0EBF842F260724FF4A1
:10337000804156481EF010FB0DF008F917F006F8D2
:103380002B48007D98B10020802302460821009040
:1033900010F0D2F90020264A0090517ED07D2023E3
:1033A0002C3205F055FB4FF47A7004F0CCFA16F08D
:1033B0003BFE474800780DF023FB4649087008465D
:1033C0000078454988731A4991F867201F49487861
:1033D00000210EF01FF8414941481DF08BF80523EC
:1033E00000223F4909313F4802F080FF01220721B6
:1033F000002017F0D3FC012017F018FD012017F072
:10340000DDFC012017F068FC00203749087005B08A
:10341000F0BD000053656E64696E67203A3030314C
:103420002D303034670B002000000240650B002077
:10343000BB290020280402401C0C00200A0C00209C
:10344000080C0020060C0020040C0020BB2D0020DE
:103450005F0B0020120C002044544D462052656D35
:103460006F7465204B696C6C00000000444D522065
:1034700052656D6F7465204B696C6C200000000014
:10348000EA2D0020574D0208C5A50020436F707932
:10349000285472616E736D69742920200000000049
:1034A000D0240020436F70792852656369766529BE
:1034B00020202020000000005265636576696E6759
:1034C00000000000410C0020C5A60020BE2E0020F8
:1034D000B60B0020B70B0020C0080020400B0020D6
:1034E000460B0020D3090020B3080020024600212B
:1034F00000201C2109E022FA01F303F00F03184415
:1035000000EB800358000B1FD9B20029F3DC22FA2C
:1035100001F303F00F0318447047000010B5044690
:1035200046F240000549088008464078204348702C
:1035300008460188472017F0D1F810BD0008002088
:103540002DE9F04106460D4614460027B846C5B1A0
:103550004FF20B57052C13D2DFE804F00306090CD9
:103560000F004EF21C670BE04DF6227708E04DF29B
:103570002D4705E04CF6354702E04FF6022700BF25
:103580002FE048F6E33743F22D58072C28D2DFE826
:1035900004F004090E13181D220048F6D73743F231
:1035A00007581DE048F6ED2743F2E15818E048F6C9
:1035B000962743F2066813E048F6081743F2797835
:1035C0000EE048F6DE5743F25A3809E048F6B36792
:1035D00043F2BA2804E048F6887743F2012800BF96
:1035E00000BF8EB135B1012D0DD13946742017F0D1
:1035F00075F808E03946442017F070F84146452038
:1036000017F06CF800BF11E035B1012D0DD139462E
:10361000752017F063F808E03946542017F05EF87B
:103620004146552017F05AF800BF00BFBDE8F081B1
:1036300010B540F2BE31132017F050F840F27B3144
:10364000122017F04BF840F27B21112017F046F8BA
:103650007A21102017F042F81921142017F03EF8B3
:1036600042F63821492017F039F848F220417B20F2
:1036700017F034F810BD000010B50446332017F0E1
:1036800005F80B490880012C06D10846007820F087
:1036900008000830087005E00548007820F00800B0
:1036A0000349087002480188332017F017F810BD4D
:1036B0000008002010B50446012C05D144F2480151
:1036C000432017F00BF804E043F22801432017F0E1
:1036D00005F810BD70B54FF47A750024002600205F
:1036E000424908604FF470404149088072E001206F
:1036F00004F029F9692016F0C9FF3E490880681EC8
:1037000085B208464078C009002841D10846407873
:10371000C0F3801000B1012636480088C0F30B04C6
:1037200024036A2016F0B2FF324908800846008858
:10373000C0F30B0004443048844202D0400084426D
:1037400000D126E0B4F5000F06D06FF07F40844230
:1037500002D04010844200D140E0244804606EB999
:10376000C4F31604204601F02BFE214908800846C8
:10377000008848B100201D49086070BD1B480068E2
:1037800040F0807019490860002019490880F4E76A
:1037900000BF682016F07AFF164908800846407876
:1037A000C009B8B908460088C0F30C04C82014FB4F
:1037B00000F040F29D11B0FBF1F4B4F5166F00D2A9
:1037C000641CB4F5FA7F05D9A0B240F480500849D2
:1037D0000880D2E7002D8AD12DB900BF002004490E
:1037E00008800249086000BFC7E700000408002005
:1037F00002080020000800205555550010B54FF470
:103800004071512016F06AFFC82004F09CF800F0C7
:10381000F9FD10BD2DE9F04105460F4616463C4620
:1038200035B1012D09D0022D18D0032D4BD116E052
:103830000021512016F052FF45E040F29D106043F8
:10384000C821B0FBF1F449F24101512016F046FFC6
:10385000C4F30C01072016F041FF34E000BF012E35
:1038600001D0032E05D10121204605F0C5FA0446FA
:1038700004E00021204605F0BFFA0446032D04D1E0
:103880004FF420401149088003E04FF400400F49F5
:1038900008800E48008840F02A01512016F01EFFD3
:1038A00040F6D721072016F019FFC4F30B010820BA
:1038B00016F014FF4FF4004000EB143081B20820E2
:1038C00016F00CFF00BF00BFBDE8F081000800202B
:1038D00010B50C2016F0DAFE2F4908800846007853
:1038E00000F0010050B12D480078022806D116F0F2
:1038F000C5F80C2016F0CAFE2749088026484078F3
:10390000C0F3C00008B1042010BD25480068807BCA
:103910000121B1EB101F04D021480068807B000911
:1039200018BB1D484078C0F3401030B91A484078A1
:10393000C0F3001008B10420E6E717484078C0F350
:10394000401030B114484078C0F3001008B904208A
:10395000DAE711484078C0F3401030B10E484078A3
:10396000C0F3001008B10420CEE70B484078C0F344
:10397000800008B10120C7E707484078C0F38010F5
:1039800008B10220C0E704484078C00908B103200C
:10399000BAE70020B8E70000000800206D0B002007
:1039A0003C0B002010B5312016F070FE0B4908804A
:1039B0000846007820F00800087008460188312089
:1039C00016F08CFE46F63831282016F087FE4AF6AF
:1039D0004031292016F082FE10BD000000080020B2
:1039E00010B5044648F22A0014490880200E30B170
:1039F0000846407820F008000830487005E00F487D
:103A0000407820F008000D4948700C48018851208A
:103A100016F064FE40F6D721072016F05FFEC4F3CF
:103A20000B01082016F05AFE4FF4004000EB143052
:103A300081B2082016F052FE10BD000000080020E0
:103A400070B50446664890F80102C51C05EB850078
:103A50004FF6FF7101EA4005102C13D2DFE804F0A5
:103A600008131E29343F4A55606B76818C97A2ADAE
:103A700042F2F351712016F031FE43F2E15172200F
:103A800016F02CFEA4E041F61C41712016F026FE33
:103A900043F2C201722016F021FE99E041F61C416A
:103AA000712016F01BFE43F2E151722016F016FE53
:103AB0008EE041F61C41712016F010FE43F6913164
:103AC000722016F00BFE83E041F60E71712016F0A5
:103AD00005FE43F2C201722016F000FE78E041F6C6
:103AE0000E71712016F0FAFD43F2E151722016F0CA
:103AF000F5FD6DE041F60E71712016F0EFFD43F615
:103B00009131722016F0EAFD62E042F25C217120F0
:103B100016F0E4FD43F2C201722016F0DFFD57E01B
:103B200042F25C21712016F0D9FD43F2E15172207E
:103B300016F0D4FD4CE042F25C21712016F0CEFD6F
:103B400043F69131722016F0C9FD41E041F61C4167
:103B5000712016F0C3FD44F2DC11722016F0BEFD98
:103B600036E041F60E71712016F0B8FD44F2DC111A
:103B7000722016F0B3FD2BE042F25C21712016F0AA
:103B8000ADFD44F2DC11722016F0A8FD20E042F2F7
:103B9000F351712016F0A2FD44F2DC11722016F0F0
:103BA0009DFD15E042F2F351712016F097FD43F2AE
:103BB000C201722016F092FD0AE042F2F351712028
:103BC00016F08CFD43F69131722016F087FD00BF90
:103BD00000BF0448007810B9284603F0B4FE70BD59
:103BE000BB290020740B002010B50021242016F002
:103BF00075FD0021702016F071FD10BD10B56F210C
:103C0000092016F06BFD41F26B01092016F066FDEC
:103C100042F26701092016F061FD43F262010920BA
:103C200016F05CFD44F25001092016F057FD45F2F4
:103C30004701092016F052FD46F23A01092016F01C
:103C40004DFD47F22C01092016F048FD48F24101D4
:103C5000092016F043FD49F23701092016F03EFD18
:103C60004AF22501092016F039FD4BF2170109200F
:103C700016F034FD4CF2E401092016F02FFD4DF250
:103C8000CB01092016F02AFD4EF2B501092016F0ED
:103C900025FD4FF29F01092016F020FD4FF4DB6156
:103CA000212016F01BFD144890F8070213490880E4
:103CB000084600884FF6FF7101EAC0100F490880DE
:103CC0000846008848F27E0108430C4908800846EF
:103CD0000188242016F002FD074890F80602803083
:103CE00006494870084640780870084601887020E8
:103CF00016F0F4FC10BD0000BB29002000080020D5
:103D000010B50446FFF77AFF2046FFF799FE0348F7
:103D1000007808B9FFF768FF10BD0000740B0020A1
:103D20002DE9F04105460E46364890F80202C71CC0
:103D300007EB87004FF6FF7101EA400719F04AFDD3
:103D400000F062F81E2003F0FEFD002454E0285D20
:103D500036282AD012DC322823D008DC232841D090
:103D60002A283BD030281AD031283FD118E03328F8
:103D700018D0342817D0352838D115E041281DD067
:103D800006DC372812D0382811D039282ED10FE080
:103D9000422817D0432819D0442827D11AE000BF61
:103DA00000BF00BF00BF00BF00BF00BF00BF00BF1B
:103DB000295D3039C8B2FFF7A3FF17E00A20FFF7EB
:103DC0009FFF13E00B20FFF79BFF0FE00C20FFF796
:103DD00097FF0BE00D20FFF793FF07E00E20FFF7A2
:103DE0008FFF03E00F20FFF78BFF00BF00BF3846B7
:103DF00003F0A9FD601CC4B2B442A8DB02F03EF996
:103E0000BDE8F081BB29002010B54BF22A3000F04C
:103E1000FDFD0121084600F08FFD402017F0AAFBB0
:103E200010BD10B504462146402016F057FC10BDC9
:103E300010B500213F2016F051FC2821592016F022
:103E40004DFC0021302016F049FC10BD10B54FF498
:103E500020513F2016F042FC44F22801592016F070
:103E60003DFC43F22801592016F038FC0C4800684C
:103E7000407800F00F0010B9FFF7C0FE01E0FFF737
:103E8000B3FE002007490870074908700749087009
:103E90001023002206A10B4802F028FA10BD0000F2
:103EA0003C0B00201C0800201B0800201D080020DF
:103EB0002020202020202020202020202020202002
:103EC000000000001E08002070B5C8254FF4004116
:103ED0003F2016F003FC48F22801592016F0FEFBA3
:103EE0002821592016F0FAFB00240FE01848005D45
:103EF000184948701649601C085C16490870084645
:103F000001885F2016F0EAFBA01C84B2102CEDDBC8
:103F100042F62801592016F0E1FB00200D490880E7
:103F200009E00C2016F0B2FB0A490880052003F0D6
:103F30000AFD681EC5B20748007800F0010008B904
:103F4000002DEED10021022016F0C8FB70BD00004C
:103F5000D40F00200008002010B50446C4B1E021B1
:103F6000702016F0BBFB43F26501722016F0B6FB21
:103F700043F2C371582016F0B1FB45F265615C2035
:103F800016F0ACFB4FF470615D2016F0A7FB07E064
:103F90000021702016F0A2FB0021582016F09EFB95
:103FA00010BD10B50021322016F098FB10BD0000A6
:103FB00010B50D2016F06AFB0E49088008464078BF
:103FC000C00908B1002010BD0A480088C0F30A04E7
:103FD00024040E2016F05AFB04440748008848F2D7
:103FE000280121440C1A204601F07EFC044620469C
:103FF000E9E70000000800203B25002010B540F64E
:104000000131322016F06AFBC8200149087010BD4A
:104010001F0C002070B505462C4620460CF0EEFF24
:10402000064800882844A0F50044A1B2382016F0C4
:1040300055FB210C392016F051FB70BD3B250020AB
:1040400010B5632016F022FB02490880084600786C
:1040500010BD00000008002010B5044604F5204003
:1040600081B24D2016F03AFB04F5DE4081B24E20BD
:1040700016F034FB10BD000010B558480078032836
:104080001DD14FF4005056498862564A1268127C7E
:104090001109544A1268D27802F0070000F004FCBB
:1040A000002000F0C5FB002000F0E0FB0020FFF73F
:1040B000E3FA002000F05CF9142003F044FC4748C8
:1040C000007800280BDDFFF7B3FAFEF7BBFEFEF722
:1040D000BFFE0020FFF722FA042016F035F941490F
:1040E0000968D1F80500FFF795FF3E4800680079A0
:1040F000C0F3420004281DDA3A480068807B0009BA
:104100003949088037480068B0F80D00C0F30B004B
:1041100036490880084600883549088031490968D1
:104120000979C1F342023049087830490988FFF71C
:1041300071FB05E02B490968D1F81A00FFF750FC24
:10414000284800680079C0F342002A4908702A48CC
:1041500090F814010B2190FBF1F201FB12002749AA
:104160000C5C2046FFF778FF1E4800680079800944
:1041700040B92348007800F0DBF82248007800F0CE
:1041800021F907E02048007800F0D2F81F480078B5
:1041900000F018F9134800680079C0F301100128F5
:1041A00003DD002000F032FA02E0012000F02EFAD8
:1041B00000F028F916480078012805D100F0A2F98E
:1041C000002000F0BDF905E0002000F09BF901207F
:1041D00000F0B6F900200149087010BD6D0B0020F9
:1041E000000002403C0B0020080800200A080020C4
:1041F0000E0800200C080020BB29002029210208FD
:1042000016080020180800201708002019080020B0
:104210001A08002010B54FF40041002016F05EFA95
:104220000A2003F090FB0021084616F057FA41F6E9
:104230000F51372016F052FAFFF7FAF94FF4807158
:10424000332016F04BFA0021342016F047FA0021F3
:10425000352016F043FA44F658411E2016F03EFA77
:104260004AF256611F2016F039FA4AF237013E2011
:1042700016F034FA4EF650117D2016F02FFA4FF456
:104280009D51262016F02AFA1848C27A01210020F2
:10429000FFF756F91548827A00210846FFF750F9D2
:1042A0001248427A01210846FFF74AF90F48027A7C
:1042B00000210120FFF744F900F0A4F8002000F0ED
:1042C00032FB002000F074F90020FFF727F9FEF719
:1042D000B9FDFEF7BDFD064890F80D0120B1044977
:1042E00091F80D0100F07EFB10BD00001B250020A1
:1042F000BB29002010B504464EF640102044044966
:104300000880084601887D2016F0E8F910BD0000FD
:104310000008002010B5652016F0B8F903490880A0
:104320000846007800F07F0010BD00000008002063
:1043300010B504460B4890F802010B49095CA01C1B
:1043400008440A494870201F064991F80211064A9C
:10435000515C084405490870084601884F2016F052
:10436000BDF910BDBB29002034210208000800203F
:1043700010B504467F200A490880A006000E487048
:104380000CB1012000E000200549097860F3C71155
:10439000034801700188362016F0A0F910BD000016
:1043A0000008002010B5672016F070F90449088055
:1043B00008460088C0F3080008800846008810BD41
:1043C0000008002010B504460B4890F802010B4984
:1043D000095CA01C08440A494870201F064991F84E
:1043E0000211064A515C08440549087008460188D4
:1043F000782016F073F910BDBB2900203F21020878
:104400000008002010B541F60F71372016F066F94C
:104410000A2003F098FA4FF40071302016F05EF98C
:104420004BF6F171302016F059F910BD10B52F4838
:1044300090F806414FF6FF7000EA04144BF20F00AB
:10444000204484B202202A4908702A480068C078B3
:10445000C0F3C100022805D12748007840F00800C9
:104460002549087023490968497801F00F0000F0D8
:104470009FF820480068407800F00F0028B104221F
:1044800001210020FFF75CF805E01C48C27A0121F9
:104490000020FFF755F8204600F0B8FA15480068EC
:1044A0000079C0F3011030B101280BD0022810D0E0
:1044B000032816D10EE00020114908700120FFF7F3
:1044C0002DF80EE001200E4908700720FFF726F8AE
:1044D00007E000BF01200A4908700520FFF71EF819
:1044E00000BF00BF042017F045F810BDBB29002015
:1044F0006D0B00203C0B00206F0B00201B250020C3
:104500003208002010B50446332016F0BFF80B49DE
:104510000880012C06D10846007820F010001030E9
:10452000087005E00548007820F010000349087085
:1045300002480188332016F0D1F810BD0008002091
:1045400010B50446332016F0A1F80B490880012C61
:1045500006D10846007820F00200801C087005E0B3
:104560000548007820F002000349087002480188DD
:10457000332016F0B3F810BD0008002010B509482C
:1045800090F8020110B10848007808B1012010BD70
:104590000C2016F07BF80549088008460078C0F327
:1045A0004000F4E7BB290020690B00200008002030
:1045B00010B5044614480480008800EBC01046F68D
:1045C000DC0101EBC0001049088008460188712019
:1045D00016F084F8312016F059F80B4908802CB9F0
:1045E0000846007820F00200087006E006480078CF
:1045F00020F00200801C0449087003480188312023
:1046000016F06CF810BD00000008002010B504463C
:10461000732016F03BF80B4908802CB1084600784F
:1046200020F01000087006E00648007820F0100026
:1046300010300449087003480188732016F04EF8C2
:1046400010BD00000008002010B5002000F0F0F8B8
:10465000002000F00BF90020FFF754FF0020FFF7C7
:104660006FFF0021302016F039F84FF4E851372061
:1046700016F034F801200149087010BD6C0B0020C1
:1046800010B5044641F60F51372016F027F80A20DE
:1046900003F059F940F28F21522016F01FF84FF421
:1046A0000071302016F01AF82CB94CF2FE113020AF
:1046B00016F014F804E04CF2FA31302016F00EF83F
:1046C00010BD000010B50020FFF71CFF0020FFF711
:1046D00037FF4A48007810B94948007818B10320DC
:1046E000FEF71CFF02E00120FEF718FF45490968AC
:1046F000D1F80900FFF78EFC424800680079C0F34A
:104700004200042819DA3F480068007C00093E494D
:1047100008803C480068B0F80F00C0F30B003B492C
:104720000880384909680979C1F342023649087896
:1047300036490988FFF76EF805E032490968D1F873
:104740001A00FFF74DF92F4800680079C0F34200C6
:104750002F4908702B490968497801F00F00FFF7CD
:1047600027FF2C4991F80501FFF7C4FD2548006893
:104770000079800928B92849B1F80300FFF751FBF7
:1047800003E025494889FFF74CFB0120FFF73EFF76
:104790001A49097811B91A49097809B1012100E0CB
:1047A00000210846FFF76CFF1C480078012806D15D
:1047B00000F03EF84FF480601949886206E001205D
:1047C00000F054F84FF48060154988610120FEF72D
:1047D00053FF0C48006880780121B1EB901F04D191
:1047E00010480078FFF7C4FD03E00F480078FFF79A
:1047F000BFFD03200D49087010BD00006A0B0020AA
:10480000680B00203C0B0020080800200A0800204C
:104810000C080020BB2900203B2500201A0800209E
:104820000000024014080020150800206D0B002035
:1048300010B50446332015F029FF0B490880012CE0
:1048400006D10846007820F020002030087005E0EE
:104850000548007820F020000349087002480188CC
:10486000332015F03BFF10BD0008002010B50446B2
:10487000332015F00BFF0B490880012C06D10846A8
:10488000007820F00400001D087005E0054800785D
:1048900020F004000349087002480188332015F015
:1048A0001DFF10BD0008002070B505460C4605B977
:1048B00070BD49F24001512015F010FF2CB940F2B3
:1048C0006F41072015F00AFF28E0012C21D1012DAE
:1048D00006D0022D0AD0032D0ED0042D18D111E0E0
:1048E00040F26F41072015F0F9FE11E04AF28F21E6
:1048F000522015F0F3FE0BE04CF28F21522015F000
:10490000EDFE05E04EF28F21522015F0E7FE00BFCC
:1049100004E048F23F21522015F0E0FEFA2003F0B7
:1049200012F800BFC4E710B504466720604381B2A7
:10493000712015F0D3FE10BD70B504460D467020F1
:1049400015F0A4FE17490880C0204870084640783A
:1049500065F3C710487008460188702015F0BEFE48
:1049600095B144B14CF2FA31302015F0B7FE032076
:10497000FEF7D4FD14E040F20231302015F0AEFE17
:104980000220FEF7CBFD0BE02CB14CF2FE113020E3
:1049900015F0A4FE04E04BF6F171302015F09EFEF8
:1049A00070BD00000008002070B504460D4664206C
:1049B00015F06CFE0949088008460088B4EB201FFA
:1049C00001DC012070BD05480088B5EB201F01DB2C
:1049D0000020F7E702480078F4E700000008002014
:1049E000790B002010B50446312015F04FFE064922
:1049F00008800846007864F3820008700846018841
:104A0000312015F06BFE10BD0008002010B50446E3
:104A1000012015F03BFE134908800846008808284D
:104A200019D2DFE800F0121804051318060700BFBA
:104A300000BF00BF04F00F00032801DDE01E84B2B8
:104A40002146482015F04AFE0AE000BF21464820D2
:104A500015F044FE04E02146482015F03FFE00BF5B
:104A600000BF10BD0008002010B50F48007800B945
:104A700010BDFFF7C7FC0D480078012805D1FFF7EE
:104A800041FD0020FFF75CFD05E00020FFF73AFD47
:104A90000120FFF755FD0A2002F055FF00200249D2
:104AA000087000BFE4E700006C0B00201A0800202B
:104AB00038B500244FF48040734988614010886104
:104AC0000BF03EFD002080230246082100900EF0EE
:104AD00033FE00200F236DA201460090022003F058
:104AE000B7FF00200F236DA201460090042003F0C1
:104AF000AFFF4FF4805251006C481CF095FE03202C
:104B00001CF010FF4FF480524FF4405167481CF0E6
:104B1000AFFF00BF14E04FF4804000EB043182107F
:104B200062481CF081FE04F110001CF0FBFE4FF403
:104B3000803000EB043102115C481CF099FF641CCA
:104B40000C2CE8D34FF480524FF4E03157481CF05E
:104B50006BFE1D201CF0E6FE4FF480524FF4E8314E
:104B600052481CF085FF002416E04FF4F03000EBB3
:104B700004314FF480524D481CF056FE04F13E00C3
:104B80001CF0D0FE4FF4783000EB04314FF480522B
:104B900046481CF06DFF641C202CE6D3002416E070
:104BA0004FF4BC2000EB04314FF480523F481CF01E
:104BB0003BFE04F192001CF0B5FE4FF4122000EB16
:104BC00004314FF4805239481CF052FF641C342CDD
:104BD000E6D3002416E04FF4462000EB04314FF4F6
:104BE000805232481CF020FE04F1CB001CF09AFEEB
:104BF0004FF44B2000EB04314FF480522B481CF053
:104C000037FF641C052CE6D3002416E04FF4502037
:104C100000EB04314FF4805224481CF005FE04F1EF
:104C2000D3001CF07FFE4FF4532000EB04314FF40F
:104C300080521E481CF01CFF641C032CE6D34FF46A
:104C400080524FF4562119481CF0EEFDEF201CF065
:104C500069FE4FF480524FF46F2114481CF008FF96
:104C60004FF480524FF4702110481CF0DDFDF1200C
:104C70001CF058FE4FF480524FF471210B481CF089
:104C8000F7FE0BF083FC38BD000002404261636B0D
:104C9000696E672075702E2E2E202000506C656185
:104CA000736520776169742020202000BE2E0020CB
:104CB00010B50BF045FC4FF48052002107481CF062
:104CC000B3FD01201CF02EFE4FF480521146034824
:104CD0001CF0CEFE0BF05AFC10BD0000BE2E0020D2
:104CE00070B50446144DE4B1681C90FBF4F0451E09
:104CF000012108461CF040F9002229464FF080406F
:104D00001CF080FF00214FF080401CF09AFF012230
:104D1000114690071CF0ABFF012188071CF096FF9D
:104D200008E0002101201CF027F900214FF080400D
:104D30001CF08CFF70BD0000FF1AB70000BFFEE73B
:104D40002DE9F84F80468946924600250026AB465D
:104D500000240027002000908A4890F84A0330B9C8
:104D6000B8F10C0F00D10AE04FF0010B07E0B8F1E9
:104D70000C0F02D14FF0010B01E04FF0000B824805
:104D800041781430405C02287ED17F48407800EBA7
:104D900080107E4901EBC0007B49497800EB41005F
:104DA000058800271CE07848407800EB80107749A0
:104DB00001EBC0007449497800EB4100018872485A
:104DC000407800EB8010714A02EBC000143000EB19
:104DD00047000088814201D13E4603E0781CC7B2FB
:104DE000FA2FE0DB00BF00BFBBF1000F07D1701C42
:104DF000FA2190FBF1F201FB1200C6B207E006F1C6
:104E0000F900FA2190FBF1F201FB1200C6B2601C1E
:104E100084B25D4A527802EB82125C4B03EBC20211
:104E2000143202EB46021088574A51780BF04AFEC2
:104E300010B9FA2C00DAD7E7FA2C11DB5248407887
:104E400000EB8010514901EBC0004F49497800EB5D
:104E5000410005804C4948780DF026FCBDE8F88FEC
:104E60004948407800EB8010484901EBC0001430FD
:104E700000EB460001884448407800EB8010434A2C
:104E800002EBC000404A00E025E0527800EB42000F
:104E900001803D48407800EB80103C4901EBC000A8
:104EA0003949497800EB4100008837494978384A48
:104EB00022F81100B9F1000F4BD0334A527802EBBF
:104EC0008212324B03EBC2012F4A53781832D05C66
:104ED00015F0E2FD3DE02C4840782D4931F81050A6
:104EE00000BFBBF1000F03D1681CC0F3090502E04D
:104EF000681EC0F309050121284600F03FFB30B9C8
:104F00002046611C8CB2B0F5806F00DAE9E7B4F599
:104F1000806F19DB1C4840781D4931F81000009063
:104F2000009800EB40004FF4804101EB001000902E
:104F30001549497801EB4101164A02EB0110302274
:104F400000991CF071FC89E7B9F1000F01D015F050
:104F5000E5FC0C4991F867200B4948780E4909781F
:104F60000CF058FA012015F029FF012015F0B4FECD
:104F7000BAF1000F03D004494878FDF7B5FF00BF30
:104F80006CE70000BB290020BB2D0020AB250020D2
:104F9000600B0020EA2D00206D0B00202DE9F04170
:104FA0000746002015F0ACF90546052015F0A8F9D4
:104FB00006460821284613F0BBFA082405E0601EC7
:104FC0001D49085C0855601EC4B2032CF7DC2E2076
:104FD0001949C8701948407948721023002218A155
:104FE0001C4801F083F90A2305221349194801F0EE
:104FF0007DF90721304613F09BFA072405E0601E77
:105000000D49085C0855601EC4B2022CF7DC2E2046
:10501000094988700948807A0872102300220EA17D
:10502000124801F063F90923052203490F4801F0F2
:105030005DF9BDE8F0810000D0240020D40F0020ED
:10504000572F45203A2020202020202020202020DB
:1050500000000000340800204E2F53203A2020206A
:1050600020202020202020200000000044080020D4
:1050700010B501220621104615F090FE15F0B6FA83
:105080000923002204A1074801F030F90020064955
:1050900008600649087010BD43482D2D2D2D2D2088
:1050A00020000000940C0020900C00208E0C0020AA
:1050B00010B51023002209A10D4801F017F91023A3
:1050C00000220B490B4801F011F900200A49087031
:1050D0000A490870012015F01BFE10BD5F2020203A
:1050E0002020202020202020202020200000000040
:1050F000AE0C002035090020AD0C0020BE0C0020B5
:1051000010B5082300220AA10C4801F0EFF808238B
:1051100000220A490A4801F0E9F80020094908601C
:105120000949087009490870012015F00DFE10BDED
:105130005F20202020202020000000009F0C002065
:105140005F090020A80C00209D0C0020AC0C002062
:1051500010B5002018490870184908801849897C42
:10516000481C022113F0E4F90223032215491648D2
:1051700001F0BCF81549B1F80100042113F0D8F989
:10518000052303222E210F480EF00EFA05230022DC
:105190000C490D48401D01F0A9F8102300220B49CD
:1051A0001E3109480A3001F0A1F801200849887031
:1051B000C870087110BD0000BF0C0020C00C00209A
:1051C000BB2D0020D0240020FA080020E40F00208E
:1051D0001409002010B515F009FA0923002205A1D1
:1051E000074801F083F80020064908600649087066
:1051F00010BD00002D2D2D2E2D2D2D2D2D0000004C
:10520000940C0020900C00208E0C002010B5084853
:1052100041781430405C10B9FFF7DCFF01E0FFF784
:1052200027FF502204214FF4DC700FF045FD10BD24
:10523000BB2D002010B500200949086009490870FD
:105240000949087C032113F073F903231A4607491F
:10525000074801F04BF801200649C87010BD000056
:10526000900C00208E0C0020BB2D0020D0240020AC
:10527000150B00200925002010B510498868082169
:1052800013F056F9092303222E210D480EF08CF954
:10529000092300220A490B4801F028F809230022BB
:1052A00009A10C4801F022F800200B4908600B49C5
:1052B000087001200A49887010BD0000BB2D002035
:1052C000D0240020020B00202D2D2D2E2D2D2D2D34
:1052D0002D000000940C0020900C00208E0C00206B
:1052E0000925002010B50B48007810B9FFF7C4FF5E
:1052F00008E008480078012802D100F00DF801E02C
:10530000FFF798FF502204214FF4DC700FF0D4FC1B
:1053100010BD0000DC0C002010B500200C49086016
:105320000C4908700C49C868062113F001F90723DD
:1053300001222E2109480EF037F9072303220749DD
:10534000074800F0D3FF01200649487010BD000057
:10535000900C00208E0C0020BB2D0020D0240020BB
:105360000B0B00200925002030B50346002000BFAC
:1053700023E0002404EB40041C5D2407250E00EB11
:1053800040040D55012404EB40041C5D240100255C
:1053900005EB40055D5D04EB2514E5B200EB400430
:1053A000641C0D55012404EB40041C5D251100EB29
:1053B0004004A41C0D55441CE0B29042D9DB30BD22
:1053C000F0B5044600271FE000250EE028460BF04C
:1053D00027FB064606F5006003F024FDA04202D13B
:1053E00046F40050F0BD681CC5B2692DEEDD04F432
:1053F000800020B16400C4F31600441C02E0640085
:10540000C4F31604781CC7B2172FDDDB0020E9E7D0
:1054100070B504460E46304606F090FC0546B6F1DF
:10542000AA3F06D10823002213A1204600F05EFF08
:1054300020E0C5F303103030207005F00F0030304D
:105440006070C5F303303030A070C5F303203030F6
:10545000E070C5F3035030302071C5F303403030A5
:1054600060710F2000EA15703030A071C5F3036041
:105470003030E07170BD00003136373737323135AA
:105480000000000038B505466C78A87830B10128D6
:105490001ED0022823D0032830D121E0601C052132
:1054A00090FBF1F201FB1200C4B20123002221465D
:1054B00028460DF07FFB032C01D0042C07D10020DF
:1054C000802302460221009006200EF035F915E0F7
:1054D000642202214FF4DC700FF0EEFB38BD00BFF8
:1054E000601C032190FBF1F201FB1200C4B2AA7808
:1054F0000123214628460DF05DFB00BF00BF64225A
:10550000022140F25C600FF0D7FB00BFE6E70146E6
:10551000092903DC01F13000C0B270470D2903DC1A
:1055200001F13700C0B2F8E70E2901D12A20F4E7D3
:105530000F2901D12320F0E72020EEE710B5024625
:105540000B460021002000BF15E020B101280DD03E
:1055500002280DD100E000BF545C802C02DB545CBB
:10556000FF2C01D1002000E0012001E0022000BF5B
:1055700000BF4C1CA1B29942E7DD10BD2DE9F041FE
:1055800004460F460025002652484078524931F81B
:105590001000A04237D0254605EB45004FF480416E
:1055A00001EB00154B49497801EB41014B4A02EBF5
:1055B0000110302229461CF037F94648407800EBAC
:1055C0004000464901EB001000780121B1EB901F2B
:1055D0001ADA17B10020BDE8F0813E4840783E4914
:1055E00031F8105005EB45004FF4804101EB0015F8
:1055F0003849497801EB4101384A02EB0110302269
:1056000029461CF011F962E0324841781430405CC0
:1056100001280DD12F4841781A3000EB4100048059
:105620002C4840782C4921F8104015F077F94EE0CD
:1056300000260FE02748407800EB8010284901EB56
:10564000C000143000EB46000088A04200D103E007
:10565000701CC6B2FA2EEDDB00BFFA2E19D10FB1C5
:105660000020B8E71B4840781B4931F8105005EB83
:1056700045004FF4804101EB00151649497801EBD4
:105680004101164A02EB0110302229461CF0CCF8E9
:105690001DE01048407800EB8010114901EBC0007C
:1056A0000C49497800EB410004800A4840780A49D7
:1056B00021F81040074A527802EB8212084B03EBA4
:1056C000C201044A53781832D05C15F0E5F9012084
:1056D00081E70000BB2D0020600B0020EA2D002098
:1056E000AB25002010B50024FEF7F2F80446042C88
:1056F00010D0012C21D13B48008802280AD039481B
:105700000088032806D0384800680079C0F34200BA
:10571000042812D1002009F051FD344800780228F5
:1057200007D033480078022806D13048007808288E
:1057300002D104202F49087010BD2F48007801289D
:1057400023D12848008830B1012805D002280AD08A
:10575000032816D10EE014E0012C03D0274800786E
:1057600000B9E9E70DE0022C03D02448007800B925
:10577000E2E706E0032C03D02048007800B9DBE71D
:1057800000BF00BF03F0B8FE29E01648008818B338
:1057900014BB1A480078F8B9144800780B2807D0D1
:1057A000134800780B2805D110480078082801D14B
:1057B000012000E0002078B9114801880088401CD1
:1057C0000F4A1080B1F5C87F09DD09F0A7FE052159
:1057D0000CA013F005FA02E000200949088000BF80
:1057E000AAE70000080800203C0B0020B3080020B6
:1057F000B2080020D40C00206D0B0020690B0020A3
:10580000840B00204552524F520000002DE9F04118
:1058100086B005460E4617464FF00008002400BF2C
:105820001FE0A046C8EBC80000EB400000F5BC2814
:105830001522414668461BF0F7FFDDF80100A8423B
:105840000DD19DF80000B04209D1102300220DF1C6
:105850000501384600F04AFD06B0BDE8F081601C45
:1058600084B2064800888442DBDB1023002204A1B6
:10587000384600F03BFD00BFEEE70000FC0B0020C7
:105880002020202020202020202020202020202018
:10589000000000001CB50822694607200AF036FD0A
:1058A0009DF800404FF6FF7000EA04249DF80100C7
:1058B000044324119DF8060000F0100008B10020F8
:1058C0001CBD9DF8010000F00F00022801DA002045
:1058D000F6E7B4F58C7F05DB40F6E760844201DC37
:1058E0000020EDE70120EBE701463220B1FBF0F0AC
:1058F000322300FB03F2881A192801D210467047A0
:1059000002F13200FBE7000010B504460F48407872
:1059100000EB40000E4A02EB00100078810920469F
:1059200000F018F880B10948407800EB40000849C1
:1059300001EB0010C0F805400448407800EB40003F
:1059400001EB0010C0F8094010BD0000BB2D002085
:10595000EA2D0020F0B502460E4600210023002566
:1059600000241C48824208D31B48824202D91B48AB
:10597000824202D31A48824201D90020F0BD0021A0
:105980001FE001EB81071748C05D022815D101EB2C
:10599000810714483844B0F801501348454301EBDF
:1059A000810710483844B0F803400F484443AA42E6
:1059B00005D3A24203D80120E0E7581CC3B2481C1B
:1059C000C1B20429DDDB042B01D10120D6E7002080
:1059D000D4E7000040771B00800BB20300BD010537
:1059E00000E1F505492A0020A086010002460021B9
:1059F00000BF09E0064800EB41000088904201D159
:105A000001207047481CC1B22029F3DB0020F8E7D1
:105A10004DA3002010B50BF079FC4F4948704F485A
:105A2000807F20B108464078112800D110BD4FF486
:105A300080514B481BF06FFC002834D14948007856
:105A4000032824D1444840784349097888421ED02D
:105A50004148407810280FDA3F480078102806DBCC
:105A600001204149087017F0B5FEFEF7CDF93A491B
:105A70004878FEF745F90AE037480078102806DA3A
:105A8000002039490870FEF7AFF800F0F7FA324805
:105A9000407831490870FF2088700020C870087174
:105AA000A1F80500C2E72C484078FF2809D02A4811
:105AB000007930B92848B0F80500401C2649A1F803
:105AC000050025484078FF281FD12348B0F805007D
:105AD0000A2806DD204800781F4988700120C87018
:105AE00001E00DF09FF800201B490871A1F80500A6
:105AF0001E48007800B36422022140F25C600FF07F
:105B0000DBF800201949087016E013484078124964
:105B10000978884210D11048B0F80500B0F52F7F01
:105B20000ADD0D4800780C4988700220C8700120F9
:105B300008710020A1F80500074800780649497857
:105B4000884206D004484078034908700020A1F834
:105B5000050000BF6AE70000570B0020BB2D0020A6
:105B6000000002406D0B0020740B00208D0C002003
:105B70002DE9F04186B04FF000080027142299A1CA
:105B800001A8FDF734F8002400250026FEF7F6FCF6
:105B9000074699480078002861D19FB99749088045
:105BA0009748007801280CD1964801780078401C6D
:105BB000944A1070142904DD0020914908701146A0
:105BC00008700CE1904800780B280FD08F480078BF
:105BD0000B2803D18C480078082807D08748018813
:105BE0000088401C854A10800529EADD0020834991
:105BF000088083480078012803D103208049087079
:105C0000EDE081480078022807D08048007802281B
:105C100010D17D48007808280CD1794800780428F4
:105C200008D16422022140F25C600FF045F80320A5
:105C3000734908707648007858B9734800780B2883
:105C400007D0724800780B2806D16F4800780828E2
:105C500002D103F051FCC2E003F020FEBFE05FB9C7
:105C6000664801880088401C644A10800129A8DD2C
:105C7000002009F0A3FAB2E06648008828B1654820
:105C80000088001F63490880A6E063480078002868
:105C9000FAD1624890F8A9005E4908800846008859
:105CA00000EBC00101EB00104FF6FF7101EA80002C
:105CB00058490880594890F8160100284ED0584895
:105CC000007870BB4C480078022847D155480068DE
:105CD0000079C0F3420020BB52480068807B000975
:105CE000F8B9FEF717FB06464F480078D0B94D4883
:105CF00000680079800918B94C48007886420ADCAF
:105D00004848006800790121B1EB901F26D148482E
:105D10000078864222DD0020FDF700FC0120424988
:105D200008701BE03F4800680079800920B93F48AF
:105D300000780A38B0420BDA3A480068007901214D
:105D4000B1EB901F0AD13A4800780A38B04205DB1F
:105D50000120FDF7E3FB002033490870FEF722FB2A
:105D600004466410A72C02DD4FF0000803E0C4F1E4
:105D7000A70000F0FF080321404612F0D9FB0723DB
:105D800000222CA12D4800F0B1FA032301222C4956
:105D90002A4800F0ABFA214890F8A90010B9012078
:105DA00028498871002506E001A8405DA04200DD79
:105DB00003E0681CC5B2122DF6DB00BF2248057057
:105DC000007800EB4000214A81180323002220487C
:105DD00000F099FA17F04EFA00200849088006B042
:105DE000BDE8F081141C202C3038444C545C646CA9
:105DF000747C848C949C00006D0B0020800B002030
:105E0000D40C0020820B0020B3080020B208002030
:105E1000770B00201A0C002032080020BB2900203C
:105E2000690B00203C0B00201E0C002016080020EF
:105E3000170800202D30303044424D00D809002092
:105E4000D0240020EB240020190C00200D72020841
:105E5000C30800201FB5FF203A4981F83C001023F9
:105E6000002239A137483D3000F040FA10230022CB
:105E700035A134484D3000F039FA1022002168462F
:105E800000F0DAF830A135A00CF0DAFE10226946F5
:105E900037480CF01DFF01230022022135480CF089
:105EA00089FE002027498875012014F0B1FF0122E6
:105EB0000721002014F072FF3CE012F0F9FE19F007
:105EC000C9FC19F0C5FF19F07BFD2B48007820B9FB
:105ED000012029490870FFF79DFD2848008828B94E
:105EE0004FF4FA70254908801AF078F924480088A0
:105EF00028B94FF47A702249088019F073FB2148C1
:105F00008078112812D01F48807812280ED01D48A2
:105F10008078FF280AD01B4882781549154812F06E
:105F200069FFFF2013494875164988700DF0DAFBA8
:105F30000EF0C6F9102214490D4800F0B7F80028F9
:105F4000BBD01FBD830A002020202020202020203D
:105F500020202020202020200000000050617373AA
:105F6000776F7264203A202020202020000000005B
:105F70001420002020210020F10B0020F60B00202F
:105F8000F80B0020570B0020D729002030B5014620
:105F90000022002400231648814204D31548814280
:105FA00001D8002030BD00221DE002EB820512481E
:105FB000405D012815D102EB82050F482844B0F856
:105FC00001400E48444302EB82050B482844B0F8D8
:105FD00003300A484343A14203D3994201D8002029
:105FE000E0E7501CC2B2042ADFDB0120DAE7000040
:105FF00080CBA4000085CF00492A0020A0860100A4
:1060000010B500240AF09CFA00BF05E004F5937077
:106010001BF088FC601CC4B2082CF7DB0AF0B6FA4F
:106020000020034908800349C88014F077FC10BDA4
:106030000C0C0020BB2D002030B50346002000BF13
:1060400004E0FF240D185C55441CA0B29042F8DB1C
:1060500030BD00000146002009B9012200E00A46D7
:10606000104605E00022044B23F81020421CD0B259
:106070000828F7DB7047000018A3002010B50020A7
:10608000FEF751FC00210120FEF756FC402014F0E1
:106090005BF904480078022803D04FF4807002496D
:1060A000086010BD6D0B00201814024030B5034687
:1060B0000C46002100BF07E0585C655CA84201D097
:1060C000002030BD481C81B29142F5DB0120F8E789
:1060D00070B506460D46002400BF11E00B4800785D
:1060E000001BA84201DA002070BD094908192A46A0
:1060F0003146FFF7DBFF012800D1F5E7601CC4B291
:10610000024800788442E9DB0020EDE71D0800200A
:106110001E0800202DE9FC4F06468B469146584646
:10612000FDF7E4F982464FF000080025002400271F
:1061300027A103C9CDE9000100BF05E0705D0A2871
:1061400000D103E0681CC5B2C82DF7DB00BF681C96
:10615000C5B205E02819305C0DF80400601CC4B21B
:106160002819305C2C2801D0082CF3DB2146684626
:1061700017F09AFB80466FF07F40804502D3FF20E6
:10618000BDE8FC8FC24519D1601CC4B2002706E0EF
:1061900028193844305C09F80700781CC7B2281960
:1061A0003844305C0A2801D0642FF1DB2C223846B9
:1061B000791CCFB209F800200020E1E7C24501D9DF
:1061C0000120DDE7C24501D20220D9E7FF20D7E751
:1061D00030303030303030302DE9F041064600BFED
:1061E000374635460AF0ACF9C7EBC70000EB400074
:1061F00000F5BC27C5EBC50000EB400000F5BC2056
:10620000000B050341F21502294636481BF00CFB32
:10621000781B84B206E0334904F11500085C085588
:10622000601C84B2B4F5805FF5DB280B1BF07AFBB1
:106230004FF4805229462B481BF01AFC05F5805577
:106240001CE041F21502294626481BF0EDFA002415
:1062500006E0244904F11500085C0855601C84B26E
:10626000B4F5805FF5DB280B1BF05CFB4FF480522C
:1062700029461C481BF0FCFB05F58055B5F5112F90
:10628000DFD34FF48052294616481BF0CDFA002484
:1062900006E0144904F11500085C0855601C84B23E
:1062A00040F6EB708442F4DB002406E0FF2104F6A4
:1062B000EB700C4A1154601C84B2152CF6DB280BD1
:1062C0001BF030FB4FF48052294606481BF0D0FBF0
:1062D00005480088401E044908800AF057F9BDE8C7
:1062E000F0810000BE2E0020FC0B002070B504469B
:1062F000002000BF04E00D5C1618A555451CA8B28F
:106300009842F8DB70BD70B50446002000BF04E081
:106310000D5C1618A555451CA8B29842F8DB70BD57
:1063200010B5002101201AF05DFE012108461AF087
:106330003BFE10BD10B5002102201AF053FE0121D2
:1063400002201AF031FE10BD10B50446E0786178E5
:10635000024A50546078C12802D202E076740020CC
:1063600058E28100794449688F440000BA0800006F
:106370000403000006030000080300000A030000F5
:10638000200300003E030000B2030000BA08000032
:10639000AA04000004050000CA050000CC050000A6
:1063A000CE050000D0050000BA080000D2050000AC
:1063B000BA080000D4050000D6050000D80500008A
:1063C000DA050000DC050000DE050000E005000045
:1063D000E2050000E4050000BA080000BA08000069
:1063E000BA080000BA080000BA080000BA080000A5
:1063F000BA080000E6050000BA080000E805000041
:10640000EA050000BA080000580600005A0600001D
:10641000BA0800005C0600005E060000600600008E
:106420006206000064060000BA080000660600006C
:10643000BA080000BA080000BA08000068060000A8
:106440006A0600006C0600006E0600007006000080
:10645000BA0800007206000074060000760600000C
:10646000780600007A0600009A0600009C060000EC
:106470009E060000A0060000AC060000AE0600006C
:10648000B0060000B2060000B4060000B606000028
:10649000B8060000BA060000BC060000BE060000F8
:1064A000C0060000C2060000C4060000C6060000C8
:1064B000C8060000CA060000CC060000CE06000098
:1064C000D0060000D2060000D4060000D606000068
:1064D000D8060000BA080000BA0800005208000000
:1064E0005408000056080000BA08000058080000D0
:1064F0005A0800005C08000084080000BA08000088
:10650000BA0800008608000088080000BA080000E9
:10651000BA080000BA080000BA080000BA08000073
:10652000BA080000BA080000BA080000BA08000063
:10653000BA080000BA080000BA080000BA08000053
:10654000BA080000BA080000BA080000BA08000043
:10655000BA080000BA080000BA080000BA08000033
:10656000BA080000BA080000BA080000BA08000023
:106570008A0800008C0800008E08000090080000C7
:10658000920800009408000096080000BA08000075
:10659000BA080000BA080000BA080000BA080000F3
:1065A000BA080000BA080000BA080000BA080000E3
:1065B000BA080000BA080000BA080000BA080000D3
:1065C000BA080000BA080000BA080000BA080000C3
:1065D000BA080000BA080000BA080000BA080000B3
:1065E000BA080000BA080000BA080000BA080000A3
:1065F000BA080000BA080000BA080000BA08000093
:10660000BA080000BA080000BA080000BA08000082
:10661000BA080000BA080000BA080000BA08000072
:10662000BA080000BA080000BA0800009808000084
:106630009A0800009C0800009E080000A0080000C6
:10664000A2080000A4080000A6080000A808000096
:10665000AA080000AC080000AE080000B008000066
:10666000B2080000B4080000B6080000B808000036
:1066700000BF00BFD7E2FE480078022805D1207A8B
:10668000032802D16F20FB490870CCE2FA48407918
:1066900050B9207AF9490978884205D0207AF7491B
:1066A00008700120F6490870BDE2E078F5490870ED
:1066B00008460078EF490870207A012803D10020AD
:1066C000F14908700CE0207A022803D10120EE493C
:1066D000087005E0207A042802D10220EA490870F7
:1066E00004F10D000AF0E8FDE749C1F8010004F1EA
:1066F00009000AF0E1FDE449C1F80500E34800782B
:1067000060B9E349096849780809022111F010FFCE
:1067100002230322DF49E048FFF7E8FD83E2A07887
:1067200010B9E078DD490870A078022872D1002005
:10673000DB4908700220DB4908700020087306233B
:106740000022D949D748801DFFF7D0FDD7484078AF
:1067500000EB4000D64901EB0010D0F80500D1490C
:10676000C1F80E00207A012809D10020487004F1F8
:1067700009000AF0A1FDCB49C1F8020016E0207A19
:10678000022806D1C74948704FF0AA30C1F802006C
:106790000CE0207A092809D10120C249487004F18F
:1067A00009000AF089FDBF49C1F80200A0220021BA
:1067B000BC483830FFF740FC607BA02815DDBD48A1
:1067C00090F89701012807D0B64A3832A02104F189
:1067D0000E0019F04BFF1DE0A023002204F10E0172
:1067E000B0483830FFF782FD14E0B24890F89701C6
:1067F000012807D0617BAB4A383204F10E0019F052
:1068000035FF07E0637B002204F10E01A548383014
:10681000FFF76CFD07E2E078A7490870A07802282E
:1068200025D19348007810BBA4480078F8B9A44853
:106830000078E0B9A3480078C8B90120A2490870DF
:106840000020A24908704FF44870A1490880002038
:10685000A04908709E480088FEF742FA022014F012
:1068600089FE9DA3A1A26421002004F025FBDAE1AA
:10687000A07818B9E078A24908705BE0A0780228F7
:1068800058D1E0789E49087008460078A12805D1C3
:1068900091A39CA2C821002004F00EFB854890F82B
:1068A0008401002846D096480078A2280FD1042001
:1068B0009949087044F244407E49888114F020F8D8
:1068C0004FF4FA6001F03FF813F060FD32E08C48BD
:1068D0000078A3281BD14AF6CD30764988818E48AE
:1068E000007808B114F00CF88B480078042805D122
:1068F0004FF4FA6001F027F813F048FD00208649B4
:10690000087075A385A2C82104F0D6FA12E07C486D
:106910000078A4280ED103207F49087043F2333059
:106920006449888113F0ECFF6BA381A2C821002089
:1069300004F0C2FA77E100BF00BF00BF73E172E16B
:1069400000BF00BF00BF00BF00BF00BF00BF00BF4F
:1069500000BF00BF67E1484890F8250088BB207A57
:10696000302101EB201077490870207A00F00F00E9
:10697000303048702E208870607A302101EB201072
:106980007049C870607A00F00F00303008712E2016
:106990004871A07A302101EB20106A498871A07AF1
:1069A00000F00F003030C8712E200872E07A3021DC
:1069B00001EB201063494872E07A00F00F0030309C
:1069C000887230E100BF00BF00BF00BF00BF00BF42
:1069D00000BF00BF00BF00BF00BF00BF00BF00BFBF
:1069E00000BF00BF1FE1A0783E2803D10120564917
:1069F000087007E0A0783F2804D1E07810B90020A3
:106A0000514908700FE100BF00BF0CE1E07810B9F8
:106A100001204D49087006E100BF00BF00BF00BF64
:106A200000BF00BF00BF00BF00BF00BF00BF00BF6E
:106A300000BF00BF00BF00BF00BF00BF00BF00BF5E
:106A400000BFF0E00A480078022805D1207A01282A
:106A500002D16F20074908700548007830B9207AC4
:106A6000012803D139490870124871E088E000001C
:106A70006E0B00203D0C0020767400204D0C002091
:106A80004E0C00203C0C0020C27D0020500C002049
:106A90003C0B0020D0240020B7090020400C00202F
:106AA000410C0020C5A60020400B0020BB2D00207B
:106AB000EA2D0020BB290020380C00206A0B0020A2
:106AC0006B0B0020680B00203B0C0020D00C00203A
:106AD000CE0C00208E0B0020202020202020202003
:106AE000202020202020202000000000456D65721D
:106AF00067656E637920416C61726D200000000053
:106B0000390C00204265696E6720536561726368C5
:106B10006564202000000000120C002052616469AE
:106B20006F2057616B652055702020200000000009
:106B3000444D522052656D6F7465205374756E20FC
:106B400000000000420C00203F0C00204F0C0020F1
:106B500090F8540318B14FF48040344988614FF4E1
:106B6000FA703349088033480068C078C0F3411098
:106B7000012805D13048007840F004002E49087003
:106B80002E480078A8B1207A98B900202B490870C7
:106B900028480068C078C0F34110012805D1264874
:106BA000007820F00400244908704FF480401F4909
:106BB0008862207A10B900202149087033E000BFB4
:106BC00000BF00BF00BF2EE0E0790A280FD11C48AB
:106BD000007860B901201A490870607C022111F028
:106BE000A7FC0223032217491748FFF77FFB1AE08F
:106BF00000BF00BF00BF00BF00BF00BF00BF00BF9D
:106C000000BF00BF00BF00BF00BF00BF00BF00BF8C
:106C100000BF00BF00BF00BF00BF00BF00BF00BF7C
:106C200000BF00BF00BF00BF10BD00000000024059
:106C3000240C00203C0B00206F0B00204F0C002088
:106C4000500C0020D0240020B70900203EB5054696
:106C50000C46002002908DF808508DF80940642001
:106C600002A904230122CDE900101146492014F0A5
:106C700029FA3EBD08B56420022301221146009086
:106C8000052014F0DFF908BD08B5642001231A4679
:106C900019460090252014F0D5F908BD70B50546B9
:106CA0000E46002404E0285D00F006F8601C84B263
:106CB000B442F8DB70BD000010B504460C48007803
:106CC00050B10C480088C0F30B000B490C54094824
:106CD0000068401C07490860214608481BF0E8F896
:106CE00000BF802105481BF0ECF80028F9D010BD4A
:106CF000670B0020640C0020EF9200200048004049
:106D000070B58AB005460C462646002002900390D6
:106D10002E490870C6EBC60000EB400000F5BC260B
:106D20001522314604A81AF07FFD9DF810000228B4
:106D300007DD27A32BA2C821012004F0BDF80AB06B
:106D400070BD9DF8100020B1012806D002280CD19A
:106D500007E001208DF8080007E002208DF8080008
:106D600003E004208DF8080000BF00BFDDF811002B
:106D7000000E8DF80900DDF81100000C8DF80A00F6
:106D8000BDF81100000A8DF80B009DF811008DF878
:106D90000C004FF47A7002A905232A46CDE90010B1
:106DA0000121062014F08EF99DF810001249087098
:106DB000DDF81100C1F80500102300220DF11501C6
:106DC0000D480930FFF792FA00BFB8E73E0C0020EB
:106DD00063616C6C2073746F707065642E2020206A
:106DE0000000000043616C6C20747970652065724E
:106DF000726F722C00000000A97D002010B588B0D1
:106E0000044620220FA16846FBF7F1FE8DF80840EA
:106E1000FF20144981F85D001F216846FFF73EFFFF
:106E20000A201149088001E0FCF712F90D4890F89A
:106E30005D00FF2803D10C4800880028F4D108B079
:106E400010BD0000685D010100000016010AFFC8C6
:106E50000128FF140250FF140350FF140450FF14C4
:106E60000550100076740020520C00202DE9FF41DF
:106E700006460F4615461C46002002900390284601
:106E800000F0F4FC05463E480670012F04D0022FA6
:106E900027D0042F50D13DE001208DF808000020BC
:106EA000384908700846C0F8055034B9102300224C
:106EB00035A10930FFF71AFA12E0012C07D110238F
:106EC000002236A12F480930FFF710FA08E0022C03
:106ED00006D11023002236A12A480930FFF706FA0E
:106EE0002AE002208DF80800012026490870084693
:106EF000C0F8055034B91023002223A10930FFF750
:106F0000F5F906E01023002224A11E480930FFF7FE
:106F1000EDF911E004208DF80800022019490870ED
:106F20004FF0AA30C1F805001023002225A1154812
:106F30000930FFF7DBF900BF00BF1248D0F80500A9
:106F4000000E8DF809000F48D0F80500000C8DF8F0
:106F50000A000C48B0F80500000A8DF80B0009483B
:106F600040798DF80C004FF47A7002A9052332465F
:106F7000CDE900100121062014F0A4F8BDE8FF813E
:106F80003E0C0020A97D00204469616C696E672079
:106F900020202020202020200000000043616C6C75
:106FA0006261636B20202020202020200000000050
:106FB00041646472657373626F6F6B2020202020C0
:106FC00000000000416C6C2043616C6C202020208C
:106FD000202020200000000070B58AB005460C4635
:106FE0002646002002900390C6EBC60000EB40004E
:106FF00000F5BC261522314604A81AF015FC9DF8B0
:10700000100040B115A31AA2C821002003F054FFBC
:1070100000200AB070BD8DF80850DDF81100000E98
:107020008DF80900DDF81100000C8DF80A00BDF89C
:107030001100000A8DF80B009DF811008DF80C006E
:107040004FF47A7002A905230122CDE90010114600
:107050000A2014F037F80120DBE700002020202070
:1070600020202020202020202020202000000000A0
:10707000436F6E74616374204572726F72212020B9
:107080000000000070B5ACB0054600240026A52223
:10709000002102A8FEF7D0FF002D33D13D4890F823
:1070A0009701012815D100BF0EE03B48005DFF2885
:1070B00002D03948005D00B908E03748015D601D25
:1070C00002AA1154601CC4B2A02CEEDB00BF661DE6
:1070D00024E0002409E03048005DFF2802D02E485B
:1070E000005D00B903E0601CC4B2A02CF3DB00BF5C
:1070F0000DF10D022146284809F0C0FA0646701D20
:1071000086B20BE0002406E02348015D601D02AA60
:107110001154601CC4B2912CF6DB96261E483838F8
:10712000407820B1012806D002280CD107E00120C8
:107130008DF8080007E009208DF8080003E0022020
:107140008DF8080000BF00BF13483838D0F802009F
:10715000000E8DF8090010483838D0F80200000CF5
:107160008DF80A000C4838384088000A8DF80B006A
:107170000948383880788DF80C0040F6B83002A9FC
:1071800033460122CDE900101146072013F09AFF83
:107190002CB070BDBB290020FDA500203EB50446E3
:1071A00009A00068029001208DF808008DF80940C0
:1071B000642002A902230122CDE9001011464920D2
:1071C00013F080FF3EBD00000100000038B504460A
:1071D00064202346012211460090452013F032FF1F
:1071E00038BD3EB505460C46002002908DF808508B
:1071F0008DF80940642002A902230122CDE9001084
:107200001146622013F05EFF3EBD000070B58EB0E7
:107210000446142103A8FBF71CFD00BFB4F811605D
:10722000D4F805004E49884203D301204D49087027
:1072300002E000204B4908702078C0F34000401C59
:107240008DF80C00607800098DF80D002078C0F3EF
:1072500080008DF80E00D4F8050000EB800045009A
:10726000280E8DF80F00280C8DF81000280A8DF8D4
:107270001100E8B28DF81200D4F8090000EB80008C
:107280004500280E8DF81300280C8DF81400280AEC
:107290008DF81500E8B28DF81600C6EBC60000EBBD
:1072A000400000F5BC261522314608A81AF0BCFAA9
:1072B0009DF8200020B1012806D002280CD107E05B
:1072C00001208DF8170007E002208DF8170003E079
:1072D00004208DF8170000BF00BF9DF81700042898
:1072E00013D0DDF82100000E8DF81800DDF8210024
:1072F000000C8DF81900BDF82100000A8DF81A0065
:107300009DF821008DF81B0008E0AA208DF81800D8
:107310008DF819008DF81A008DF81B0000208DF8EB
:107320001C001148006880780121B1EB901F01D149
:10733000012000E000208DF81D0000208DF81E00C7
:10734000207D8DF81F00642003A914230122CDE9BC
:1073500000101146822013F0B5FE0EB070BD000083
:1073600000366E01340C00203C0B00202DE9F0416A
:1073700098B00446002700250226A84622220021B4
:1073800003A8FEF759FE0CB900BF29E0A4F10108DB
:1073900008EB48004FF4502202EB001130220CA8F9
:1073A0001AF042FA9DF8310020B1012805D00228D8
:1073B00009D105E00127072605E00427122602E08F
:1073C0000527222600BF00BF002506E010A8415D6A
:1073D000A81C03AA1154681CC5B2B01EA842F5DC53
:1073E000E0B28DF80C008DF80D70642003A93346CF
:1073F0000122CDE900101146812013F063FE18B080
:10740000BDE8F081F0B5BDB006460025002481221C
:10741000002102A8FEF710FE374607EB87004FF465
:10742000462101EB00175022394629A81AF0FCF931
:1074300000BF3CE02DA830F8150042F210718842E0
:1074400033DA2DA830F81570C7EBC70000EB400009
:1074500000F5BC271522394623A81AF0E5F99DF856
:107460008C00012821D19DF88D1000EB8400C01CF8
:1074700002AA1154BDF88D00C0F30721012000EBD2
:107480008400801C1154DDF88D00C0F307410120F9
:1074900000EB8400401C1154DDF88D00000E01212A
:1074A00001EB84015054601CC4B2681CC5B2202D8D
:1074B000C0DB8DF80840642002A9CDE9001001204E
:1074C00000EB840302460146842013F0FBFD3DB02F
:1074D000F0BD3EB505460C46002002908DF80850E0
:1074E0008DF80940642002A902230122CDE9001091
:1074F0001146572013F0E6FD3EBD3EB50446002080
:107500000290E0B28DF80800200A8DF80900200CE6
:107510008DF80A00200E8DF80B00642002A90423C8
:107520000122CDE9001011462A2013F0CBFD3EBD0B
:1075300038B50446642023460122114600900B20F2
:1075400013F080FD38BD00000EB50EA207CA8DE80D
:107550000700FF200E4981F884000A216846FFF7E2
:107560009DFB0A200B49088001E0FBF771FD0848EC
:1075700090F88400FF2803D1064800880028F4D141
:107580000EBD000068840101000000010010000031
:1075900076740020520C002038B504460D46012DAB
:1075A00008D1642000230122114600900C2013F022
:1075B00049FD07E0642023460122114600900C207B
:1075C00013F040FD38BD38B504466420234601223F
:1075D00011460090482013F035FD38BD38B50446FB
:1075E00064200090601CC3B201221146552013F0A4
:1075F00029FD38BD38B504466420234601221146D2
:1076000000904D2013F01EFD38BD38B504466420AF
:107610002346012211460090022013F013FD38BDCD
:107620000EB50EA207CA8DE8070000200E490870AB
:107630000A216846FFF732FB14200C49088001E05C
:10764000FBF706FD0848007818B9084800880028AC
:10765000F6D10120044908700EBD00006842010106
:1076600000000001FF1000003F0C0020520C002021
:1076700038B50446642023460122114600904C2070
:1076800013F0E0FC38BD000000B587B0182208A157
:1076900001A8FBF7ACFA01200B490870182101A8DA
:1076A000FFF7FCFA00200849087007B000BD000091
:1076B000683E01010000000F0F0F0F0F0F0F0F0F9B
:1076C0000F0F0F0F0F0F0F103F0C002038B504469F
:1076D00064202346012211460090092013F0B2FCD9
:1076E00038BD000010B5022019F03AFD28B1022083
:1076F00019F026FD01200149088010BD9E080020D8
:1077000000B585B01C4819F07BFD684619F00BFDEB
:107710000120ADF80A000020ADF8080017480190DC
:1077200001208DF80F008DF80D0015480090012004
:107730008DF80E0000208DF80C0002208DF811004D
:1077400001208DF8100069460B4819F01FFD01213A
:107750000948083819F08CFD05210748FC3019F05C
:107760008EFD00220221044819F041FD012102484A
:1077700019F0D4FC05B000BD086002409C08002050
:107780004C20014070B504460D460F2C03DC20460A
:107790000BF0B2FB70BD102C0CD0112C02D0122CAF
:1077A00017D100E000BF642202214FF4DC700DF01D
:1077B00083FA0EE00848007840B912F017FF502213
:1077C00004214FF4DC700DF077FA01E000F03CF991
:1077D00000BF00BF00BFDDE7AD0C002030B50346A1
:1077E00014460022002000BF20E09D5C2D090D54AE
:1077F0000D5C0A2D03DA0D5C30350D5402E00D5C92
:1078000037350D54451CE8B29D5C05F00F050D544D
:107810000D5C0A2D03DA0D5C30350D5402E00D5C71
:1078200037350D54451CE8B2551CEAB2A242DCDBE8
:1078300030BD0246002000BF13E0C0F107039B00EB
:1078400022FA03F303F00F030B540B5C0A2B03DA49
:107850000B5C30330B5402E00B5C37330B54431C8E
:10786000D8B20828E9DB704770470000014600BF26
:1078700000BF234BB1FBF3F210460001DB11534371
:10788000A1EBC3111F4BB1FBF3F2104400019B119C
:107890005343A1EB83111C4BB1FBF3F210440001E5
:1078A0005B115343A1EB431142F21073B1FBF3F2AE
:1078B000104400011B115343A1EB03114FF47A73E1
:1078C000B1FBF3F21044000102EB4203C3EBC2131D
:1078D000A1EBC3016423B1FBF3F21044000102EBFE
:1078E000C20303EB0213A1EB83010A23B1FBF3F202
:1078F0001044000102EB8203A1EB430108447047EE
:107900008096980040420F00A08601000146C1F316
:10791000821000EB80024FF6FF7303EA4200C1F3CE
:10792000C202104400EB800203EA420001F00702A9
:107930001044704701E000BF00BF011EA0F101022A
:10794000D0B2F8D1704770B50446002509E04FF475
:10795000FA7019F083FB43F2C82019F0B7FB681CDA
:1079600085B24FF4FA7094FBF0F0A842EFDC4FF4CC
:10797000FA7094FBF0F100FB114086B2304619F02A
:107980006DFB70BD2DE9F047044600260025A84692
:10799000B4F80271A94694F8000110B10020BDE8C6
:1079A000F087002084F80401B4F802112046FDF7A6
:1079B000C5FD06460C21204610F0B2F981460EB1F5
:1079C000012E13D13D4604E0681C205C6055681C04
:1079D00085B2B4F80601401EA842F5DCFF206055D0
:1079E000B4F80601401EA4F8060116E0781E85B220
:1079F00004E0A81C205C6055681C85B2B4F8060140
:107A0000801EA842F5DCFF206055FF21681C215430
:107A1000B4F80601801EA4F80601B9F1000F0CD1DC
:107A2000204601F0EBF820460AF0F2FC80460120E7
:107A300003494871034880F814800120AFE7000033
:107A4000F4240020830A002010B513480078401E5B
:107A500000F00F00104908705F2010490E4A12789C
:107A600088540D4800780F2805D020210B4A0A4879
:107A70000078401C11541023002208490848FEF7E2
:107A800035FC012013F044F9502204214FF4DC703E
:107A90000DF012F910BD0000AD0C0020AE0C00205E
:107AA0003509002010B5164800680A21B0FBF1F036
:107AB0001349086013480078C01D00F00700114901
:107AC00008705F2010490F4A127888540D480078DA
:107AD000072805D020210C4A0A480078401C115480
:107AE0000823002208490948FEF700FC012013F092
:107AF0002BF9502204214FF4DC700DF0DDF810BD9D
:107B0000A80C00209D0C00209F0C00205F09002085
:107B100070B504460D46012D76D10A2C06D00E2CE8
:107B200045D00F2C66D0102C2AD12AE05848007876
:107B3000042806D0642202214FF4DC700DF0BCF85A
:107B400070BD0021534842781430815412F0E6FE93
:107B50005049497801EB41014F4A02EB01103023B3
:107B600000224E49FEF7C2FB4A49487812F07AFFDC
:107B700007F00EFD502203214FF439700DF09CF8F0
:107B80005EE043480078042803D145480078012886
:107B900002D107F0FDFC03E04148007802F072F9E1
:107BA000502204214FF4DC700DF086F848E03C4888
:107BB000007808B9012000E0002039490870084623
:107BC000007802F05FF970B900203549087035A3DC
:107BD00039A2642103F070F9642202214FF4DC70B1
:107BE0000DF06AF805E06422022140F25C600DF0BD
:107BF00063F825E02A48007838B1642202214FF466
:107C0000DC700DF059F89BE71BE0304890F810014C
:107C1000062804D006202D4981F8100103E0022037
:107C20002A4981F810011E48007802F02BF912F061
:107C300067FE6422022140F25C600DF03DF800BF57
:107C400023E00F2C21D11648007830B164220221A4
:107C50004FF4DC700DF030F872E71C4890F810011A
:107C6000401C0B2190FBF1F201FB1200174981F837
:107C700010010B48007802F005F912F041FE642271
:107C8000022140F25C600DF017F800BF58E70000D9
:107C9000D40C0020BB2D0020EA2D00204A2E00200D
:107CA000D50C002020202020202020202020202053
:107CB00020202020000000004E6F20416E616C6F7C
:107CC000672043482020202000000000BB2900201E
:107CD00070B504460D46092C03DC20460BF04CF928
:107CE00070BDA4F10A00092832D2DFE800F00812C2
:107CF000090A0B071505060000BF00BF00BF00BF43
:107D000000BF00BF642202214FF4DC700CF0D4FFEE
:107D10001EE000F025F81BE00F480078042806D18B
:107D2000642202214FF4DC700CF0C6FFD8E70B4848
:107D3000007850B9FDF7E4F912F058FC5022042104
:107D40004FF4DC700CF0B8FFCAE7FFF7ABFE00BFE2
:107D500000BF00BFC4E700009E0C00209D0C002067
:107D600010B5FDF7CDF91F480078012809D1022090
:107D70001C4908700A2300221BA11E48FEF7B6FA10
:107D800026E018480078022819D104201549087007
:107D90000A23002218A11748FEF7A8FA082019495B
:107DA00008700823002218A11A48FEF79FFA08233A
:107DB000002218490F480A30FEF798FA08E001201F
:107DC000084908700A23002213A10A48FEF78EFA18
:107DD000012012F0B9FF6422022140F25C600CF035
:107DE0006BFF10BD9E0C002047726F7570204361C1
:107DF0006C6C000055090020416C6C2043616C6C78
:107E0000202000009D0C00203136373737323135C5
:107E1000000000009F0C0020496E6469766964755B
:107E2000616C000010B50B48007838B90A4800684A
:107E3000B0F81110FF20FEF763FF07E000230748AA
:107E4000026807480178FF20FFF710F80020054975
:107E5000086010BD3E0C00203C0B0020A80C002048
:107E60009E0C0020E00B002070B504460D4629460C
:107E7000204610F075F870BD10B5044615F0D0FC22
:107E800015F0F4FC1E4890F88D0108B113F0FAFBD0
:107E90001C480078012803D180021B49886203E056
:107EA0004FF48060184988613CB918480068B0F800
:107EB00011100120FEF724FF1EE0012C08D1002341
:107EC00013480268134801780120FEF7CFFF13E042
:107ED000022C08D101231048026810480178184686
:107EE000FEF7C4FF08E0032C06D102230848012155
:107EF00002680846FEF7BAFF03200949087010BD62
:107F0000BB290020340C0020000002403C0B002064
:107F1000A80C00209E0C0020140C0020130C002044
:107F20006E0B002010B50AF031FE0AF039FE002079
:107F300015F002FD00BF02201A49086040F6B83073
:107F40001949088001E0FBF783F81848807E18B1D2
:107F5000154800880028F6D11448807E40B10220E0
:107F60001049103108604FF47A70FFF7ECFCE2E73B
:107F7000FEF78AFE00210846FFF7ABFA0220FFF762
:107F800025F90F20FFF71FFB0020FFF707F901205D
:107F9000FFF76EFB002006490870012005490870B4
:107FA00010BD000018040240520C0020767400201E
:107FB0005E0B0020730B00202DE9FF4180460D462B
:107FC00016461F46A6F12000C6B2C6EBC6004FF407
:107FD000CE1202EB40010E22684619F025FC012F5B
:107FE0001CD1002417E01DF80400C043C0B20DF8F6
:107FF000040004F0010030B91DF8040000F0FE0098
:108000000DF8040005E01DF8040000F07F000DF8F5
:108010000400601CC4B20E2CE5DB0DE0022F0BD176
:10802000012407E01DF8040040F080000DF8040072
:10803000A01CC4B20E2CF5DB002418E02819C1B234
:1080400040460CF01BFD1DF814000CF06DFD2A19C4
:10805000D1B208F10102D0B20CF010FD012101EB08
:1080600044011DF801000CF05FFD601CC4B2072C38
:10807000E4DBBDE8FF81F0B58BB006460D46174640
:10808000A7F12000C7B2C7EBC7004FF4CE1202EB36
:1080900040010E2207A819F0C7FB072201A907A873
:1080A000FDF762F9002426E02819C1B230460CF031
:1080B000E5FC04EB440101AA505C0CF035FD2A19E3
:1080C000D1B2721CD0B20CF0D9FC04EB4401491CB3
:1080D00001AA505C0CF028FD2A19D1B2B21CD0B212
:1080E0000CF0CCFC04EB4401891C01AA505C0CF0A0
:1080F0001BFD601CC4B2072CD6DB0BB0F0BD00002A
:108100002DE9F0418AB006460D4617469846A7F17C
:108110002000C7B207EB4710204A8118212201A88E
:1081200019F082FBB8F1010F0AD1002406E001A882
:10813000005DC04301A90855601CC4B2212CF6DBC8
:10814000002426E02819C1B230460CF097FC04EB5D
:10815000440101AA505C0CF0E7FC2A19D1B2721C50
:10816000D0B20CF08BFC04EB4401491C01AA505C1A
:108170000CF0DAFC2A19D1B2B21CD0B20CF07EFCA1
:1081800004EB4401891C01AA505C0CF0CDFC601C7E
:10819000C4B20B2CD6DB0AB0BDE8F08132C51900A1
:1081A0002DE9F05F05468A4616461F4600244FEA31
:1081B000E60806F00709A346454504DB454504D11A
:1081C000B9F1000F01D0BDE8F09F002405E0802048
:1081D000204140EA0B0B601CC4B24C45F7DB002485
:1081E0000DE0291BC8B251460CF048FC0FB1FF212D
:1081F00000E0002108460CF097FC601CC4B2444526
:10820000EFDBB9F1000F0BD0291BC8B251460CF0BF
:1082100035FC0FB1594600E0002108460CF084FC03
:1082200000BFD0E72DE9F04106460C46002500BF0F
:108230005EE0C4F10101022202EB4101C8B229460D
:108240000CF01CFC00200CF06FFCC4F101010322B7
:1082500002EB4101C8B229460CF010FC00200CF0E2
:1082600063FCC4F10101042202EB4101C8B22946BA
:108270000CF004FC00200CF057FC022101EB44013F
:10828000C8B229460CF0FAFB16B11B48405D01E06C
:108290001A48405D074638460CF046FC032101EBC6
:1082A0004401C8B229460CF0E9FB1EB1E81D124991
:1082B000085C02E0E81D1149085C074638460CF0EE
:1082C00033FC042101EB4401C8B229460CF0D6FB73
:1082D00026B105F10E000849085C03E005F10E0027
:1082E0000649085C074638460CF01EFC681CC5B2FF
:1082F000072D9EDBBDE8F081825202086D52020814
:108300007FB5054615A30FCB8DE80F00012D0FD0CB
:10831000022D07D0032D11D1BD208DF804008DF85A
:10832000050000BFBD208DF807008DF8080000BFD4
:10833000BD208DF80A008DF80B0000BF00BF722130
:1083400000200CF09BFB002405E01DF804000CF05D
:10835000EBFB601CC4B20E2CF7DB7FBD3C3CFF8105
:10836000818181818181818181FF00002DE9F0413E
:1083700006460024002500BF1AE004F15800C1B2EF
:1083800005200CF07BFB2648075D38460CF0CCFB43
:1083900004F15800C1B206200CF070FBE01D20492A
:1083A0000F5CE11D1E4A505C0CF0BEFB601CC4B2A9
:1083B000072CE2DB00242FE0002529E005F1600016
:1083C00004EB84021044C1B205200CF057FB16B137
:1083D0001448405D01E01448405D074638460CF003
:1083E000A3FB05F1600004EB84021044C1B2062037
:1083F0000CF044FB1EB1681D0A49085C02E0681DD0
:108400000949085C074638460CF08EFB681CC5B26B
:10841000052DD3DB601CC4B2032CCDDBBDE8F0819D
:108420004B52020863520208595202082DE9F041EA
:1084300006460F461446394630460CF01FFB002511
:1084400004E018200CF070FB681CC5B2A542F8DBF4
:10845000BDE8F0812DE9F04387B080460E46154611
:108460001F46E8B240388121C1EB2521C1EB411202
:1084700002EB811100EB4109E8B27F2801DDA9F18F
:108480000109C9EBC9004FF4CF1202EB80011C2295
:10849000684619F0C9F9012F1CD1002417E01DF816
:1084A0000400C043C0B20DF8040004F0010030B96C
:1084B0001DF8040000F0FE000DF8040005E01DF8B2
:1084C000040000F07F000DF80400601CC4B21C2CF6
:1084D000E5DB0DE0022F0BD1012407E01DF80400BD
:1084E00040F080000DF80400A01CC4B21C2CF5DB89
:1084F000002418E03019C1B240460CF0BFFA1DF854
:1085000014000CF011FB3219D1B208F10102D0B203
:108510000CF0B4FA012101EB44011DF801000CF04C
:1085200003FB601CC4B20E2CE4DB07B0BDE8F08393
:108530002DE9F04192B007460D461646F0B240389C
:108540008121C1EB2621C1EB411202EB811100EB2D
:108550004108F0B27F2801DDA8F10108C8EBC8008E
:108560004FF4CF1202EB80011C220BA819F05CF92A
:108570000E2269460BA8FCF7F7FE002426E0281916
:10858000C1B238460CF07AFA04EB44011DF8010040
:108590000CF0CAFA2A19D1B27A1CD0B20CF06EFAD9
:1085A00004EB4401491C1DF801000CF0BDFA2A1926
:1085B000D1B2BA1CD0B20CF061FA04EB4401891CB0
:1085C0001DF801000CF0B0FA601CC4B20E2CD6DB12
:1085D00012B0BDE8F08110B5782204210120FFF728
:1085E00025FF782204210620FFF720FF042000F059
:1085F000DCFB7C2000F0D9FB10BD000070B5064606
:108600000C4615460A23002206F122010848FDF710
:108610006DFE2DB9FF200649313981F83B0003E09A
:108620000348313880F83B4001200249487270BD50
:10863000B40A0020F424002038B50446062C2DD2BC
:10864000DFE804F0030B141C24130120032319A2F8
:108650006B21009000F0FCF929E00120032316A211
:108660006B21009000F0F4F921E000BF012003230A
:1086700012A26B21009000F0EBF918E00120032317
:108680000FA26B21009000F0E3F910E0012003231A
:108690000CA26B21009000F0DBF908E0002003231E
:1086A00009A26B210090012000F0D2F900BF00BFA9
:1086B00038BD000041424300616263003132330043
:1086C00050593100505932002020200070B500264A
:1086D000002415E0A11CC8B228210CF0CFF9002518
:1086E0000AE004EB440005EB001007490E5C30463D
:1086F0000CF01AFA681CC5B2302DF2DB601CC4B253
:10870000062CE7DB70BD0000CD5202082DE9FC41CC
:1087100006460D460DA103C9CDE90001002400BFA6
:1087200010E004F17B00C1B230460CF0A7F915B19E
:108730001DF8040000E00020074638460CF0F4F96C
:10874000601CC4B2052CECDBBDE8FC813078FC3049
:108750003000000010B50446B4F80801102800DC11
:1087600010BDB4F80A0102210FF0E2FE07480078BC
:10877000074981F8280005484178054880F8291004
:1087800001200449C87100BFEAE70000D02400209E
:10879000830A0020F424002070B5002400BF15E0F7
:1087A000214601200CF06AF90A48055D28460CF0C4
:1087B000BBF9214602200CF061F904F10E000549D5
:1087C0000D5C28460CF0B0F9601CC4B20E2CE7DB3F
:1087D00070BD00009752020810B5002400BF08E0E9
:1087E000214603200CF04AF90C200CF09DF9601C86
:1087F000C4B2802CF4DB10BD70B50446002500BF68
:1088000032E0042101EB4401C8B229460CF036F9EC
:108810001748465D30460CF087F9052101EB44010D
:10882000C8B229460CF02AF9A81D11490E5C304641
:108830000CF07AF9C4F10101042202EB4101C8B243
:1088400029460CF01BF900200CF06EF9C4F101016F
:10885000052202EB4101C8B229460CF00FF90020B5
:108860000CF062F9681CC5B2062DCADB70BD0000B1
:10887000B35202082DE9FC4106460D460DA103C97D
:10888000CDE90001002400BF10E004F17B00C1B27B
:1088900030460CF0F3F815B11DF8040000E000209C
:1088A000074638460CF040F9601CC4B2052CECDBDE
:1088B000BDE8FC813030FC78300000002DE9F0414B
:1088C0000446002500266078C01EC7B20A23002295
:1088D00030A104F12200FDF709FD208A052190FB5B
:1088E000F1F000EB800086B287B9A08900EB800030
:1088F0002B4901EB4000C08800EB8000294901EBC7
:10890000400005896D0005F5CC150FE0A08900EB4E
:108910008000234901EB4000C08800EB8000224921
:1089200001EB400005896D0005F5C41505EB460512
:10893000618A701D814206DB0A22294604F1220069
:1089400018F072FF0DE0608A052190FBF1F201FB47
:1089500012004FEA40084246294604F1220018F06E
:1089600063FFA079042805D0002211462046FFF7B6
:1089700045FE0CE0208A052190FBF1F201FB12007C
:1089800000F0FF08012241462046FFF737FEBDE810
:10899000F081000020202020202020202020000026
:1089A0004C2100204A210208303102082DE9F0470D
:1089B00081468A4614461E460027B846202C01DB15
:1089C0007F2C00DD2024A4F1200087B207EB870074
:1089D00087B2514648460CF051F800250BE0084894
:1089E000384410F805800EB14FEA680840460CF094
:1089F0009BF8681CC5B2052DF1DBBDE8F0870000CF
:108A0000E44D02082DE9FC4105460E460EA103C9BE
:108A1000CDE90001002400BF11E005F1150020445C
:108A2000C1B207200CF02AF816B11DF8040000E0CE
:108A30000020074638460CF077F8601CC4B2052CBD
:108A4000EBDBBDE8FC8100000406FF06040000002B
:108A50002DE9F05F82460F4615469B460024A1464D
:108A60003E46D04600BF4FE0285D802814DA285DDE
:108A7000002811DD792E06DD802F04DA002608F1AA
:108A8000020000F007082A5D314640460A9BFFF7C6
:108A900093FAF01DC6B235E0285DFF2801D0285DAD
:108AA00088B9792E06DD802F04DA002608F102004D
:108AB00000F007080023202231464046FFF77CFAE9
:108AC000F01DC6B21EE015F804904FF6FF7000EAE4
:108AD0000929601C285C48441FFA80F9722E06DDC3
:108AE000802F04DA002608F1020000F007084A4649
:108AF000314640460A9BFFF7ADFC06F10E00C6B2B8
:108B0000601C84B2601C84B25C45ADDBBDE8F09FA4
:108B10002DE9F04781460E46154698460024002769
:108B200000BF31E0285D80280BDA285D002808DDD1
:108B30002A5DC4EBC4003044C1B24846FFF79BFA3B
:108B400020E0285DFF2801D0285D40B9C4EBC400B7
:108B50003044C1B220224846FFF78DFA12E02F5D63
:108B60004FF6FF7000EA0727601C285C384487B284
:108B7000C4EBC4003044C1B23A464846FFF7D8FCC3
:108B8000601C84B2601C84B24445CBDBBDE8F08736
:108B90002DE9F04780460D4616461F46DDF8209029
:108BA000002400BF0BE0325D04EB440005EB8000C5
:108BB000C1B24B464046FFF7A3FA601C84B2BC42E8
:108BC000F1DBBDE8F0872DE9F04781460D461646FA
:108BD0001F46DDF820A0A84600240BE03A5D53466E
:108BE00041464846FFF7E2FE08F1060000F0FF08A4
:108BF000601CC4B2B442F1DBBDE8F08770B586B04A
:108C00000446142233A101A8F9F7F1FF0026B4F8B5
:108C10000A014FF6FF7101EA0015B4F808011028A7
:108C20001BDC61191023002201A8FDF75FFB112353
:108C3000002201A92C48FDF759FB94F8040138B132
:108C400094F8020100F00F002749173981F82A0033
:108C500001202649887106B070BD05F10F0081B270
:108C60002046FCF76BFC0646012E06D16119112344
:108C7000002201A8FDF73AFB05E06119102300224C
:108C800001A8FDF733FBB4F80A0148B12946204694
:108C9000FCF754FC0646022E02D120208DF8040079
:108CA0001123002201A91048FDF720FB94F80401CC
:108CB00038B194F8020100F00F000B49173981F820
:108CC0002A000120094988712046FFF743FD00BFB3
:108CD000C1E700002020202020202020202020206C
:108CE00020202020200000009A0A0020F4240020E8
:108CF00070B505460C46294604200BF0BFFE0CB1AA
:108D0000FE2100E0002108460BF00EFF2946052059
:108D10000BF0B4FE0CB17F2100E0002108460BF0FF
:108D200003FF70BD2DE9F04705460E469046994673
:108D30000024294600200BF0A1FE00BF0DE0B9F190
:108D4000000F03D100200BF0EFFE04E018F80470D0
:108D500038460BF0E9FE601CC4B2B442EFDBBDE85C
:108D6000F0872DE9F05F0746894690461D46DDF8FD
:108D700028A04FF0000B002413E03919C8B249466F
:108D80000BF07CFE002608E004FB05601AF800B03A
:108D900058460BF0C9FE701CC6B2AE42F4DB601C34
:108DA000C4B24445E9DBBDE8F09F70B505462946ED
:108DB00001200BF063FEF8200BF0B6FEF8200BF05C
:108DC000B3FE02240BE0294620460BF057FEFF209D
:108DD0000BF0AAFEFF200BF0A7FE601CC4B2062C0D
:108DE000F1DB294606200BF049FE1F200BF09CFE0C
:108DF0001F200BF099FE70BD30B504460D4625B11D
:108E000084F0280404F5206401E004F500642046A1
:108E100000F008F804460DB184F40074C4F316049D
:108E2000204630BD30B503460022184640F6E32404
:108E3000002106E0520000F001052A4440084D1CC4
:108E4000E9B20C29F6DBD00200210BE0C1F11605D6
:108E500020FA05F525B1C1F10B0504FA05F56840C6
:108E60004D1CE9B20C29F1DB00EBC22200200021ED
:108E700006E0400002F00105284452084D1CE9B20A
:108E80001729F6DB30BD000010B500243548007806
:108E9000022801D106F09CFB33480078022802D159
:108EA000012006F08BF927E0302130480278007865
:108EB000401C2E4B18702E4881542E48006800EB41
:108EC000800040002B4908602748007802280CD118
:108ED0002948407829490978884206D004231A464F
:108EE00023492748FDF702FA06E004231A462049E1
:108EF00023481238FDF7FAF91C4800780428D3DB20
:108F00001C48006808B9002403E01A480088401E85
:108F100084B200212046FCF731FBD0B1194991F809
:108F2000672015494878002108F074FA012011F0F3
:108F300045FF012011F0D0FE0F494878F9F7D4FF22
:108F40000D4840780D49087006210F480FF048FE83
:108F500003E00A480078F9F7C7FFFCF789F806F044
:108F6000FDFA10BD6E0B00206D0B00208E0C002052
:108F7000940C0020900C0020BB2D00205F0B0020E3
:108F8000F5090020BB290020280A002070B5002424
:108F90001F48857C12E030211E4802780078401C72
:108FA0001C4B18701C4881541C48008800EB800042
:108FB0004FF6FF7101EA4000184908801548007813
:108FC0000228E8DB1548008808B9002403E01348AC
:108FD0000078401EC4B24F2C16DC0D48807CA042A5
:108FE00012D00B48847407F0F5FF0D48007820B1CB
:108FF0000748857407F0EEFF01E011F08FFC084987
:10900000B1F8010007F01CF8FCF7A2F870BD0000F1
:10901000BB2D0020BF0C0020C20C0020C00C002083
:10902000E40F002010B51BE01C480078032804D191
:109030001A480078401C19490870302117480278F6
:109040000078401C154B187015488154154800884D
:1090500000EB80004FF6FF7101EA400011490880E3
:109060000E4800780528DFDB0E480088B0F5207F29
:1090700010DB0C480088B0F5876F0BDC09480088CE
:109080000949A1F8010011F097FC0749B1F8010066
:1090900006F0D6FFFCF75CF810BD0000BF0C002006
:1090A000C20C0020C00C0020E40F002010B52048A6
:1090B0000078022801D106F08BFA1E4800780228B9
:1090C00002D1012006F07AF818E01B480078032846
:1090D00004D119480078401C1749087030211648FF
:1090E00002780078401C144B1870144881541448BE
:1090F000006800EB80004000114908600E480078CD
:109100000928E2DB0E480068FCF7FEFB0D494878B1
:10911000F9F7EAFE0B4840780B490870FCF75AF85B
:109120000849487811F09EFC06F018FA10BD0000BE
:109130006E0B00206D0B00208E0C0020940C002084
:10914000900C0020BB2D00205F0B002070B5044662
:1091500060484078102800D170BD5E4840780228F1
:1091600000D1F9E75B484078042800D1F4E759487A
:1091700040780F2804D158480088022800DCEBE72B
:1091800054488088022800DAE6E752488088B4FB19
:10919000F0F100FB11404F494880002088710846DB
:1091A00080794E49C87401204D490871494840787A
:1091B00013280DD2DFE800F0840A841084290D788A
:1091C00035384A7E696E7174847B810013F0A0FC8F
:1091D00076E013F0FDFF73E013F0FAFC41480088DD
:1091E00090B94048408806280ED13A48408839490D
:1091F000897908443749898890FBF1F201FB120014
:10920000C5B228460BF016FD5AE032480078042813
:1092100003D1012012F00CFE02E0002012F008FE43
:109220004EE013F09FF94BE013F044F929484088D1
:109230002849897908442749898890FBF1F201FB84
:109240001200C5B2284607F059FE39E021480078DF
:10925000032803D1012013F091FA15E01D4800788E
:10926000042811D1002013F089FA1A4840881949BE
:10927000897908441749898890FBF1F201FB1200B3
:10928000C5B2284608F002F81AE01649887813F0AB
:1092900057FE15E013F02EFD12E013F03FFB0FE038
:1092A000002013F0C5F90BE012F044FD08E012F0C5
:1092B000CFFB05E012F04AFF02E012F0EDFF00BF25
:1092C00000BF044841880078401E064A22F810106A
:1092D00000BF41E7E80C0020FE0B00203D0A002003
:1092E0007B0A002018A3002010B50FE0302112489F
:1092F00002780078401C104B1870104881541048B8
:10930000006800EB800040000D4908600A480078C2
:109310000328EBDB0A480068FF2803D3FF20094934
:10932000087403E0064800780649087411F0F6FA5C
:10933000FBF780FF10BD00008E0C0020940C002075
:10934000900C0020BB2D002010B518E014480078C8
:10935000032804D112480078401C114908703021BC
:109360000F4802780078401C0D4B18700D4881544E
:109370000D48006800EB800040000B490860084879
:1093800000780928E2DB084800680849886011F085
:10939000C5FA10F0E5FF06F02DFBFBF76DFF10BDE1
:1093A0008E0C0020940C0020900C0020BB2D00207F
:1093B00010B518E013480078012804D1114800784E
:1093C000401C1049087030210E4802780078401C7B
:1093D0000C4B18700C4881540C48006800EB80005E
:1093E00040000A490860074800780728E2DB074880
:1093F00000680749C86011F091FA10F0B1FFFBF75F
:109400008BFF10BD8E0C0020940C0020900C0020CF
:10941000BB2D002010B5044694B110200D494870B2
:10942000002088808871C871488001220721104679
:1094300011F0B4FC012011F0CFFC0920064908709E
:109440001023002205A10A48FCF750FF12F0E0F9B2
:1094500010BD0000E80C0020B308002041646472D5
:1094600065737320426F6F6B202020200000000086
:109470003E0A002010B5044664B3184880790128DC
:1094800003D117480068174908601648006800F5BE
:109490008001091DC822144818F0C6F906200F499A
:1094A0008880112048700020488088710120C87190
:1094B00000200E4981F8260001220721104611F0F4
:1094C0006DFC012011F088FC002009490871092079
:1094D0000849087012F0BCFA10BD0000E80C00202A
:1094E000B00F0020AC0F0020866F00203D0A002046
:1094F0007B0A0020B308002010B54FF4804041499A
:109500008861414890F86300032801D010F00AFFF9
:109510003D4890F8672002213C48007807F07AFF28
:109520003B480078082801D106F002FA3848007854
:10953000032804D106F0F2FD0120364908703448B2
:109540000078032806D03248007818B130480078F7
:1095500001280DD100202E490870012011F02EFCA9
:10956000012011F0B9FB01220721104611F016FC71
:10957000012029490870294908702949087226499B
:109580004870264988720020264908804FF4807070
:1095900025490860FAF74AFF0120FAF7DDFCFAF7DF
:1095A00055FC00202149086021490880164890F8A0
:1095B0007E0001280BD11F48407814490978884261
:1095C00005D0124800781B49487011F0A7F90F48E0
:1095D0000078194981F8630001201849C8710C48C6
:1095E000007870B91648007858B1124841781430A4
:1095F000405C18B9FF2009F09FFD02E0FF2009F050
:10960000D3FB10BD00000240BB2900205F0B0020EF
:10961000B308002055080020C0080020E0240020E6
:10962000122500201A0C002028140240DC0B002018
:109630008C0B0020BB2D0020C3090020EB24002050
:109640008E0C002010B5474890F8004204EBC4008F
:1096500000EB04104FF6FF7101EA80044FF48040E4
:10966000414988624010886140480078052807D049
:109670003F480078052813D13C48007808280FD1CE
:109680003C4844823C4800783A4908740846037CC8
:1096900000223A49FCF72AFE0120364948742EE0A0
:1096A000304890F80302012804D02E4890F80302B5
:1096B000032824D12B4890F8041200F20A2000EB72
:1096C0000110C07BD8B12B484482264890F8041280
:1096D00000F20A2000EB0110C07B264908740846FE
:1096E000037C204890F8042200F20A2000EB0211CB
:1096F00000222048FCF7FAFD01201E494874194851
:1097000090F80B0108B111F0BDFF14F089F814F0C6
:10971000ADF8FAF7D7FF0120194908701949087008
:1097200012480078022807D011480078022805D195
:109730000E480078082801D1012000E0002008B977
:1097400010F054FF002010490860104908601049CB
:10975000088010480078104981F8630001200F4903
:10976000C87110BDBB29002000000240B3080020D2
:10977000B2080020AA2E0020AD0C0020AE0C002064
:10978000C0080020E0240020D00B0020DC0B0020CB
:109790008C0B00205F0B0020C3090020EB2400206D
:1097A00070B504460E46154674B307201B49487031
:1097B00040F201108880002088710120C87118488B
:1097C000007840B90846808895FBF0F100FB115005
:1097D000124948800DE011480078401E114931F8C7
:1097E00010000E49898890FBF1F201FB12000B4931
:1097F000488001220721104611F0D0FA012011F013
:10980000EBFA092008490870102300223146074866
:10981000FCF76CFD12F08EFA70BD0000E80C002021
:10982000B50F002018A30020B30800203E0A002036
:109830002DE9F04104460F4615461E46E4B10520C9
:10984000134948704FF4806088800846808895FBF3
:10985000F0F100FB11500E49488000208871012072
:10986000C87101220721104611F098FA012011F069
:10987000B3FA092007490870102300223946064828
:10988000FCF734FD304612F0D3FABDE8F081000059
:10989000E80C0020B30800203E0A002000200D49FB
:1098A00008804FF480400C4988610C480068C078FB
:1098B000C0F3C100012805D10948007840F0040038
:1098C000074908700120074908704FF4C87006491D
:1098D00008807047800B0020000002403C0B0020F5
:1098E0006F0B00206D0B0020240C002070B5044687
:1098F0000D46002C72D0082D04D0092D21D00A2D40
:109900005DD13DE04E48407800EB40004D4901EB11
:109910000010807B00094C4908804948407800EBE2
:109920004000484901EB0010B0F80D00C0F30B00F7
:10993000464908801023002245A14A48FCF7D6FC7E
:109940003DE03F48407800EB40003E4901EB00100D
:10995000807B00093C4908803948407800EB400092
:10996000384901EB0010B0F80D00C0F30B00374987
:109970000880102300223CA13A48FCF7B7FC1EE007
:109980002F48407800EB40002E4901EB0010007C8E
:1099900000092D4908802A48407800EB40002949F9
:1099A00001EB0010B0F80F00C0F30B00274908804E
:1099B0001023002231A12B48FCF798FC00BF00BF08
:1099C0002148008830B1012809D002280ED0032890
:1099D00014D10CE000202E4948800FE02CE01B48F9
:1099E000008807F029F82A49488007E000BF174897
:1099F000008807F0CBFA2649488000BF00BF00204E
:109A000023498871042048700120C8711549491EF6
:109A100081F83800102300221EA112482630FCF7DE
:109A200065FC01220721104611F0B8F9012011F060
:109A3000D3F909201C49087012F0ECFA70BD00003F
:109A4000BB2D0020EA2D0020A00F0020A20F002037
:109A50004354432F444353202020202020284129D1
:109A6000000000003E0A00205258204354432F4477
:109A7000435320202028412900000000545820434F
:109A800054432F4443532020202841290000000044
:109A9000E80C00202A205377697463682054797099
:109AA0006520202000000000B308002010B5044607
:109AB000002C39D01E48008838B91EA322A2642188
:109AC000002001F0F9F9002010BD19480088234951
:109AD00088801023002222A12648FCF707FC0B20D7
:109AE0001E49487000208871C8712348007810B959
:109AF000002048800DE019480078401E1F4931F8C9
:109B000010001649898890FBF1F201FB12001349FD
:109B1000488001220721104611F040F9012011F080
:109B20005BF909201649087012F010FB0120CBE701
:109B30000C0C00202020202020202020202020206D
:109B400020202020000000004E6F2043616C6C201C
:109B50005265636F7264732000000000E80C0020FF
:109B600043616C6C204C6F67202020202020202037
:109B7000000000003E0A0020B50F002018A30020BE
:109B8000B308002070B50546002D43D02648408814
:109B90002549897908442449898890FBF1F201FB21
:109BA00012044FF4931000EB4414202221461F4866
:109BB00017F03AFE05201C498880122048701C4886
:109BC000007810B9002048800DE017480078401E4A
:109BD000184931F810001449898890FBF1F201FB13
:109BE00012001149488000200F4988710120C87176
:109BF0000020114981F8260001220721104611F0AA
:109C0000CDF8012011F0E8F800200C490871092076
:109C10000B490870102300220AA10748401CFCF7DA
:109C200065FB12F039FB70BDE80C0020C5A70020D1
:109C3000B50F002018A300203D0A00207B0A002059
:109C4000B308002043616C6C204C6F6720202020FB
:109C500020202020000000002DE9F047054688461E
:109C600016461C46DDE90879002D52D001202E4908
:109C7000487008468480304608F06AFE022C1DDDDC
:109C80002A48007840B92848808897FBF0F100FB0B
:109C90001170254948800DE023480078401E244972
:109CA00031F810002049898890FBF1F201FB120085
:109CB0001D49488000201C4988711CE000201A4979
:109CC00048801A48007840B90846808897FBF0F130
:109CD00000FB1170144988710DE013480078401E94
:109CE000134931F810001049898890FBF1F201FB0B
:109CF00012000D4988710C4880F807900122072155
:109D0000104611F04BF8012011F066F809200949BE
:109D100008701023002241460748FCF7E7FA12F0CA
:109D2000F7FEBDE8F0870000E80C0020B50F00202A
:109D300018A30020B30800203E0A00202DE9F041BE
:109D400004460F4615461E4674B309201B49487049
:109D50001B4800888880002088710846C571194812
:109D6000007840B90846808896FBF0F100FB11604E
:109D7000124948800DE011480078401E124931F820
:109D800010000E49898890FBF1F201FB12000B498B
:109D9000488001220721104611F000F8012011F03F
:109DA0001BF8092009490870102300223946084889
:109DB000FCF79CFA12F07EFBBDE8F081E80C002075
:109DC000FC0B0020B50F002018A30020B3080020D2
:109DD0003E0A00207CB505460C4624A103C9CDE906
:109DE00000014FF46160B4FBF0F086B2042130460C
:109DF0000EF09EFB042300221E496846FCF776FA0B
:109E00004FF46160B4FBF0F100FB11403C21B0FB6A
:109E1000F1F6022130460EF08BFB02230422154995
:109E20006846FCF763FA3C20B4FBF0F100FB1146F6
:109E3000022130460EF07CFB022306220D496846C3
:109E4000FCF754FA082269460B4808F041FF012349
:109E50001A460521094808F0ADFE02200849887518
:109E600001220821284601F037FD7CBD202020205A
:109E700020202020D0240020142000202021002099
:109E8000830A002010B58CB00446302249A16846F0
:109E9000F8F7ADFE002C3DD105F0ACFD514890F82F
:109EA0001001032806DC0020FAF72CFB0120FAF74A
:109EB00047FB05E00120FAF725FB0020FAF740FBFD
:109EC000484890F81001484A02EB00110F23002285
:109ED0004648FCF718FA0923002245A143481030F0
:109EE000FCF704FA0C23002244A140481930FCF787
:109EF000FDF93023002269464448FCF7F7F943484E
:109F0000434908600846006810F0C8FF0020414936
:109F1000087042E04048407800EB40003F4901EBC8
:109F2000001000780121B1EB901F02D000200CB08E
:109F300010BDFAF736F805F05DFD37494878F8F7B7
:109F4000D3FF35484078364908700F23002235A1E9
:109F50002648FCF7D8F92E490968D1F805000821F0
:109F60000EF0E6FA03230022324920481030FCF7B5
:109F7000BDF92E211D48C174052304222D49C91C99
:109F80001030FCF7B3F90C2300221CA1174819303C
:109F9000FCF7ACF904201F490870012010F0C6FE40
:109FA00001220721104610F0F9FE02202249087014
:109FB0000120BCE7401040040010199D0210199DBB
:109FC000020000000000000000000100000000008E
:109FD00000000000FFFFFFFFFFFFFFFFFFFFFFFF8D
:109FE000FFFFFFFFBB290020AD690208D008002059
:109FF0003030302E30303030300000002020202033
:10A000002020202020202020000000004A2E0020B8
:10A010003C0B0020D40C0020BB2D0020EA2D00209A
:10A020005F0B002052656D6F7465204354432F44CD
:10A0300043532000D0240020B308002010B54FF473
:10A040000050A949886240008861A8480068C0782B
:10A05000C0F34110022805D1A548007840F008005F
:10A06000A3490870A34890F86300032801D010F0BA
:10A0700059F96420A0490870202011F07BFA4FF4B0
:10A0800080709E4908609E48007820B106F046F82E
:10A0900001209B4908709B48D0F801109A48FBF7B3
:10A0A000B7F99848D0F8051097484530FBF7B0F954
:10A0B00094480078012807D19249D1F80500F9F7B2
:10A0C00015FA9249086006E08E49D1F80100F9F7C7
:10A0D0000DFA8E490860072300228DA18A480830B6
:10A0E000FCF704F9122300228BA187481030FCF7FB
:10A0F000FDF80120844981F83F008C4908708148AF
:10A10000007848700020C1F80A007E48D0F80500A9
:10A11000C1F806007B48D0F80100C1F80200062310
:10A120000022834981480E30FCF7E0F8714890F82E
:10A130009401754981F85200242300227DA17248C0
:10A140001030FCF7D3F86F48007820B1012814D004
:10A1500002283DD123E00120804908700A23002213
:10A160007FA169483530FCF7C1F8042300227FA1A4
:10A1700065484130FCF7BAF82AE0022077490870B8
:10A180000A2300227BA160483530FCF7AFF8042396
:10A1900000227BA15C484130FCF7A8F818E00020C1
:10A1A0006E4908701223002277A157481030FCF73F
:10A1B0009DF80A23002279A153483530FCF796F820
:10A1C0000423002278A150484130FCF78FF800BFEB
:10A1D00000BF7748007838B90123002275A14A48AA
:10A1E0004030FCF783F806E00123002272A14648C4
:10A1F0004030FCF77BF83F4890F8672002216C481C
:10A20000007807F007F96D48007803281DD06C48E6
:10A210000078032803D169480078082815D06748DA
:10A22000007890B16648007818B96448007808282A
:10A230000BD062480078012807D0614800780128D7
:10A2400011D15E48007808280DD107205B490870BD
:10A25000012010F04FFD012010F03EFD01220721EA
:10A26000104610F09BFD01205649087056490870B1
:10A27000564908725349487053498872002054491E
:10A2800008805449088054490870022053490870D6
:10A290004FF47A7052490880164890F88D0108B141
:10A2A00011F0F0F900204F4908604F490880C8209C
:10A2B0004E4908800F4890F87E0001280BD14C4889
:10A2C00040783B490978884205D0394800784849A8
:10A2D000487010F023FB36480078464981F8630047
:10A2E00001204549C87110BD000002403C0B002010
:10A2F0006F0B0020BB290020700C002018140240B6
:10A3000055080020C27D00206A090020140C00209E
:10A31000202020202020200020202020202020205D
:10A320002020202020202020202000004E7000200F
:10A33000400B002020202020202020202020202032
:10A34000202020202020202020202020202020200D
:10A35000202020202020202000000000130C0020BE
:10A36000496E646976696475616C00005349443ACA
:10A370000000000047726F75702043616C6C000034
:10A380004749443A00000000416C6C2043616C6C0A
:10A39000202020202020202020200000416C6C2044
:10A3A00043616C6C202000004149443A00000000E9
:10A3B0005F0B00204100000042000000B3080020B5
:10A3C000B2080020C0080020E02400201225002050
:10A3D000880B0020860B0020720B00206E0B0020E3
:10A3E000FA0B0020DC0B00208C0B0020100C00204E
:10A3F000BB2D0020C3090020EB24002010B54FF432
:10A400000050634988616348007848B90120624977
:10A41000087062A366A2C821002000F04DFD10BDA7
:10A420004FF480405A4988626648D0F80510664863
:10A43000FAF7EEFF0723002264A163480830FBF718
:10A4400055FF2423002263A15F481030FBF74EFF25
:10A45000102300225B4909315B481030FBF746FFAF
:10A460000020594981F83F00644908705548007838
:10A4700048700020C1F80A005248D0F80500C1F821
:10A4800006005F4800680078C0F3C00030B15C4847
:10A490000068D0F81600C1F8020005E05948D0F86D
:10A4A00080015649C1F8020006230022564953484C
:10A4B0000E30FBF71BFF2423002246A14248103038
:10A4C000FBF714FF3F48007820B1012812D0022882
:10A4D0002FD11FE0102300223A4909313A481030A9
:10A4E000FBF704FF0A23002248A137483530FBF769
:10A4F000FDFE1EE01023002232490931324810309F
:10A50000FBF7F4FE0A23002243A12F483530FBF766
:10A51000EDFE0EE01223002242A12B481030FBF783
:10A52000E5FE0A23002244A127483530FBF7DEFE72
:10A5300000BF00BF012043490870434908704348E9
:10A54000007838B90123002241A11F484030FBF7B1
:10A55000CDFE06E0012300223EA11B484030FBF760
:10A56000C5FE00203C49086001200A49087010F02F
:10A570003DF800203949086039490880334800789F
:10A58000384981F8630001203749C87100BF46E7A8
:10A59000000002406E0B0020750B002020202020C0
:10A5A000202020202020202020202020000000002B
:10A5B0004265696E67204D6F6E69746F72656420C5
:10A5C00000000000A97D00206A0900202020202032
:10A5D000202020002020202020202020202020209B
:10A5E000202020202020202020202020202020206B
:10A5F0002020202020202020000000004E7000207D
:10A600003C0B0020BB290020400B0020496E6469F0
:10A6100076696475616C000047726F7570204361E4
:10A620006C6C0000416C6C2043616C6C202020201D
:10A630002020202020200000416C6C2043616C6CA5
:10A6400020200000C0080020E02400205F0B002034
:10A650004100000042000000D00B0020DC0B002075
:10A660008C0B0020C3090020EB24002010B50E48FD
:10A6700040880D49897908440B49898890FBF1F29B
:10A6800001FB12044FF4572000EB04244FF48072B6
:10A690002146064817F0C8F80023A02203493831A4
:10A6A00003A001F0F1F810BDE80C0020C5A50020C2
:10A6B00044726166747320202020202020202020F6
:10A6C0000000000070B504460E46154664B308202D
:10A6D0001A4948704001888000208871C871184864
:10A6E000007840B90846808895FBF0F100FB1150D6
:10A6F000124948800DE011480078401E114931F898
:10A7000010000E49898890FBF1F201FB12000B4901
:10A71000488001220721104610F040FB012010F074
:10A720005BFB0920084908701023002231460748C6
:10A73000FBF7DCFD11F016FF70BD0000E80C0020F7
:10A74000B50F002018A30020B30800203E0A002007
:10A7500000B591B04022002101A8FBF76DFC4FF439
:10A76000807200212048FBF767FC2048407858B9E8
:10A77000052201A91D481030FDF730F80A2201A971
:10A78000194808F0A5FA1EE01848407801280BD1B6
:10A79000102201A915481030FDF720F8202201A948
:10A7A000114808F095FA0EE01048407802280AD1C6
:10A7B000202201A90D481030FDF710F8402201A910
:10A7C000094808F085FA012303220221084808F00D
:10A7D000F1F90020074988750122102106A001F037
:10A7E0007BF811B000BD00001420002095A50020CA
:10A7F00020210020830A002045646974204B65797C
:10A8000020202020202020200000000070B50025FE
:10A81000FF24FF20484981F83C001023002247A173
:10A8200045483D30FBF762FD1023002243A142481A
:10A830004D30FBF75BFD41A145A008F001FA102265
:10A840004849494808F044FA0123002202214748B8
:10A8500008F0B0F9002038498875012010F0D8FAC6
:10A8600001220721104610F099FA60E008F03AFF43
:10A8700009F026FD0EF01CFA14F0ECFF15F0E8FAD2
:10A8800015F09EF83A48007820B901203849087040
:10A89000FBF7C0F83748008828B94FF4FA703549FB
:10A8A000088015F09BFC3448008828B94FF47A7072
:10A8B0003149088014F096FE30488078112836D04F
:10A8C0002E488078122832D02C488078FF282ED04D
:10A8D0002A488278244925480EF08CFA2348447D82
:10A8E000FF2022494875254988700A2C01D0102C78
:10A8F0001DD101251D48007810B11C4805F062F8F3
:10A900000A2C0ED11023002217491648FBF7EEFC43
:10A9100010F052F8502203214FF439700AF0CCF9AC
:10A9200005E0502204214FF4DC700AF0C5F9002D37
:10A930009CD000F025F870BD830A00202020202044
:10A940002020202020202020202020200000000087
:10A9500053746174696F6E204E616D65203A2020DA
:10A960000000000002100020142000202021002000
:10A97000F10B0020F60B0020F80B0020570B0020F5
:10A9800010B505F037F806F025FB2948007848B1E6
:10A990003023002227492648FBF7B5FC10F00CF8BD
:10A9A0000FF0BCFFFAF7D4FB1023002220491E3120
:10A9B0002148FBF79BFC21480078032807D020485A
:10A9C0000078032805D11D480078082801D101200E
:10A9D00000E0002048BB1B494878F8F785FA194881
:10A9E0004078194908700020184908601849088003
:10A9F0001448C07C60B91748006800780121B1EBA9
:10AA0000901F02D1F9F720FE0FE0FCF709FE0CE0E1
:10AA1000104800680078800938B90A488178002019
:10AA2000FCF7BAFD01200C4908700FF045FC10BD81
:10AA3000E40F0020D284020804090020B30800209B
:10AA4000B2080020BB2D00205F0B0020DC0B002093
:10AA50008C0B00203C0B0020730B002070B50446CB
:10AA60000D4601200E494870084685800020488028
:10AA700088710120C87101220721104610F08EF95B
:10AA8000012010F0A9F909200649087010230022BE
:10AA900021460548FBF72AFC12F03AF870BD000089
:10AAA000E80C0020B30800203E0A002070B5002406
:10AAB00000253248407800EB4000314901EB00109E
:10AAC000D0F805002D49497801EB41012C4A02EBF1
:10AAD0000111D1F80910884213D901242748407880
:10AAE00000EB4000114601EB0010D0F805002349AF
:10AAF000497801EB410102EB0111D1F80910451A27
:10AB000013E000241D48407800EB40001C4901EB95
:10AB10000010D0F809001949497801EB4101184AA1
:10AB200002EB0111D1F80510451A082128460DF055
:10AB3000FFFC08221349144808F0CAF801231A46FA
:10AB40000521124808F036F80120114988750122C4
:10AB5000082110A000F0C0FE1023002212A10C4812
:10AB60003D30FBF7C3FB1023002214A108484D30F1
:10AB7000FBF7BCFB064880F83C4070BDBB2D0020B5
:10AB8000EA2D0020D02400201420002020210020C5
:10AB9000830A00204F666673657420536574202015
:10ABA00020202020000000002B202020202020201A
:10ABB000A6E9537769746368000000002D20202007
:10ABC00020202020A6E95377697463680000000004
:10ABD00010B51448007840B1124804F0F3FE50223A
:10ABE00004214FF4DC700AF067F80F480078012860
:10ABF0000BD100200C4908700FF0F8FC5022042102
:10AC00004FF4DC700AF058F80BE001200749087097
:10AC1000502204214FF4DC700AF04EF801200AF0B3
:10AC2000FFF810BD20210020E80C0020B50F002007
:10AC300010B50446ACB10F200F4948700F4800888A
:10AC400088800020488088710120C8710122072176
:10AC5000104610F0A3F8012010F0BEF809200849B2
:10AC600008701023002207A10B48FBF73FFB0020D0
:10AC700011F0DEFC10BD0000E80C0020FC0B0020F1
:10AC8000B308002045646974204D656D62657220CB
:10AC900020202020000000003E0A00202DE9F04185
:10ACA0000546884616461F46069C75B30A201F496E
:10ACB000487004F1FA008880002088710846C67147
:10ACC0001B48007840B90846808897FBF0F100FBEC
:10ACD0001170164948800DE014480078401E15494F
:10ACE00031F810001149898890FBF1F201FB120044
:10ACF0000E49488001220721104610F04FF801202C
:10AD000010F06AF809200C4908701023002241460F
:10AD10000A48FBF7EBFA204611F030FD1CB9034955
:10AD2000887806F0B3FABDE8F0810000E80C002056
:10AD3000B50F002018A30020B30800203E0A002011
:10AD400070B505460C462046F8F7D0FB06460821AC
:10AD50000DF0EEFB08220949094807F0B9FF01236D
:10AD60001A460221074807F025FF0020064988758A
:10AD700001220821284600F0AFFD70BDD02400203C
:10AD80001420002020210020830A002070B50646F0
:10AD9000002E6ED03C4840883B49897908443A49A6
:10ADA000898890FBF1F201FB12054FF45E2000EB65
:10ADB00005254FF480722946344816F035FD334896
:10ADC000007B01280DD0012030490873020229467A
:10ADD0002E4816F0E1FD022280214FF45E2007F09C
:10ADE0007BFA00240BE029483830005DFF2803D0AF
:10ADF00026483830005D00B903E0601CC4B2A02CC6
:10AE0000F1DB00BF214A5178D2F802001232FAF782
:10AE1000FDFC052000EB24101B4988800E204870A3
:10AE20001B48007810B9002048800DE016480078D3
:10AE3000401E184931F810001349898890FBF1F23F
:10AE400001FB12001049488000200F498871C87129
:10AE5000114981F826000122072110460FF09EFFBC
:10AE600001200FF0B9FF00200C49087109200C499E
:10AE70000870102300220BA10748401CFBF736FA8C
:10AE800011F04CFD70BD0000E80C0020C5A50020AD
:10AE9000B50F002018A300203D0A00207B0A0020E7
:10AEA000B3080020496E626F7820202020202020E7
:10AEB00020202020000000002DE9F04104460D462E
:10AEC00016461F461C480078022803D01A4800780E
:10AED000042801D1BDE8F08118480078082809D07D
:10AEE00016480078164908700122062110460FF016
:10AEF00055FF08E013480078A04204D00122062143
:10AF000010460FF04BFF08200C4908700E480560F2
:10AF10000C480470102300223146401CFBF7E6F970
:10AF200010230022394607481130FBF7DFF90120D2
:10AF30000FF026FF00BFCDE7120C0020B308002061
:10AF4000B2080020E00A0020EC0B002010B5002021
:10AF50000B49487001208880002088710120C87149
:10AF6000084981F839000122072110460FF016FF29
:10AF700001200FF031FF09200349087010BD0000C7
:10AF8000E80C00203D0A0020B308002010B510494D
:10AF9000497801EB41010F4A02EB0111D1F81A0087
:10AFA0000D49FCF746FC08220B490C4807F090FEBF
:10AFB0000123032202210A4807F0FCFD0020094971
:10AFC00088750122082108A000F086FC10BD000051
:10AFD000BB2D0020EA2D0020D024002014200020CA
:10AFE00020210020830A00204D75746520436F6482
:10AFF00065202020202841290000000010B50446CB
:10B000002CB14FF4807200210548FBF715F800239E
:10B01000A0220349383103A000F036FC10BD000027
:10B02000C5A500204E657720534D532020202020B9
:10B03000202020200000000010B51B48C079D0B9A6
:10B0400000201A4908701A48007810B1184804F016
:10B05000B9FC012009F0E4FE30B1502203214FF485
:10B06000397009F029FE1EE0642202214FF4DC70E1
:10B0700009F022FE17E001F0D5FF70B10C4800780E
:10B0800010B10B4804F09EFCFFF7A2FD50220321F3
:10B090004FF4397009F010FE05E0642202214FF4EC
:10B0A000DC7009F009FE10BDE80C0020B50F00208F
:10B0B000202100202DE9F04107460C4615461E468A
:10B0C000294620460DF034FA2A460949094807F076
:10B0D000FFFD01231A460521074807F06BFD0748CD
:10B0E000867501222946384600F0F6FBBDE8F0815E
:10B0F000D02400201420002020210020830A0020DA
:10B100002DE9F04104460F4615461E46D4B10320F2
:10B110001149487008468580808896FBF0F100FB55
:10B1200011600D494880002088710120C8710122FA
:10B13000072110460FF032FE01200FF04DFE0920CE
:10B14000064908701023002239460548FBF7CEF85F
:10B1500011F03EFDBDE8F081E80C0020B3080020AE
:10B160003E0A002070B50646002E5CD03348408869
:10B170003249897908443149898890FBF1F201FB11
:10B1800012054FF4672000EB05254FF48072294625
:10B190002B4816F049FB00240BE029483830005DAD
:10B1A000FF2803D026483830005D00B903E0601C5A
:10B1B000C4B2A02CF1DB00BF214A5178D2F80200C2
:10B1C0001232FAF723FB062000EB24101B4988807B
:10B1D0000D2048701B48007810B9002048800DE011
:10B1E00016480078401E184931F810001349898824
:10B1F00090FBF1F201FB12001049488000200F493A
:10B200008871C871114981F8260001220721104672
:10B210000FF0C4FD01200FF0DFFD00200C49087184
:10B2200009200C490870102300220BA10748401C7C
:10B23000FBF75CF811F05EFD70BD0000E80C00202B
:10B24000C5A50020B50F002018A300203D0A00204E
:10B250007B0A0020B30800204F7574626F782020AD
:10B2600020202020202020200000000010B50E48C3
:10B2700040880D49897908440B49898890FBF1F28F
:10B2800001FB12044FF4562000EB04244FF48072AB
:10B290002146064816F0C8FA0023A0220349383197
:10B2A00003A000F0F1FA10BDE80C0020C5A50020B5
:10B2B00044656661756C7420534D53202020202016
:10B2C0000000000070B505460C46002D7ED0012C14
:10B2D00006D0022C1AD0032C2ED0042C58D141E0D9
:10B2E0004248008838B942A346A264210020FFF7F3
:10B2F000E3FD002070BD3D48008847498880102349
:10B30000002246A14A48FAF7F1FF41E04948008887
:10B3100038B937A348A264210020FFF7CDFD0020F3
:10B32000E8E7444800883C4988801023002247A170
:10B330003F48FAF7DBFF2BE04948008838B92CA3D7
:10B3400048A264210020FFF7B7FD0020D2E744485F
:10B350000088314988801023002247A13448FAF739
:10B36000C5FF15E04948008838B921A348A26421E7
:10B370000020FFF7A1FD0020BCE7444800882649D3
:10B3800088801023002247A12948FAF7AFFF00BFA9
:10B3900000BF0C202049487000208871C8714648C1
:10B3A000007810B9002048800DE01B480078401E4E
:10B3B000424931F810001849898890FBF1F201FBED
:10B3C0001200154948800122072100E008E01046DC
:10B3D0000FF0E4FC01200FF0FFFC09203849087051
:10B3E000204611F0ADFD012084E70000040C002090
:10B3F000202020202020202020202020202020204D
:10B4000000000000496E626F7820456D70747920ED
:10B410002020202000000000E80C0020496E626F10
:10B420007820202020202020202020200000000044
:10B430003E0A0020060C00204F7574626F7820458C
:10B440006D70747920202020000000004F75746218
:10B450006F782020202020202020202020000000A5
:10B46000080C002044726166747320456D70747915
:10B4700020202020000000004472616674732020A8
:10B480002020202020202020000000000A0C002086
:10B49000456D70747920202020202020202020203D
:10B4A0000000000044656661756C7420534D5320A4
:10B4B0002020202000000000B50F002018A300204D
:10B4C000B30800201CB515A103C9CDE9000108226D
:10B4D0006946144807F0FCFB01231A460221124872
:10B4E00007F068FB0020114988750122082110A08F
:10B4F00000F0F2F900200D4981F83C0010230022F1
:10B5000010A10A483D30FAF7F1FE1023002212A1E3
:10B5100006484D30FAF7EAFE1CBD0000FFFFFFFFB2
:10B52000FFFFFFFF1420002020210020830A0020BD
:10B530004469616C204E6F2E202020202020202086
:10B5400000000000496E646976696475616C2020B2
:10B55000202020200000000047726F75702043619A
:10B560006C6C2020202020200000000070B50024FA
:10B57000002504F03FFA6D4841781430405C012802
:10B5800023D100BF6949097909B10D2100E00C21DF
:10B59000084601220021F9F7D3FB2846691C8DB229
:10B5A000B0F5806F0ADA6148407800EB40006049EE
:10B5B00001EB0010C078C0090028E3D1B5F5806F19
:10B5C0007BD1002004F09EFA70BD584841781430B9
:10B5D000405C022821D100BF5449097909B10D21ED
:10B5E00000E00C21084601220021F9F7A9FB2846BA
:10B5F000691C8DB2FA280ADA4C48407800EB40000A
:10B600004B4901EB0010C078C0090028E4D1FA2DA5
:10B6100064D1002004F076FAD6E74448407800EB85
:10B620004000434901EB0010D0F805403F48007945
:10B6300008BB00BF3F48006804443F48844209D823
:10B640003E48D0F85003A04204D33C48D0F84C0305
:10B65000A04202D93948D0F84C433448407800EB36
:10B660004000334A02EB0010007881092046FAF7C7
:10B6700071F918BBDEE700BF2E480068241A304875
:10B68000844209D32D48D0F85003A04204D32B485C
:10B69000D0F84C03A04202D92848D0F850432348A0
:10B6A000407800EB4000224A02EB0010007881094C
:10B6B0002046FAF74FF908B9DEE70FE02046FAF71F
:10B6C00023F91E4991F86720184948781D490978DF
:10B6D00005F0A0FE01201C49087148711349487803
:10B6E000F7F702FC194800680078800920B94FF488
:10B6F00048701749088002E0C820154908800F48A3
:10B7000090F8A30001280CD10C4890F8A50011492D
:10B710000860084600684FF47A7148430D49086094
:10B7200002E000200B49086000BF4DE7BB2D002060
:10B73000EA2D0020A00B002000E1F505BB29002028
:10B7400040771B006D0B0020EB2400203C0B0020F9
:10B75000900B0020940B002010B54148007820F099
:10B76000C00040303E4908703E488068C1F805007E
:10B770003C488068C1F809000846807B20F0F00052
:10B7800088730846B0F80D006FF30B00A1F80D00A8
:10B790000846007920F00E0008710846007920F074
:10B7A000300008710846007820F030000870084624
:10B7B0002D490860084600680FF070FB2A480068B1
:10B7C0000079C0F3011020B1012809D0022815D159
:10B7D0000DE00323002225A12548FAF787FD0DE09F
:10B7E0000323002223A12248FAF780FD06E0032369
:10B7F000002221A11E48FAF779FD00BF00BF0EF01C
:10B80000AFFD1E4800781A491A3908701549C868F2
:10B8100006210CF08DFE072301222E21184807F087
:10B82000C3FE07230322164911481038FAF75EFDBC
:10B830000C49087C03210CF07BFE03231A461049B7
:10B840000B48801FFAF752FD01200FF0D3FA0122B6
:10B85000072110460FF0A2FA0B200A49087010BD0C
:10B860004A2E0020BB2D00203C0B0020464D20001E
:10B870001B0B0020414D200053534200DC0C0020E4
:10B88000D0240020B30800202DE9F04105460E46E3
:10B8900017461C463A4631460C4807F019FA0C4840
:10B8A0004078052802D100200949487008484178AD
:10B8B0000123002207F07EF9002006498875224600
:10B8C0001021284600F008F8BDE8F081142000207F
:10B8D00020210020830A002070B504460D4616463C
:10B8E00002201C494870084685800020887108465F
:10B8F000C671FF20184981F83C001023002217A1CF
:10B9000015483D30FAF7F2FC1023002213A112482B
:10B910004D30FAF7EBFC0122072110460FF03EFAFA
:10B9200001200FF075FA0A20114908701023002237
:10B9300021460948401CFAF7D9FC0A220021064892
:10B940003130FAF779FB0622002103482B30FAF751
:10B9500073FB70BDE80C0020830A0020202020200B
:10B960002020202020202020202020200000000057
:10B97000B308002010B51023002243A14748FAF76E
:10B98000B5FC1023002246A144481030FAF7AEFC63
:10B990001023002247A141482030FAF7A7FC0B23CF
:10B9A000052249493D482030FAF7A0FC1023002227
:10B9B00046A13A483030FAF799FC494800781338E4
:10B9C00007283DD2DFE800F0040C141C242C3400BE
:10B9D0000B23052243A131483030FAF787FC37E0CA
:10B9E0000B23052242A12D483030FAF77FFC2FE0CF
:10B9F0000B23052241A129483030FAF777FC27E0D4
:10BA00000B23052240A125483030FAF76FFC1FE0D8
:10BA10000B2305223FA121483030FAF767FC17E0DD
:10BA20000B2305223EA11D483030FAF75FFC0FE0E2
:10BA30000B2305223DA119483030FAF757FC07E0E7
:10BA40000B2305223CA115483030FAF74FFC00BF0C
:10BA500000BF102300223BA110484030FAF746FCFB
:10BA600002213D4800780CF063FD3C4801780B480A
:10BA700080F8451039484178084880F8471005217A
:10BA800037A0FEF7EBFF10BD564552203A52542D19
:10BA900034442056332E323500000000F00C0020D4
:10BAA000444154453A323032362D30322D30352033
:10BAB00000000000444D52203A2020202020202069
:10BAC0002020202000000000420C002049432020BC
:10BAD0003A202020202020202020202000000000CC
:10BAE0001C0C0020323551383020314D42202000CE
:10BAF000323551313620324D42202000323551331B
:10BB00003220344D42202000323551363420384D19
:10BB1000422020003235513132382031364D42003A
:10BB20003235513235362033324D420032355135BF
:10BB300031322036344D4200556E6B6E6F776E2079
:10BB400020202000424154543A302E3056202020EC
:10BB50002020202000000000B60B0020D024002070
:10BB600056657273696F6E202020202020202020CF
:10BB70000000000010B53C48007820F0C0004030C4
:10BB80003949087039483A49097850F8210036494E
:10BB9000C1F805000846807B20F0F0008873084655
:10BBA000B0F80D006FF30B00A1F80D000846007906
:10BBB00020F00E0008710846007920F0300008716E
:10BBC0000846007920F0C00008710846294908603D
:10BBD000084600680FF062F9022125480078401CF1
:10BBE0000CF0A6FC0223032223492448FAF77EFB2B
:10BBF0001E491F4A127851F8220008210CF098FCC7
:10BC000003231A461C491D48401DFAF76FFB2E21DD
:10BC10001A48401E4172032304221749C91C801D83
:10BC2000FAF764FB16480078042807D01548007816
:10BC3000042805D112480078082801D1012000E02D
:10BC4000002058B901200FF0FFF80122072110460B
:10BC50000FF0A4F804200A49087003E001200A4903
:10BC60004870887010BD00004A2E0020B84D0208B0
:10BC7000D10C00203C0B0020D02400201A09002009
:10BC8000B3080020B2080020260900202DE9F04169
:10BC900004460E4617461D468CB306201D494870C3
:10BCA000FA208880002088710846C5711A480078FB
:10BCB00060B91A4841781830405C1649898890FB71
:10BCC000F1F201FB1200134948800DE011480078A1
:10BCD000401E134931F810000E49898890FBF1F29B
:10BCE00001FB12000B4948800122072110460FF08A
:10BCF00055F801200FF070F809200A490870102348
:10BD0000002231460848FAF7F1FA11F061FABDE86D
:10BD1000F0810000E80C0020B50F0020BB2D0020B2
:10BD200018A30020B30800203E0A0020010A6FF08B
:10BD3000FF0202EA002290B2084370470146002049
:10BD4000CAB210430002090ACAB210430002090A2B
:10BD5000CAB210430002090A084370472DE9FF47A1
:10BD60000446002500260027A846A946FEA30FCBBF
:10BD70008DE80F00292C81F0DC80DFE814F0290029
:10BD800031005600A000D000EF00290144018201DB
:10BD90009901CE01EE02050324036A0379038B03A4
:10BDA000AE03D103F4033B048704B905CD050006B7
:10BDB0000F066F0456066506750625048306B3064E
:10BDC000C906100769074F085F08AA08BA08CA0819
:10BDD000642202214FF4DC7008F06EFFBDE8FF879B
:10BDE000E548407800EB4000E44901EB00100078A2
:10BDF0000121B1EB901F06D0642202214FF4DC70C8
:10BE000008F05AFFEAE7DC494878F7F76DF8DA48B6
:10BE10004078DB4908700020DA490860DA49088078
:10BE20000120DA49087001F084B8D348407800EB6B
:10BE30004000D24901EB00108078800908B9012048
:10BE400000E00020CC49497801EB4101CB4A02EBEC
:10BE50000111897860F38711C748407800EB4000F2
:10BE600002EB00108170CA4991F86720C2494878F6
:10BE7000002105F0CFFA0127BF48407800EB4000D1
:10BE8000BE4901EB001080780121B1EB901F06D173
:10BE9000C0A3C5A264210020FFF70EF805E0BDA3F2
:10BEA000C6A264210020FFF707F80120C849C87026
:10BEB0006422022140F25C6008F0FEFEB3E7C54850
:10BEC0000078032803D0C3480078042800D185E710
:10BED00003F090FDA848807808B9012000E0002018
:10BEE000A549887008468078BB4988720120BB4903
:10BEF0004871012680468146B94908709E4880787D
:10BF000030B910230022B7A16846FAF7EFF905E02F
:10BF100010230022B8A16846FAF7E8F983E79C48A5
:10BF200090F87E0008B9012000E00020984981F8CF
:10BF30007E000125A846A946084690F87E0030B943
:10BF400010230022B1A16846FAF7D0F905E01023CA
:10BF50000022B3A16846FAF7C9F964E79D48007862
:10BF6000032803D09B480078042800D136E701203D
:10BF7000B04908700846007897490872012097492F
:10BF8000C87003F037FD7C494878F6F7ADFF7A4872
:10BF900040787B49087000207A4908607A49088017
:10BFA0000EF024FBFFF7E2FA7AA3A3A2642100209B
:10BFB000FEF782FF764890F85C0010B10EF012F8A0
:10BFC00005E06422022140F25C6008F075FE2AE779
:10BFD0006F4890F8600008B9012000E000206C492B
:10BFE00081F860000125084690F8600010B908F05B
:10BFF0000DFE01E00EF096F96422022140F25C6031
:10C0000008F05AFE0FE7624991F80C11481CC1175D
:10C0100000EB91718910A0EB81015D4A82F80C114F
:10C020000125104690F80C0130B95AA387A264216B
:10C030000020FEF741FF1DE0554890F80C01012853
:10C0400006D154A386A264210020FEF735FF11E03B
:10C050004F4890F80C01022806D14EA385A2642116
:10C060000020FEF729FF05E04AA387A264210020F3
:10C07000FEF722FF6422022140F25C6008F01CFE01
:10C08000D1E654480078032803D0524800780428A9
:10C0900000D1A3E63848C07C38B180480078012838
:10C0A00002DC4C48007800B198E6FEF769FCBAE67D
:10C0B000374890F86700401C032190FBF1F201FB28
:10C0C0001200334981F86700084690F8670042493A
:10C0D000C8710125A846A9462D4890F8670030B9D7
:10C0E000102300226EA16846FAF700F911E02848F3
:10C0F00090F86700012806D1102300226DA1684640
:10C10000FAF7F4F805E0102300226FA16846FAF769
:10C11000EDF801203149887085E62E480078032823
:10C1200003D02C480078042800D157E601206B4941
:10C13000087000206A4908704FF448706949088007
:10C1400000206949087003F055FC114890F8680018
:10C15000012804D00E4890F86800022802D1064950
:10C160004878C3E0E1E000002020202020202020AB
:10C170002020202020202020BB2D0020EA2D002080
:10C180005F0B0020DC0B00208C0B0020690B0020D3
:10C19000BB2900202020202020202020202020201B
:10C1A0002020202000000000506F7765723A204860
:10C1B000696768202020202000000000506F77650C
:10C1C000723A204C6F7720202020202000000000B1
:10C1D000380A00206E0B0020C0080020E024002058
:10C1E000730B00204475616C205374616E64627936
:10C1F0003A4F6666000000004475616C205374611C
:10C200006E6462793A4F6E2000000000545820504E
:10C2100072696F726974793A45646974000000004C
:10C220005458205072696F726974793A4275737903
:10C23000000000006B0B00205363616E6E696E6737
:10C2400020202020202020200000000054582045DD
:10C250006E6420546F6E653A204F666600000000E1
:10C26000545820456E6420546F6E653A203031205A
:10C2700000000000545820456E6420546F6E653AEB
:10C280002030322000000000545820456E642054B5
:10C290006F6E653A204D4443000000006D0B002096
:10C2A00054616C6B61726F756E64203A204F6666E4
:10C2B0000000000054616C6B61726F756E64202029
:10C2C00020202020000000005265766572736520F2
:10C2D0004672657120202020000000006A0B0020BB
:10C2E000D00C0020CE0C00208E0B0020F6F7FCFDB9
:10C2F000FE484078FE4908700020FE490860FE496B
:10C300000880FA48407800EB4000FC4901EB00103F
:10C310000078800918B90120FBF7D8F905E0F8F793
:10C32000D1F901210846F8F707FBF54890F86800B5
:10C3300020B1F34890F86800022806D1F14800883F
:10C34000F8F7CEFC02200FF015F9AFF2B813EEA209
:10C3500064210020FEF7B0FD65E5F0480078032871
:10C3600003D0EE480078042800D137E50020EC49DE
:10C37000087008460078FDF785FD502203214FF430
:10C38000397008F099FC4EE50120E549087008462F
:10C390000078FDF777FD78B90020E1490870AFF229
:10C3A0000C23E0A26421FEF787FD642202214FF4F2
:10C3B000DC7008F081FC05E0502203214FF4397055
:10C3C00008F07AFC2FE5C948407800EB4000CB49E3
:10C3D00001EB001000780121B1EB901F06D0642220
:10C3E00002214FF4DC7008F067FCF7E403F002FB75
:10C3F000C34890F81501D04908700120CF49087052
:10C400004003CF498861B9494878F6F76DFDB748D0
:10C410004078B74908700020B6490860B6490880DE
:10C42000F8F750F901210846F8F786FAB448B0F851
:10C4300000010A2190FBF1F01FFA80FA5046F8F74C
:10C4400072FAAFF2B023BFA264210020FEF734FDE0
:10C45000E9E40020C04908700220C04908700020AB
:10C46000C871BF49088028204880FEF7E5FDDAE45E
:10C47000052011F073F930B16422022140F25C60B2
:10C4800008F01AFC05E0642202214FF4DC7008F089
:10C4900013FCC8E4042011F061F980B1B1480078C0
:10C4A00068B9AFF21033B0A264210020FEF704FD9A
:10C4B0006422022140F25C6008F0FEFB0CE0AFF267
:10C4C0002C33AEA264210020FEF7F6FC6422022188
:10C4D0004FF4DC7008F0F0FBA5E4022011F03EF907
:10C4E00080B1A048007868B9AFF25833A8A264219F
:10C4F0000020FEF7E1FC6422022140F25C6008F0BB
:10C50000DBFB0CE0AFF27433A6A264210020FEF73F
:10C51000D3FC642202214FF4DC7008F0CDFB82E4EE
:10C52000032011F01BF980B18E48007868B9AFF292
:10C530009C33A1A264210020FEF7BEFC64220221EC
:10C5400040F25C6008F0B8FB0CE0AFF2B8339FA299
:10C5500064210020FEF7B0FC642202214FF4DC705D
:10C5600008F0AAFB5FE4012011F0F8F8F0B17D4873
:10C57000007868B9AFF2E43399A264210020FEF795
:10C580009BFC502203214FF4397008F095FB1AE010
:10C59000AFF2004397A264210020FEF78DFC5022E9
:10C5A00004214FF4DC7008F087FB0CE0AFF21C4371
:10C5B00095A264210020FEF77FFC642202214FF443
:10C5C000DC7008F079FB2EE44D4890F86100401CC7
:10C5D000052190FBF1F201FB1200494981F861004D
:10C5E0000DF0A0FE01256422022140F25C6008F0FB
:10C5F00063FB18E4424890F8940108B9012000E078
:10C6000000203F4981F89401002084490870844942
:10C6100008803B4890F8940130B982A386A2642137
:10C620000120FEF749FC05E088A383A264210120D4
:10C63000FEF742FC39480078022808D1304890F8CB
:10C640009401874981F852000120864908716422CB
:10C65000022140F25C6008F02FFB04E22F480078D2
:10C66000032803D02D480078042800D12FE403F0DC
:10C67000C1F9FFF77FFA41F270707B4908805022C0
:10C6800003214FF4397008F017FBECE117484078AC
:10C6900000EB4000194901EB001000780121B1EBDB
:10C6A000901F06D0642202214FF4DC7008F004FBD6
:10C6B0000DE40E48407800EB4000104901EB0010FB
:10C6C0000079C0F30110401C032190FBF1F201FB43
:10C6D00012000649497801EB4101084A02EB0111B9
:10C6E000097960F3051101484078BFE0BB2D0020B7
:10C6F0005F0B0020DC0B00208C0B0020EA2D0020BB
:10C70000BB290020CE0C0020456D657267656E6305
:10C710007920202020202020000000006E0B002027
:10C72000D50C00204E6F20416E616C6F672043482E
:10C7300020202020000000008F0B0020680B00202C
:10C740000000024053656E642053696E676C65207B
:10C75000546F6E6500000000B50F0020E80C00204B
:10C7600018A30020390C002052656D6F74652053AA
:10C7700074756E3A20A1CC202000000052656D6FC8
:10C780007465205374756E3A20A1C120200000000A
:10C7900052656D6F7465204B696C6C3A20A1CC209A
:10C7A0002000000052656D6F7465204B696C6C3A17
:10C7B00020A1C1202000000057616B652055703A10
:10C7C00020A1CC20202020202000000057616B6594
:10C7D0002055703A20A1C1202020202020000000F8
:10C7E000526164696F204F6E6C696E652020202055
:10C7F00000000000526164696F204F66666C696ECC
:10C800006520202000000000436865636B204661BE
:10C81000696C65642020202000000000720B00205D
:10C82000860B002053686F772043616C6C65722023
:10C83000496E666F0000000043616C6C65642053B4
:10C84000686F773A202020200000000053686F773F
:10C850002043616C6C656420496E666F00000000C7
:10C860006A090020BD090020D20C002000EB400026
:10C8700002EB00100171FD4991F86720FC494878EE
:10C88000FC49097804F0C6FD0127B946F84840780C
:10C8900000EB4000F84901EB00100079C0F30110F3
:10C8A000012806D110230022F4A16846F9F71EFDE5
:10C8B00018E0EF48407800EB4000EF4901EB001032
:10C8C0000079C0F30110022806D110230022F0A144
:10C8D0006846F9F70BFD05E010230022F1A1684638
:10C8E000F9F704FD4FF001080120F349487020E3F7
:10C8F000F2480078032803D0F0480078042800D1DB
:10C9000013E403F077F8FEF727FF502203214FF4DA
:10C91000397008F0D1F90CE3E8480078032803D017
:10C92000E6480078042800D11FE5D148407800EBA4
:10C930004000D14901EB001000780121B1EB901FBC
:10C940000DD10020DE4908700220DE490870002069
:10C95000C8710220DC490880002048800CE00020DB
:10C96000D74908700220D74908700020C8710320F9
:10C97000D549088005204880FEF75EFBD9E20020FB
:10C98000CF4908700220CF4908700020C871CE49F5
:10C9900008800A204880FEF74FFBCAE2C7480078AB
:10C9A000032803D0C5480078042800D1DDE403F053
:10C9B00021F8AF48407800EB4000AF4901EB001090
:10C9C0000078800908B9012000E00020A8494978D2
:10C9D00001EB4101A84A02EB0111097860F38711CC
:10C9E000A348407800EB400002EB001001704FF0CC
:10C9F00001090127B8469E48407800EB40001146E7
:10CA000001EB001000780121B1EB901F06D110233B
:10CA10000022AEA16846F9F769FC05E01023002268
:10CA2000AFA16846F9F762FC83E20020A4490870D0
:10CA30000220A44908700020C871A34908801C2066
:10CA40004880FEF7F9FA74E200209D490870022040
:10CA50009C4908700020C87106209B49088000206E
:10CA60004880FEF7E9FA64E2002095490870012049
:10CA7000944908700020C871062093490880FEF789
:10CA8000DBFA56E2794890F80D0108B9012000E080
:10CA90000020764981F80D014FF001090125A846D3
:10CAA0009448007820B100209249087002F05AFCA6
:10CAB0006E4890F80D019049C87301208F49C871E4
:10CAC0006A4890F80D0130B1102300228CA168460D
:10CAD000F9F70CFC05E0102300228EA16846F9F757
:10CAE00005FC26E20020764908700220754908708E
:10CAF0000020C871744908805D48407810B918203A
:10CB0000488002E01B2070494880FEF795FA10E249
:10CB10005748407800EB4000574901EB001000787F
:10CB2000800930B1642202214FF4DC7008F0C4F8AF
:10CB30001BE44F48407800EB40004F4901EB0010E8
:10CB40000078C0434A49497801EB41014A4A02EB67
:10CB50000111097860F300014548407800EB40007E
:10CB600002EB001001700127B846B94640484078F2
:10CB700000EB4000114601EB0010007800F00100CE
:10CB800030B11023002268A16846F9F7AFFB05E039
:10CB90001023002269A16846F9F7A8FBC9E13448CF
:10CBA000407800EB4000344901EB00100078800928
:10CBB00030B1642202214FF4DC7008F07DF814E4F7
:10CBC0003E480078032803D03C480078042800D170
:10CBD0000BE402F00FFF2648407800EB40002649A6
:10CBE00001EB001000788008C0432149497801EB2F
:10CBF0004101214A02EB0111097860F382011C48CE
:10CC0000407800EB400002EB0010017018484078BB
:10CC100000EB4000114601EB00100078C0F38000EB
:10CC200030B9102300224AA16846F9F75FFB05E0FE
:10CC3000102300224BA16846F9F758FB6422022119
:10CC400040F25C6008F038F80127B846B94670E158
:10CC50000748407800EB4000074901EB00100078DE
:10CC6000800910B16422022186E08AE0BB290020FD
:10CC7000BB2D00206D0B0020EA2D00205258204DC6
:10CC80006F6465203A20414D2020202000000000E4
:10CC90005258204D6F6465203A2053534220202083
:10CCA000000000005258204D6F6465203A20464D28
:10CCB0002020202000000000380A00206E0B0020F9
:10CCC000B50F0020E80C002018A30020416E616C15
:10CCD0006F67204D6F646520202020200000000039
:10CCE0004469676974616C204D6F64652020202061
:10CCF00000000000790B0020C0080020E024002084
:10CD0000416E616C6F6720564F58203A204F6E205D
:10CD100000000000416E616C6F6720564F58203A4A
:10CD2000204F66660000000050726F6D6973637576
:10CD30006F75733A204F6E200000000050726F6DC7
:10CD4000697363756F75733A204F66660000000063
:10CD50004475616C20536C6F74203A204F666620D6
:10CD6000000000004475616C20536C6F74203A2001
:10CD70004F6E2020000000004FF4DC7007F09CFF95
:10CD800074E48F480078032803D08D480078042885
:10CD900000D16BE402F02EFE8A48407800EB4000A0
:10CDA000894901EB001000784008C0438549497863
:10CDB00001EB4101844A02EB0111097860F3410162
:10CDC0008048407800EB400002EB001001707D4885
:10CDD000407800EB4000114601EB00100078C0F3F2
:10CDE000400030B91023002278A16846F9F77EFA96
:10CDF00005E0102300227AA16846F9F777FA7D4909
:10CE000091F867206F494878002104F003FB012066
:10CE1000794948700127804681468AE00020774999
:10CE200008700220764908700020C87104207549F6
:10CE3000088014204880FEF7FFF87AE061484078C7
:10CE400000EB4000604901EB00100078800930B130
:10CE5000642202214FF4DC7007F02EFF06E45848EC
:10CE60000078032803D056480078042800D11FE436
:10CE700002F0C0FD5348407800EB4000524901EBFE
:10CE80000010808AA8B100204E49497801EB410189
:10CE90004D4A02EB01118882102300225AA16846F4
:10CEA000F9F724FA01205449087101278046814688
:10CEB0000EE00020514908700220514908700020FE
:10CEC000C87104204F49088017204880FEF7B4F845
:10CED0002FE00020494908700220494908700020CD
:10CEE000C87104204749088016204880FEF7A4F83E
:10CEF0001FE00020414908700220414908700020CD
:10CF0000C87104203F49088015204880FEF794F836
:10CF10000FE00020394908700220394908700020CC
:10CF2000C8710220374908800E204880FEF784F837
:10CF300000BF00BFBFB1234841781430405C20B926
:10CF4000204948780DF08EFD0DE01E4A5278334B93
:10CF500033F812101B4A527802EB42021A4B03EBD1
:10CF600002100DF070FC0DB10DF0CAFC0EB10DF009
:10CF7000D5FCB8F1000F17D010F09AF9002010F08E
:10CF8000B5FC012010F0B2FC0E494878F5F7ACFF73
:10CF90000C484078224908700DF028FB64220221D9
:10CFA00040F25C6007F088FEB9F1000F06D0AFF6E2
:10CFB0001C636A4664210020FDF77EFF00BF9FE4EA
:10CFC0006E0B0020BB2D0020EA2D0020444D522086
:10CFD00054696D6520536C6F743A20310000000075
:10CFE000444D522054696D6520536C6F743A203261
:10CFF00000000000BB290020380A0020B50F0020E7
:10D00000E80C002018A30020444D5220456E6372A6
:10D010007970743A204F666600000000600B0020B3
:10D020005F0B00202DE9F0478CB000260027B046AA
:10D03000B146B246F8484088F74989790844F6492C
:10D04000898890FBF1F201FB120084B2F24800786B
:10D05000032841F0AF84F148008800286FD1EF48E1
:10D06000408829281DD2DFE800F0151D2D43576F99
:10D070008391A5B9C7F5F3F2F1F0EFEEEDECEBEA31
:10D08000E9E8E7E6E5E4E3E2E1E0DFDEDDDCDBDA88
:10D09000D9D8D70010230022E149E248F9F726F950
:10D0A000012748E3DF484C3890F85C00A04203D1E8
:10D0B00001200CB0BDE8F087DA494C3981F85C40BA
:10D0C000012738E3D7484C3890F85D00A04201D1E1
:10D0D0000120EEE7D3494C3981F85D40012708462D
:10D0E00090F85D00D04908730120D049C87122E34F
:10D0F000CC484C3890F85F00A04201D10120D8E71D
:10D10000C8494C3981F85F4091F85F0005F0A0F9FB
:10D11000C749086001270EE3C2484C3890F8600008
:10D12000A04201D10120C4E7BE494C3981F86040DA
:10D13000084690F8600018B10DF0F4F802E0FCE247
:10D1400007F064FD0127F6E2B6484C3890F862001B
:10D15000A04201D10120ACE7B2494C3981F86240CC
:10D1600091F8620005F074F9B24908600127E2E223
:10D17000AC484C3890F86100A04201D1012098E7FA
:10D18000A8494C3981F861400127D4E2A5484C38C0
:10D1900090F86500A04201D101208AE7A1494C39ED
:10D1A00081F8654091F8650005F052F9A2490860E0
:10D1B0000127C0E2A1488078A04201D1012078E790
:10D1C0009E498C700846807897498872012097495B
:10D1D00048719B49087080468246ACE291484C38C1
:10D1E00090F87E00A04201D1012062E78D494C39C0
:10D1F00081F87E4001279EE290484079A04201D10B
:10D20000012056E78D494C71487905F0B7F88D49F2
:10D2100008604FF001088EE28CE28AE26BE25FE286
:10D220003BE22EE221E208E2FBE1EEE1E1E1D4E1C2
:10D23000C6E1AEE1A2E18AE172E166E14EE134E1EC
:10D2400027E1B3E076E067E058E049E03DE02EE01A
:10D2500016E0FFE773484C3890F86700A04201D110
:10D26000012026E76F494C3981F86740084690F85D
:10D2700067006D49C87101206C49887001275AE226
:10D2800068484C3890F86300A04201D1012010E7B3
:10D2900064494C3981F8634000206B4908606B4950
:10D2A00008800120664908708246012743E25D48F4
:10D2B0004C3890F8A300A04201D10120F9E6594969
:10D2C0004C3981F8A340012735E25C480079A0423F
:10D2D00001D10120EDE659490C714FF001082AE215
:10D2E00050484C3890F8A500A04201D10120E0E65A
:10D2F0004C494C3981F8A54001271CE249484C387B
:10D3000090F8A600A04201D10120D2E645494C394F
:10D3100081F8A64001270EE242484C3890F8A4005C
:10D32000A04201D10120C4E63E494C3981F8A44015
:10D33000012700E23B484C3890F8EA0038B9062152
:10D34000374810F0B1FA642100FB01F504E0082130
:10D35000334810F0A9FA054632484C38D0F84C034F
:10D360003B49884214D32F484C38D0F84C033949F4
:10D37000884206D22B484C38D0F84C0336498842B4
:10D3800006D828484C38D0F84C033449884207D393
:10D3900033A338A264210120FDF78EFD002088E62A
:10D3A00020484C38C0F84C530127C4E11D484C3884
:10D3B00090F8EA0038B90621194810F075FA64218E
:10D3C00000FB01F504E00821154810F06DFA054650
:10D3D00014484C38D0F850031D49884214D31148E2
:10D3E0004C38D0F850031B49884206D20D484C38BF
:10D3F000D0F850031849884206D80A484C38D0F86B
:10D400005003164988423FD315A31AA26421012074
:10D41000FDF752FD00204CE6E80C002018A3002088
:10D4200014200020072A0020C0080020E02400204B
:10D43000BC0B0020C80B0020C40B0020BB2D00201B
:10D44000730B0020A00B0020DC0B00208C0B0020B5
:10D4500040771B0000BD0105800BB20300E1F5051C
:10D460006973206F7574206F662072616E67652026
:10D470000000000020526573756C74696E67206649
:10D480007265712000000000F748C0F85053012772
:10D4900051E1F54890F86800A04201D1012008E66A
:10D4A000F14981F86840012745E1EF4890F87F0095
:10D4B000A04201D10120FCE5EC48C078012806D14A
:10D4C000EBA3F0A26421FDF7F7FC0020F1E5E649AB
:10D4D00081F87F4004F078FD01272CE1E348007DCE
:10D4E000A04201D10120E4E5E0490C75002010F0D4
:10D4F000FDF9DE48407828B90020F5F7F5FC00205A
:10D50000E54908704FF0010815E1D848807DA04238
:10D5100001D10120CDE5D5498C754FF001080AE114
:10D52000D248007EA04201D10120C2E5CF490C764D
:10D53000002010F0DBF9CD48407828B90020F5F73D
:10D54000D3FC0020D44908704FF00108F3E0C7482D
:10D55000407DA04201D10120ABE5C44844750120C3
:10D5600010F0C4F9C1484078012804D1F5F7BCFC9B
:10D570000120C94908704FF00108DCE0BB48C07DBC
:10D58000A04201D1012094E5B848C4754FF00108CC
:10D59000D1E0B648407EA04201D1012089E5B348E0
:10D5A0004476012010F0A2F9B0484078012804D157
:10D5B000F5F79AFC0120B84908704FF00108BAE06D
:10D5C000AA49497801EB4101B44A02EB0110214616
:10D5D0000DF039F94FF0010AADE030220021684624
:10D5E000F8F72AFD214668460DF02DF94FF0010AA3
:10D5F000A1E09D4890F8E900A04201D1012058E542
:10D60000994981F8E940012795E0974890F8EA00A8
:10D61000A04201D101204CE5934981F8EA4001275D
:10D6200089E0914890F84A03A04201D1012040E5E9
:10D630008D4981F84A4301277DE08B4890F85403D7
:10D64000A04201D1012034E5874981F85443944830
:10D650000078022807D093480078022803D04FF4BE
:10D66000804091498862012765E07F4890F8A900D1
:10D67000A04201D101201CE57B4981F8A940012786
:10D6800059E0794890F86900A04201D1012010E5E5
:10D69000754981F8694001274DE00421834810F065
:10D6A00003F90546C5EB0510850002217F48001DE2
:10D6B00010F0FAF80544C5EB0510850002217B48FF
:10D6C000801D10F0F1F805446748D0F86A00A842C0
:10D6D00001D10120EDE46448C0F86A5001272AE036
:10D6E0006248C07CA04201D10120E2E45F49CC74D1
:10D6F0004FF001081FE00CB90120DAE4012C02D13F
:10D700000CF05CFE12E0022C02D105F0FDF90DE0F8
:10D71000032C02D105F036F908E0042C02D10CF0FC
:10D720004DFF03E0052C01D105F0FCFA0CF02EFEB4
:10D7300001E000BF00BF01F076BC5D480088012811
:10D7400019D15B48408810B948498C7710E0584897
:10D750004088042806DC56484088401E43491F3153
:10D760000C5405E052484088401C40491F310C547D
:10D770004FF00108DFE74E480088022872D14C487C
:10D78000408817281AD2DFE800F00C1A28364753D1
:10D790006095A2AEBAC6D2DEF3FFF0EFEEEDECEB91
:10D7A000EA00314890F80201A04201D1012080E452
:10D7B0002D4981F802414FF0010A012755E12A481D
:10D7C00090F80B01A04201D1012072E4264981F8B2
:10D7D0000B414FF0010A012747E1234890F80C0163
:10D7E000A04201D1012064E41F4981F80C414FF0AF
:10D7F000010A012739E104212C4810F055F80546AB
:10D800001948B0F80011A94201D1012051E416498C
:10D81000A1F80051012728E1134890F81501A04212
:10D8200001D1012045E4104981F8154101271CE18F
:10D830000D4890F80501A04201D1012039E40A49C0
:10D8400081F805410127BA460FE1074890F8060123
:10D85000A04201D101202CE4034981F806410127AF
:10D86000BA4602E102E10000BB290020BB2D0020E6
:10D8700043616E6E6F742062652073657421202091
:10D880000000000053696E676C6520646973706CFA
:10D8900061792020000000005F0B0020EA2D0020AD
:10D8A0006D0B00206E0B00200000024014200020B1
:10D8B00018A30020F64890F81401A04201D10120DD
:10D8C00007E4F34981F814410127BA46CDE0F04856
:10D8D00090F81001A04201D1012010E4EC4981F838
:10D8E00010410127C1E0EA48B0F81101A04201D17E
:10D8F000012004E4E648A0F811410127B5E0E4481E
:10D9000090F80002A04201D101200CE4E04981F826
:10D9100000420127A9E0DE4890F80102A04201D1AF
:10D92000012018E4DA4981F8014201279DE0D84836
:10D9300090F80202A04201D101200CE4D44981F800
:10D940000242012791E0D24890F80302A04201D19F
:10D95000012014E4CE4981F80342012785E078E0F4
:10D960006BE05EE040E033E026E019E00CE0FFE72A
:10D97000C74890F80402A04201D101200DE4C44937
:10D9800081F80442012770E0C14890F80502A042E6
:10D9900001D1012013E4BE4981F80542012764E06A
:10D9A000BB4890F80602A04201D1012007E4B84923
:10D9B00081F80642012758E0B54890F80702A042D6
:10D9C00001D1012011E4B24981F8074201274CE05E
:10D9D000AF4890F80802A04201D1012005E4AC490B
:10D9E00081F80842012740E0A94890F80D01A042C3
:10D9F00001D1012005E4A64981F80D41A548007830
:10DA000020B10020A349087001F0ACFCA04890F8B8
:10DA10000D01A149C8730120A049C87101278246A0
:10DA200023E09B4890F80F01A04201D1012018E4A7
:10DA3000974981F80F41012717E0954890F80E01AA
:10DA4000A04201D101200CE4914981F80E41012747
:10DA50000BE08F4890F81601A04201D1012016E496
:10DA60008B4981F81641012700BF64E68C48008885
:10DA7000032876D18A484088122830D2DFE800F0A7
:10DA800009303E4C61778797A7B7FEFEFEC7D8ECFA
:10DA9000FEF9082183480FF007FF054682498D42B1
:10DAA00007D982A386A264210020FDF705FA002091
:10DAB00004E42846F9F7DAFE7549D1F88011884266
:10DAC00001D1012006E42846F9F7D0FE7049C1F8DB
:10DAD00080014FF0010A01207E4908700127CDE046
:10DAE0006B4890F88D01A04201D101200DE46849F6
:10DAF00081F88D414FF0010A0127BFE0644890F89A
:10DB00008E01A04201D101200DE4614981F88E41CE
:10DB10004FF0010A0127B1E0052162480FF0C4FE71
:10DB200005465B48B0F88F11A94203D04EF660203D
:10DB3000854201D9012032E45549A1F88F510127CE
:10DB40009CE0052157480FF0AFFE05465048B0F85D
:10DB50009111A94203D04EF66020854202D90120DE
:10DB60001DE48CE04A49A1F89151012786E048481C
:10DB700090F89301A04201D1012010E4444981F8BA
:10DB800093410120534908708246012776E04048BE
:10DB900090F88701A04201D101203CE43C4981F882
:10DBA000874101204B4908708246012766E03848CA
:10DBB00090F88801A04201D101202CE4344981F879
:10DBC00088410120434908708246012756E03048C9
:10DBD00090F88501A04201D101201CE42C4981F874
:10DBE000854101203B4908708246012746E02848CC
:10DBF00090F88601A04201D101200CE4244981F86B
:10DC000086410120334908708246012736E02048CA
:10DC100090F89401A04201D1012040E41C4981F810
:10DC2000944100202C4908702C490880012725E0E8
:10DC3000174890F89501A04201D101202FE4144922
:10DC400081F895410020244908702449088001206A
:10DC500020490870012711E00D4890F89801A04272
:10DC600002D101201BE404E0094981F89841012711
:10DC700004E0012C01D1F8F7C3F900BF5BE50848C7
:10DC8000008804287ED1064840881C2859D227E005
:10DC9000BB290020790B0020C0080020E0240020D0
:10DCA00018A3002014200020DFFCFF0020202020EB
:10DCB00020202020202020202020202000000000E4
:10DCC0004944204F7574204F662052616E6765206D
:10DCD00000000000730B0020720B0020860B002058
:10DCE000DFE800F00E30556486A6C9F1F0EFEEEDE6
:10DCF000ECEBEAE9E8E7E6E5E4E3E2E1E0DFDEDDDC
:10DD0000FE48407800EB4000FD4901EB0010007830
:10DD1000B4EB901F01D1012007E4F848407800EBF4
:10DD20004000F74901EB0010007864F38710F349D5
:10DD3000497801EB4101F24A02EB011108704FF002
:10DD4000010A43E2ED48407800EB4000EC4901EB6A
:10DD500000100078C0F30110A04201D1012012E4AC
:10DD6000E648407800EB4000E54901EB0010007800
:10DD700064F30510E149497801EB4101E04A02EB07
:10DD8000011100E0FEE308704FF0010AD9E7DB491A
:10DD9000497801EB4101DA4A02EB011101F120005F
:10DDA00010230022D749F8F7A1FACAE7D3484078F0
:10DDB00000EB4000D24901EB00108078B4EB901FDB
:10DDC00001D101201BE4CD48407800EB4000CC4954
:10DDD00001EB0010807864F38710C849497801EBA3
:10DDE0004101C74A02EB011188704FF0010AEDE1D1
:10DDF000C248407800EB4000C14901EB0010C078F8
:10DE0000B4EBD01F01D1012005E4BC48407800EB01
:10DE10004000BB4901EB0010C07864F3C710B7495C
:10DE2000497801EB4101B64A02EB0111C870CDE11E
:10DE3000B248407800EB4000B14901EB0010807817
:10DE400000F03F00A04201D1012014E4AB4840782B
:10DE500000EB4000AA4901EB0010807864F3050054
:10DE6000A649497801EB4101A54A02EB01118870EE
:10DE70004FF0010AAAE10821A2480FF015FD05465E
:10DE8000A14890F83C00F8B99C48407800EB40006D
:10DE90009B4901EB0010D0F8050005441EE0F2E3B9
:10DEA000F2E3F2E3F2E3F2E3F2E3CAE39DE36FE3CA
:10DEB0003FE305E3D6E2A7E278E24AE220E2F1E1BD
:10DEC00085E10AE169E030E08C48407800EB4000F1
:10DED0008B4901EB0010D0F80500451B2846F8F7E8
:10DEE00055F848B9AFF68823AFF6782264210120AF
:10DEF000FCF7E2FF00205AE48048407800EB400045
:10DF00007F4901EB0010D0F80900A84201D101209F
:10DF10004DE47A48407800EB4000794901EB00106D
:10DF2000C0F809504FF0010A50E1784890F8EA0033
:10DF300038B9062173480FF0B7FC642100FB01F5E6
:10DF400004E008216F480FF0AFFC05462846F8F7BB
:10DF50001DF848B9AFF6F823AFF6E8226421012096
:10DF6000FCF7AAFF002022E46448407800EB400060
:10DF7000634901EB0010D0F80900A84201D101204B
:10DF800015E45E48407800EB40005D4901EB00106D
:10DF9000C0F809504FF0010A18E15D480078574970
:10DFA000497801EB4101564A02EB0111897B60F38C
:10DFB00007115248407800EB400002EB00108173DB
:10DFC00053480088A8B94D48407800EB40001146FE
:10DFD00001EB0010B0F80D006FF30B0000F6FF70BE
:10DFE0004649497801EB410102EB0111A1F80D000E
:10DFF00030E047480088012816D1464830F8141010
:10E000003E48407800EB40003D4A02EB0010B0F87B
:10E010000D0061F30B003949497801EB410102EB36
:10E020000111A1F80D0015E0E0B202F0F9FC33494E
:10E03000497801EB4101324A02EB0111B1F80D10B0
:10E0400060F30B012D48407800EB400002EB00101C
:10E05000A0F80D102948407800EB4000284901EB5A
:10E060000010807B01092548407800EB4000244ADD
:10E0700002EB0010007C61F307102049497801EBA6
:10E08000410102EB011108741C48407800EB40008C
:10E09000114601EB0010B0F80D001849497801EB6A
:10E0A000410102EB0111B1F80F1060F30B011348AD
:10E0B000407800EB400002EB0010A0F80F100F4872
:10E0C000407800EB4000114601EB00100078012180
:10E0D000B1EB901F00D18A46DEE30D480078074976
:10E0E000497801EB4101064A02EB0111897B60F39B
:10E0F00007110248407800EB40000DE0BB2D0020E6
:10E10000EA2D002014200020830A0020BB290020D3
:10E11000A00F00205C20020802EB00108173FE4873
:10E120000088A8B9FD48407800EB4000114601EB9B
:10E130000010B0F80D006FF30B0000F6FF70F74908
:10E14000497801EB410102EB0111A1F80D0030E02B
:10E15000F1480088012816D1F14830F81410EF4832
:10E16000407800EB4000EF4A02EB0010B0F80D00E1
:10E1700061F30B00E949497801EB410102EB011120
:10E18000A1F80D0015E0E0B202F04AFCE34949783D
:10E1900001EB4101E34A02EB0111B1F80D1060F30C
:10E1A0000B01DE48407800EB400002EB0010A0F8C5
:10E1B0000D10DA48407800EB4000DA4901EB00101E
:10E1C00000780121B1EB901F00D18A4664E3D24868
:10E1D0000078D249497801EB4101D24A02EB0111A2
:10E1E000097C60F30711CD48407800EB400002EB5A
:10E1F00000100174C8480088A8B9C848407800EBEE
:10E200004000114601EB0010B0F80F006FF30B0057
:10E2100000F6FF70C149497801EB410102EB0111A1
:10E22000A1F80F0030E0BC480088012816D1BC4896
:10E2300030F81410B948407800EB4000B94A02EBBE
:10E240000010B0F80F0061F30B00B449497801EBFE
:10E25000410102EB0111A1F80F0015E0E0B202F05C
:10E26000DFFBAE49497801EB4101AE4A02EB0111F7
:10E27000B1F80F1060F30B01A848407800EB4000A4
:10E2800002EB0010A0F80F10A448407800EB40000B
:10E29000A44901EB001000780121B1EB901F00D1DF
:10E2A0008A46F9E29D48407800EB40009D4901EB29
:10E2B00000100079C0F34200A04201D1012015E412
:10E2C0009648407800EB4000964901EB0010007939
:10E2D00064F343009149497801EB4101914A02EB13
:10E2E000011108718D48407800EB4000114601EBA8
:10E2F000001000780121B1EB901F00D18A46CBE2DB
:10E30000894890F8061104F099FA05468348407848
:10E3100000EB4000834901EB0010D0F81A10A9422D
:10E3200001D1012007E47D48407800EB40007D49A1
:10E3300001EB0010C0F81A507848407800EB40001C
:10E3400001EB001000780121B1EB901F00D18A464B
:10E35000A2E27248407800EB4000724901EB0010E5
:10E360000079B4EB901F01D1012006E46B4840789E
:10E3700000EB40006B4901EB0010007964F387105B
:10E380006649497801EB4101664A02EB01110871C7
:10E390006248407800EB4000114601EB0010007825
:10E3A0000121B1EB901F00D18A4675E25B484078AD
:10E3B00000EB40005B4901EB0010C07800F0070063
:10E3C000A04201D1012008E45448407800EB40000D
:10E3D000544901EB0010C07864F302004F494978BA
:10E3E00001EB41014F4A02EB0111C8704B484078E4
:10E3F00000EB4000114601EB001000780121B1EB69
:10E40000901F00D18A4647E24448407800EB400024
:10E41000444901EB0010407800F00F00A04201D108
:10E4200001200BE43D48407800EB40003D4901EB02
:10E430000010407864F303003849497801EB41014A
:10E44000384A02EB011148703448407800EB400034
:10E45000114601EB001000780121B1EB901F00D1B3
:10E460008A4619E22D48407800EB40002D4901EB27
:10E470000010C078C0F3C100A04201D101204BE4DC
:10E480002648407800EB4000264901EB0010C07898
:10E4900064F3C4002149497801EB4101214A02EBB0
:10E4A0000111C8701D48407800EB4000114601EB97
:10E4B000001000780121B1EB901F00D18A46EBE1FA
:10E4C0001648407800EB4000164901EB0010007937
:10E4D000C0F30110A04201D101201DE40F48407893
:10E4E00000EB40000F4901EB0010007964F30510C8
:10E4F0000A49497801EB41010A4A02EB011108710E
:10E500000648407800EB4000114601EB001000780F
:10E510000121B1EB901F09E0A00F0020BB2D0020CE
:10E520005C200208EA2D00201420002000D18A4639
:10E53000B2E1FA48407800EB4000F94901EB0010E5
:10E540000078C0F38000A04201D1012007E4F34825
:10E55000407800EB4000F24901EB0010007864F3D2
:10E560008200EE49497801EB4101ED4A02EB0111CD
:10E570000870EA48407800EB4000114601EB0010BB
:10E58000007800E08CE1800908B94FF0010A83E1CE
:10E59000E248407800EB4000E14901EB00100078D0
:10E5A000C0F34000A04201D101200BE4DB484078D9
:10E5B00000EB4000DA4901EB0010007864F3410001
:10E5C000D649497801EB4101D54A02EB01110870A7
:10E5D000D248407800EB4000114601EB0010007873
:10E5E000800908B94FF0010A56E1CC48407800EBA9
:10E5F0004000CB4901EB00104078B4EB101F01D173
:10E60000012022E4C548407800EB4000C44901EBFA
:10E610000010407864F30710C049497801EB4101CC
:10E62000BF4A02EB01114870BC48407800EB400043
:10E63000114601EB00100078800908B94FF0010A7B
:10E640002AE1B648407800EB4000B54901EB0010E4
:10E65000B0F81100A04201D101204CE4AF4840784D
:10E6600000EB4000AE4901EB0010A0F81140AB48B0
:10E67000407800EB400001EB00100078800908B9F9
:10E680004FF0010A08E1DAE09EE070E042E021E0AC
:10E69000FFE7A248407800EB4000A14901EB0010E1
:10E6A000C07CA04201D1012025E49C49497801EBBE
:10E6B00041019B4A02EB0111CC749848407800EB71
:10E6C0004000114601EB00100078800908B94FF0B6
:10E6D000010AE1E09148407800EB4000904901EBED
:10E6E0000010808AA04201D1012004E48B484078C8
:10E6F00000EB40008A4901EB001084828748407893
:10E7000000EB400001EB00100078800908B94FF0E1
:10E71000010AC1E08148407800EB4000804901EBEC
:10E720000010C078C0F34110A04201D101201AE4CA
:10E730007A48407800EB4000794901EB0010C0783E
:10E7400064F346107549497801EB4101744A02EBC4
:10E750000111C8707148407800EB4000114601EB90
:10E7600000100078800908B94FF0010A94E06B4866
:10E77000407800EB40006A4901EB0010007800F09F
:10E780000100A04201D1012099E56448407800EBE6
:10E790004000634901EB0010007864F300005F491A
:10E7A000497801EB41015E4A02EB011108705B48B8
:10E7B000407800EB4000114601EB00100078800922
:10E7C00008B94FF0010A67E0082156480FF06CF8CD
:10E7D000054655498D4209D9AFF63033AFF62032A0
:10E7E00064210020FCF768FB002068E52846F9F763
:10E7F0003DF84A49497801EB4101494A02EB0111D0
:10E80000D1F81610884201D1012058E52846F9F7C1
:10E810002DF84249497801EB4101414A02EB0111CF
:10E82000C1F816003D48407800EB4000114601EB6E
:10E8300000100078800908B94FF0010A2CE0374831
:10E84000407800EB4000364901EB00100078C0F33F
:10E85000C000A04201D1012031E53048407800EBF2
:10E8600040002F4901EB0010007864F3C3002B49EE
:10E87000497801EB41012A4A02EB0111087027484F
:10E88000407800EB4000114601EB00100078800951
:10E8900008B94FF0010A00BF00BF4FF00109C2E301
:10E8A000224800880628FAD120484088052829D126
:10E8B000012CF4D1AFF60C431DA264210020FCF71B
:10E8C000FBFA04F00FFF05F051F901F039FE0026C4
:10E8D00005E006F1D70013F025F8701CC6B2182E1B
:10E8E000F7DB01F053FE0020164908801649088026
:10E8F00016490880164908801649487201201649B1
:10E90000087190E309484088062833D1134890F8ED
:10E910009601A04224D10120D1E40000BB2D0020AB
:10E92000EA2D002014200020DFFCFF0018A30020A7
:10E93000436C65617220416C6C20534D5320202044
:10E9400000000000080C0020040C0020060C002031
:10E95000020C0020C0080020E0240020BB29002079
:10E96000FC4981F896414FF0010A0120FA490870EC
:10E97000012758E3F948408807280BD1F54890F85B
:10E980009701A04201D1012099E4F24981F8974111
:10E99000012748E3F14840880828B2D1ED4890F8B3
:10E9A0004B03A04201D1012089E4EA4981F84B439D
:10E9B000012738E3EA480078042815D1E7480088A1
:10E9C00005289ED1E548808828B910230022E54912
:10E9D000E548F7F78BFCE1498878E349091F0CF01B
:10E9E0005BF84FF0010A1EE3DD48007805287CD172
:10E9F000DA480088032879D1D84840880A287FD18E
:10EA0000D64880880128B4D1D448C08830B10128C4
:10EA10000BD002280DD0032871D124E0102300224E
:10EA2000D049D248F7F762FC69E0D049491F0C7021
:10EA300065E00821CB480EF037FF0546CC498D42F2
:10EA400009D9AFF69853AFF6885264210020FCF73D
:10EA500033FA002033E42846F8F708FFC349491F7A
:10EA6000C1F801004BE0012C48D1C248008842F2B5
:10EA70001071884208DBAFF6CC53BFA2642100209E
:10EA8000FCF71AFA00201AE4B848401F0078012861
:10EA900008DDAFF6E853BDA264210020FCF70CFAB4
:10EAA00000200CE4B149491FD1F80100F4F71EFD24
:10EAB000AF49884209D9AFF60C63AFF6FC52642126
:10EAC0000020FCF7F9F900202CE4AFF62063B4A293
:10EAD00064210020FCF7F0F904F004FE05F046F88C
:10EAE000A249491FA348008802E0FEE0ECE007E0ED
:10EAF0000BF024FF02F014FA4FF0010A00BF92E27B
:10EB0000964840880B283ED19448C08820B10228FE
:10EB100009D0032836D11AE0102300229149A548D4
:10EB2000F7F7E4FB2EE0012C10D1AFF680639CA236
:10EB300064210020FCF7C0F904F0D4FD05F016F8BC
:10EB40009C499D4800880BF04FFFA2461AE0012C1B
:10EB500017D104F0C7FD05F009F8002608E04FF6CC
:10EB6000FF719448103000EB46000180701CC6B263
:10EB7000202EF4DB8F49904800880BF035FF4FF0D2
:10EB8000010A00BF4FE2754840880C28B7D173488E
:10EB9000C08830B101280BD002280DD0032806D13F
:10EBA0007CE00E2300226F498448F7F79FFB8AE040
:10EBB0008249891E4C7086E000266CE06948805DC1
:10EBC000FF2822D106F0010078B9304606EBD0715B
:10EBD0004A107A490E31895C41F0F00206EBD0719F
:10EBE0004B1076490E31CA5453E0304606EBD071D3
:10EBF0004A1072490E31895C41F00F0206EBD07168
:10EC00004B106E490E31CA5443E05649885DF4F703
:10EC100031F9054606F00100F0B9304606EBD07137
:10EC20004A1066490E31895C01F00F0206EBD07183
:10EC30004B1062490E31CA5406EBD0714A105F493D
:10EC40000E31895C41EA0511CAB206EBD0714B1056
:10EC50005A490E31CA541CE0304606EBD0714A10B6
:10EC600056490E31895C01F0F00206EBD0714B1071
:10EC700052490E31CA5406EBD0714A104F490E3139
:10EC8000895C2943CAB206EBD0714B104B490E3157
:10EC9000CA54701CC6B2402E90DB14E0012C11D176
:10ECA000AFF6F8733EA264210020FCF705F904F0EA
:10ECB00019FD04F05BFF294988884049891E0BF043
:10ECC00051FEA24600BFAEE124480088062879D153
:10ECD00022484088002875D12048C088012871D179
:10ECE000012C6FD108F0C8FD30E41D4800780628DB
:10ECF00069D11A48008803287ED1184840880A281C
:10ED000060D11648808800285CD114480089052805
:10ED10000AD2DFE800F0030A0E6078001023002218
:10ED200010491248F7F7E2FA85E01049491F0C70C4
:10ED300081E008210B480EF0B7FD05460C498D42D5
:10ED400042D91F4B03F1140264210020FCF7B4F8F0
:10ED500000202AE4BB290020730B002018A3002008
:10ED6000E80C00201420002091A300202DA30020F7
:10ED7000DFFCFF00FC0B0020436F6E746163747353
:10ED80002046756C6C2120200000000054797065CD
:10ED9000204572726F722120202020200000000088
:10EDA000536176696E6720446174612E2E2E2E2E7B
:10EDB000000000003DA30020000C002097A50020CB
:10EDC000ACDC000880E010E12846F8F74FFDB249BE
:10EDD000C1F801002FE0012C14D1B04BAFF240027A
:10EDE00064210020FCF768F804F07CFC04F0BEFE0F
:10EDF000AB49C888A84900E01EE00BF09FFD02F077
:10EE00008FF8A24617E0012C14D1A44BA5A26421CF
:10EE10000020FCF751F804F065FC04F0A7FEA049BF
:10EE2000C888F7F7D9F902F07BF80320A2490870E7
:10EE30004FF0010A00BFF6E099480088062843D148
:10EE400097484088C0B99648C088E8BB9448008974
:10EE500010B1012838D105E091484189002008F01F
:10EE60004FFE21E4954890F83C0095490870002138
:10EE7000012008F045FE17E48948408801282AD17E
:10EE80008748008910B1022824D106E08D4AD2F8C3
:10EE90000210507808F03AFD06E4012C19D17F4B9E
:10EEA00080A264210020FCF707F804F01BFC04F0AA
:10EEB0005DFE7B4881884FF45E200BF037FC824872
:10EEC0000088401E804900E08EE0088003207A49D7
:10EED000087000BFA7E07248408802282BD1704814
:10EEE000008910B1022825D109E0012C06D1754A0C
:10EEF000D2F80210507808F009FD18E41AE0012C4D
:10EF000017D1664B67A264210020FBF7D5FF04F000
:10EF1000E9FB04F02BFE624881884FF467200BF078
:10EF200005FC6A480088401E684908800320624941
:10EF3000087000BF77E05A484088032828D1584815
:10EF40000089012802D0022821D105E0012C02D13C
:10EF500008F092FC18E41AE0012C17D14F4B51A293
:10EF600064210020FBF7A8FF04F0BCFB04F0FEFDC9
:10EF70004B4881884FF457200BF0D8FB5448008849
:10EF8000401E5349088003204B49087000BF4AE0E7
:10EF900043484088042846D141480089012802D0CE
:10EFA000022821D105E0012C02D108F065FC1CE407
:10EFB0001AE0012C17D1394B3AA264210020FBF74B
:10EFC0007BFF04F08FFB04F0D1FD354881884FF4BE
:10EFD00057200BF0ABFB3E480088401E3C490880A0
:10EFE00003203549087000BF1DE03348007807282A
:10EFF00019D12B480088062815D12948408910B11D
:10F00000012810D105E026488189002008F078FD0C
:10F0100022E42A4890F83C00294908700021012088
:10F0200008F06EFD18E40FB10BF06AFCB8F1000FA8
:10F0300001D00BF073FCB9F1000F17D025484178CF
:10F040001430405C20B9234948780BF00BFD0DE0EB
:10F05000204A5278204B33F812101E4A527802EBA5
:10F0600042021E4B03EB02100BF0EDFBBAF1000F56
:10F070000FD00EF01DF900200EF038FC01200EF02C
:10F0800035FC14494878F3F72FFF124840781449AB
:10F090000870012040E4000028A30020ACDC000838
:10F0A00018A30020436C656172696E672044617427
:10F0B000612E2E2E00000000E80C0020830A0020A4
:10F0C000B40F0020C5A50020040C0020060C002071
:10F0D000080C0020BB2D0020600B0020EA2D002032
:10F0E0005F0B0020827922B142781AB14278012A5E
:10F0F00000D07047FF220275002282710281828057
:10F10000428181F80421FF22034B83F82A20012247
:10F11000024B9A7100BFECE7830A0020F424002020
:10F1200010B500201F4908701F48007858B1002012
:10F130001D49087002200BF007F90EF071FB00204A
:10F14000F8F7C4FA29E0194890F8680020B1174888
:10F1500090F86800022804D102200BF0F5F80EF0B8
:10F160005FFB124890F86800012804D00F4890F81F
:10F170006800022811D10E48407800EB40000D498C
:10F1800001EB00100078800918B90020F8F79EFA0A
:10F1900003E0F6F773FF00F0E5F84FF4005006497E
:10F1A000886210BD6A0B00203B0C0020BB290020A8
:10F1B000BB2D0020EA2D00200000024010B50446BF
:10F1C0004FF48040544988620020F4F7A7F90A20E0
:10F1D000F8F7B9FB04200BF0B7F80020F4F7BCFEF9
:10F1E000F4F726FEF4F700FD4C48007820F00C0000
:10F1F0004A490870F4F740FF0EF05AF800204849D9
:10F2000008804849088048490860484908804FF408
:10F210008070474908604748007878B146490968D6
:10F22000D1F80900F6F7B2FE28B90020414908706C
:10F230004249088002E0FAF705FA10BD1CB94FF404
:10F24000C870F8F780FB3E4991F867203D4948783F
:10F25000002102F0DFF83C480078012802D10BF0D1
:10F260002BF826E001200BF0A9FD3848007830B1DA
:10F2700037480078E8B935480078082819D135486A
:10F28000007858B12F4841781430405C18B9FF20FD
:10F2900003F052FF02E0FF2003F086FD01200BF097
:10F2A0001BFD2A48007820B90122072110460BF0E7
:10F2B00075FD26480078042807D0254800780428E2
:10F2C00007D122480078082803D141F27070224902
:10F2D000088022480078E8B1194890F8A300022875
:10F2E00003D1012000F00EFC14E0154890F8A300B3
:10F2F00080B9134890F8A60019490880084600888C
:10F3000000EB4001C1EBC0104FF6FF7101EAC000F5
:10F310001349088000BF90E7000002406F0B0020F7
:10F32000800B0020840B0020DC0B00208C0B0020C5
:10F33000181402402E0800203C0B0020300800204A
:10F34000BB290020BB2D002055080020B308002059
:10F35000B20800208E0C0020D20C00206B0B002085
:10F36000900B002010B5424890F80C0130B10128F4
:10F3700005D0022804D003281AD107E018E000BF06
:10F380003B4991F80C010BF06BFC11E00120F4F704
:10F39000E3FD1023002236494C313648F6F7A6FF2C
:10F3A000F4F792FD0020F4F7D7FDF4F741FD00BF1C
:10F3B00000BFF4F719FCF6F761FE4FF400502E4938
:10F3C00088622E480068D0F805002C490968D1F8F9
:10F3D0000910884211D02648B0F8110168B1012007
:10F3E000274908702248B0F8110100EB80004FF661
:10F3F000FF7101EA400023490880F4F73DFE2248EE
:10F400000078022807D021480078022805D11E483C
:10F410000078082801D1012000E00020B8B91C487C
:10F4200040781C49097888420FD0012207211046F4
:10F430000BF0B4FC1248007838B915494878F3F756
:10F4400053FD13484078134908700BF0CFF80020A3
:10F450001149087001201149087000201049086006
:10F4600010490860104908801049086010BD00006C
:10F47000BB290020D40F0020000002403C0B0020DC
:10F48000770B00209A0B0020B3080020B208002060
:10F49000BB2D00205F0B0020C0080020E0240020CE
:10F4A000D00B0020DC0B00208C0B0020E00B002098
:10F4B00010B5184890F80302022804D0154890F8B7
:10F4C0000302032825D1134890F8041200F20A2001
:10F4D00000EB0110C07BE0B100200F4948820D48CD
:10F4E00090F8041200F20A2000EB0110C07B0A49D8
:10F4F00008740846037C074890F8042200F20A20AA
:10F5000000EB021100220448F6F7F0FE0220024947
:10F51000487410BDBB290020AA2E002010B50B484E
:10F52000007820F00800094908700020F3F7F6FF82
:10F5300004200AF009FF0020054908800120054940
:10F54000087000020449086010BD00006F0B002025
:10F55000840B00206D0B0020181402400020074986
:10F560000870074908800749087004480078064970
:10F57000087701200549887070470000760B00204D
:10F58000980B0020130C0020C3090020EB2400205E
:10F5900010B504200A490870F4F703FD0948007803
:10F5A000022802D10120FFF709FE07494878F3F746
:10F5B0009BFC05484078054908700BF017F810BD12
:10F5C000D40C00206D0B0020BB2D00205F0B002011
:10F5D00010B54FF480407649886200207549087064
:10F5E00075480068C078C0F34110012805D1734800
:10F5F000007820F00400714908706F480068C078F6
:10F60000C0F34110022805D16C48007820F00800B2
:10F610006A49087000206A49087001206949087029
:10F620000DF046FE20200AF08FFE4FF480706649F0
:10F6300008600020654908704FF47A7064490880BA
:10F6400000206449086064490880C8206349088034
:10F65000634991F8672063494878002101F0DAFE98
:10F6600061480078012802D10AF026FE42E05F4896
:10F670000078072807D05E48007807283AD15B4811
:10F680000078082836D100205849087001200BF076
:10F6900095FB01200BF020FB514890F8980110B128
:10F6A00054480078A0B15348007858B14D4841788B
:10F6B0001430405C18B9FF2003F03EFD02E0FF204B
:10F6C00003F072FB0122072110460BF067FB11E0EB
:10F6D0004648007846490870082044490870404868
:10F6E00090F898014449086008460068642148433E
:10F6F000414908604148007818B3394890F8A300A0
:10F70000022803D1012000F0FDF914E0344890F8FC
:10F71000A30080B9324890F8A6003949088008460D
:10F72000008800EB4001C1EBC0104FF6FF7101EA09
:10F73000C000334908802A4991F88E010BF058FF28
:10F7400010BD3048007802280CD12548B0F88F0150
:10F7500008B32348B0F88F012B49088001202B49BA
:10F76000087018E02748007801280CD11C48B0F830
:10F77000910180B11A48B0F8910123490880012015
:10F780002249087007E0002020490870144991F8C8
:10F790008E010BF02DFF1D4800781D4908770120D0
:10F7A0001C4988701C480BF063F800BFC8E70000D4
:10F7B00000000240500C00203C0B00206F0B00208A
:10F7C000C0080020E0240020281402406E0B002016
:10F7D000FA0B0020DC0B00208C0B0020100C00200A
:10F7E000BB290020BB2D002055080020B3080020B5
:10F7F000B20800208E0C0020EC0B00206B0B0020C8
:10F80000900B0020130C0020980B0020760B00209A
:10F81000C3090020EB2400204E70002010B54FF4E7
:10F820000050274988622748007850B100202549B8
:10F8300008702549086025490880C82024490880A7
:10F8400010BD0020234908700120234908700020C2
:10F85000224908700AF0CAFE214991F88E010BF086
:10F86000C7FE00201849086018490880C8201849B8
:10F8700008801C48007802280CD11948B0F88F0184
:10F88000C0B11748B0F88F01174908800120174907
:10F8900008700FE01348007801280BD11048B0F829
:10F8A000910138B10E48B0F891010F49088001204C
:10F8B0000E4908700E480AF0DBFF00BFC0E70000E9
:10F8C00000000240750B0020DC0B00208C0B002098
:10F8D000100C0020C0080020E02400206E0B002047
:10F8E000BB290020130C0020980B0020760B002071
:10F8F0004E70002010B5044600F010FC0948C07C92
:10F9000058B90948006800780121B1EB901F02D175
:10F91000F5F7AAF801E0F7F7B7FE0AF067FE03482B
:10F92000047010BDBB2D00203C0B002055080020AA
:10F9300010B521480078214908700020204908604E
:10F940000122062110460BF029FA1C4800780C28E9
:10F950002FD2DFE800F0062E0A0E12161A1E2E22F3
:10F96000262A01200BF02AFA23E001200BF0DEF911
:10F970001FE001200BF0F6F91BE001200BF064FA08
:10F9800017E001200BF0C4F913E001200BF0DCF9C3
:10F990000FE001200BF0AEF90BE001200BF01CFA98
:10F9A00007E001200BF034FA03E001200BF022FA0B
:10F9B00000BF00BF10BD0000B2080020B308002047
:10F9C000EC0B002010B5044600202070A080A07130
:10F9D0002081A081E081208260820622002104F142
:10F9E0001600F6F729FB0122072106200BF0D6F9B5
:10F9F00010BD000010B500202049087020480068A4
:10FA0000C078C0F34110012805D11E48007820F0CD
:10FA100004001C4908704FF480401B4988621B4851
:10FA20000078032801D1FFF79DFC184800780228D0
:10FA300002D10120FFF7C2FB15480078022817D138
:10FA4000FFF7C6FDC8201349088001E0F3F700FB6B
:10FA5000114800786F2803D00E4800880028F5D19F
:10FA600000200B490870FF200B4908700B490870F3
:10FA7000FFF774FD0DF01CFC10BD00004F0C0020C2
:10FA80003C0B00206F0B0020000002406D0B00209B
:10FA90006E0B0020520C00203D0C00203C0C00207E
:10FAA00010B50020114908801149087011484078AC
:10FAB00011490978884207D00E494878F3F714FABB
:10FAC0000C4840780C4908700C48007830B10C485C
:10FAD000007850B909480078082806D1012207218A
:10FAE00010460BF05BF90AF081FD10BD9A0B002067
:10FAF000770B0020BB2D00205F0B0020B3080020F7
:10FB0000B208002010B5044600202A4908700846B3
:10FB100000782949087201202849C870FFF76AFF58
:10FB20004FF4804026498862264890F8A40060B9C6
:10FB30005CB92F222449254811F076FE0AF0E6FA36
:10FB4000224948780DF0D2FE20E020484178143058
:10FB5000405C012802D10AF0E1FE17E01B48417821
:10FB60001430405C02280DD1184A527802EB821200
:10FB7000174B03EBC201154A53781832D05C0AF0D8
:10FB80008BFF03E0114948780AF06CFF0F49487871
:10FB9000F3F7AAF90AF02AFD00200E4908600E4981
:10FBA00008600E490860502204214FF4DC7005F013
:10FBB00083F810BD6B0B0020C0080020E02400205B
:10FBC00000000240BB29002060C00100BB2D0020C6
:10FBD000AB250020DC0B0020E00B0020CC0B00202C
:10FBE00010B5002009490870F6F748FA4FF40050A4
:10FBF00007498862F4F740FA0AF0F8FC002005494A
:10FC00000860054908800549086010BD680B0020A0
:10FC100000000240DC0B00208C0B0020E00B0020D9
:10FC200010B505494878F3F75FF903484078034970
:10FC300008700AF0DBFC10BDBB2D00205F0B00201C
:10FC40001FB5002402A811F01FFB00208DF80C0046
:10FC500001208DF80D008DF80E008DF80F000003C7
:10FC6000029002A9414811F019FB01208DF80D0006
:10FC700002208DF80E000003029002A93B4811F00B
:10FC80000DFB05220D21394811F04EFB01208DF8A6
:10FC90000D008003029002A9344811F0FFFA0522FA
:10FCA0000E21324811F040FB01208DF80D00C003F9
:10FCB000029002A92D4811F0F1FA05220F212B48DC
:10FCC00011F032FB4FF48050284918310860684623
:10FCD00011F09EFC00208DF8000001208DF801003D
:10FCE00000208DF802008DF803008DF8040001203B
:10FCF0008DF805008DF806008DF8070069461C4850
:10FD000011F0AEFC01211A4811F08DFC11F0BCFD80
:10FD10001849088008460078182803D0084600785B
:10FD2000192821D111F0E8FD044604F00100D8B9EA
:10FD300011F08EFE44F00204204611F0BBFEC820F4
:10FD4000F7F701FE11F084FE4FF480500749283187
:10FD50000860B72011F0F0FB4FF4805003491831D0
:10FD60000860C820F7F7EFFD1FBD00000004024047
:10FD7000003800401C0C002070B504461A48867CF0
:10FD8000002500BF1EE00C2C0AD11748807C401CC7
:10FD9000502190FBF1F201FB12001349887409E035
:10FDA0001148807C4F30502190FBF1F201FB120092
:10FDB0000D49887401F00EF90C48007800B903E091
:10FDC000681CC5B2502DDEDB00BF0748807CB04206
:10FDD00001D00AF0A3FD0549B1F8010000F030F9A7
:10FDE000F5F7B6F970BD0000BB2D0020E40F002030
:10FDF00070B505461048B0F801400C2D07D1601CC5
:10FE000084B2B4F5876F09DD4FF4207406E0601EFC
:10FE100084B2B4F5207F01DA4FF487640648A0F875
:10FE200001400AF0C9FD0449B1F8010000F008F9E9
:10FE3000F5F78EF970BD0000E40F002070B50446A0
:10FE40000D46002674480078032803D072480078D5
:10FE5000042802D100F080F970BD012D7ED1092C5B
:10FE600014DC6E480078012803D1204603F00CF919
:10FE700005E06A48007810B9204603F0C7F864220C
:10FE8000022140F25C6004F017FFE5E7A4F10A00EC
:10FE900007281AD2DFE800F004922A2B44631A00E4
:10FEA000502203214FF4397004F006FF5B480078BC
:10FEB000012802D1F9F7B6F807E05848007810B9E0
:10FEC000F9F764F801E0FAF7A1FC77E0544800780C
:10FED00010B1F5F73DF902E00020FFF70BFD5022CD
:10FEE00004214FF4DC7004F0E7FE67E000BF4C48EB
:10FEF000007800B1B0E749480078012803D12046D6
:10FF0000FFF776FF05E04548007810B92046FFF777
:10FF100033FF6422022140F25C6004F0CDFE4DE02C
:10FF20003F48007810B1F5F713F995E73B480078A2
:10FF3000401C032190FBF1F201FB120037490870CD
:10FF400008460078374948700120374948706422D4
:10FF5000022140F25C6004F0AFFE2FE02FE0304859
:10FF6000007810B1F5F7F4F876E700261BE02F488B
:10FF7000807C401C502190FBF1F201FB12002B49C8
:10FF8000887401F027F82A48007850B13023002205
:10FF900028492748F6F7B7F90AF00EFD0AF0BEFC2B
:10FFA00003E0701CC6B2502EE1DB00BF2049B1F85F
:10FFB000010000F045F8F5F7CBF800BF2AE00C2C63
:10FFC00002D00D2C25D100E000BF00201A49087096
:10FFD00000F094F810200AF0B7F90C2C09D114485D
:10FFE000B0F80100C01C1549088003200A490870B8
:10FFF00008E00F48B0F80100C01E10490880042036
:020000040801F1
:10000000054908706422022140F25C6004F054FE4D
:1000100000BF00BF00BF1FE755080020CB0C002029
:10002000BF0C0020F808002014090020BB2D002080
:10003000E40F0020D2840208CA0C0020C80C002063
:1000400038B50546B5F53E7F09DC0A208DF800007D
:10005000DF208DF8010001202449087008E00A2003
:100060008DF800005F208DF8010000201F49087006
:1000700002226946052000F01FFA04226946022088
:1000800000F044F9284600F081F804469DF800008D
:1000900000F0FE008DF8000000208DF80200E0B2B4
:1000A0008DF8030004226946022000F005FA200AB8
:1000B0008DF802009DF8020040F080008DF80200EB
:1000C000E0B28DF8030004226946022000F0F4F942
:1000D00007480078032808DA0648008810B9042089
:1000E0000549886110200BF045FA38BD54080020FE
:1000F000550800206E0C00200000024038B5044670
:100100000A208DF8000044F010008DF80100022252
:100110006946052000F0D0F938BD000008B50CA0F4
:10012000006800900020FFF7E9FF012269460220E5
:1001300000F0C2F94FF480400649086040100860A2
:10014000800004491039086010200AF0FDF808BD4D
:10015000410000002808024010B5094800880949FC
:10016000A1F801000AF028FC02200749087005499F
:10017000B1F80100FFF764FFF4F7EAFF10BD0000DB
:10018000C80C0020E40F00205508002010B50246DE
:10019000064C247814B14FF4207101E04FF43E7105
:1001A0000123541A94FBF3F4A0B210BD54080020AC
:1001B00010B592B04FF400401F4908606420F7F773
:1001C000C2FB002410E01D4830F81400000A01A909
:1001D00001F81400194810F81400012101EB440142
:1001E00001AA5054601CC4B2222CECDB442201A9A9
:1001F000002000F061F9FA20F7F7A5FB9DF8370021
:1002000000F07F008DF8370002220DF13601192031
:1002100000F052F99DF8370040F080008DF837006B
:1002200002220DF13601192000F046F93C20F7F7C3
:100230008AFB12B010BD00002808024056080020BA
:1002400010B54FF4005005490860012010F03EFF42
:100250004FF480400149086010BD000018080240BA
:1002600070B500F053F94FF4804027490860012031
:1002700010F02CFF4FF40050234910390860012082
:1002800010F024FF4FF400501F49086040001E4941
:1002900010390860012010F019FF002400F022F945
:1002A00000251BE06006040E4FF40050164908605C
:1002B000012010F00BFF4FF480411348283811F053
:1002C0002AF808B144F001044FF400500E491039E7
:1002D0000860012010F0FAFE681CC5B2082DE1DBB1
:1002E00000F014F94FF480400749103908600120EC
:1002F00010F0ECFE4FF4005003490860012010F0AC
:10030000E5FE204670BD0000280802402DE9F041BE
:1003100007460D4616460121384600F00DF8002428
:1003200004E0FFF79DFF2855601CC4B2B442F8DB1F
:10033000FFF786FFBDE8F0812DE9F04105460E4646
:10034000002400F0E3F84FF480402949086000BF22
:100350004010086000BF400025491031086000BF10
:1003600040100860802700BF17E007F0800020B130
:100370004FF480401E49086004E04FF480401C495F
:10038000103108604FF400501949086018491031C5
:1003900008607806070E601CC4B2082CE5DB4FF439
:1003A0000050134908601249103108606806050EB4
:1003B00006B13543002417E005F0800020B14FF46A
:1003C00080400B49086004E04FF480400849103138
:1003D00008604FF400500649086005491031086074
:1003E0006806050E601CC4B2082CE5DBBDE8F08190
:1003F0001808024010B500F089F84FF48040114908
:100400000860012010F062FE4FF400500D491039D1
:100410000860012010F05AFE4FF4005009490860AE
:10042000012010F053FE4FF40050064910390860C7
:10043000012010F04BFE4FF4804002491039086053
:1004400010BD00002808024070B5044600F05EF8B8
:100450004FF4804017490860012010F037FE4FF438
:100460000050144910390860012010F02FFE4FF49D
:10047000005010490860002519E004F0800028B100
:100480004FF480400B491039086003E04FF480407E
:10049000084908604FF400500649103908606006AA
:1004A000040E4FF4005003490860681CC5B2082DC3
:1004B000E3DB70BD280802402DE9F04107460D46F8
:1004C000164600213846FFF737FF002404E0285D78
:1004D000FFF7BAFF601CC4B2B442F8DBFFF78AFF33
:1004E000BDE8F0811CB5684610F0CEFE00208DF806
:1004F00006004FF48040009002208DF80500694608
:10050000014810F0CBFE1CBD000802401CB5684637
:1005100010F0BAFE02208DF8070000208DF80400CC
:1005200001208DF806008003009000208DF8050062
:100530006946024810F0B2FE1CBD000000080240EF
:1005400010B50E4800880A3084B25CB102E0012088
:10055000F7F7F9F90A48007820B1201EA4F101014B
:100560008CB2F4D10748007808B10DF07FF9012072
:100570000549087003F086F810BD00007A0C0020D1
:10058000740C00206D0C00209A08002010B503F0B8
:1005900091F800200149087010BD00009A08002061
:1005A00070B5054600242B48407800EB40002A49EE
:1005B00001EB0010D0F805400C2D18D100BF2748E2
:1005C000006804442648844200D9264C21484078DB
:1005D00000EB4000204A02EB001000788109204621
:1005E000F5F7B8F9E0B920481C490860E7E700BF13
:1005F0001A480068241A1B48844200D2184C154837
:10060000407800EB4000144A02EB001000788109AA
:100610002046F5F79FF918B9134810490860E7E735
:100620000C49487901F0AAFE0C4908602046F5F70C
:100630006BF90E4991F86720064948780C4909780A
:1006400000F0E8FE01200B49087148710A49487022
:1006500070BD0000BB2D0020EA2D0020A00B002063
:1006600000E1F50540771B00A0860100BB290020B2
:100670006D0B0020EB240020380A00202DE9F84FF4
:1006800005468B4616464FF0000800240027A24678
:10069000A1460020009000BF49E0285D80280ADACA
:1006A0002A5D3846791C8FB2325400223846791CB4
:1006B0008FB2325439E015F804804FF6FF7000EA2B
:1006C0000828601C285C40441FFA80F808F0FF00EE
:1006D00040388121C1EB282100EB012A47F6605008
:1006E000824502D34FF0000912E04FF47C1000EB7A
:1006F0004A010222684611F097F89DF800904FF6E3
:10070000FF7000EA09299DF8010048441FFA80F9AA
:100710003846791C8FB206F800904FEA29223846F5
:10072000791C8FB23254601C84B2601C84B25C4568
:10073000B3DB3846BDE8F88F1CB5684610F0A4FD61
:1007400000208DF806004FF44070009001208DF8D5
:1007500005006946794810F0A1FD4FF40060009053
:100760006946774810F09AFD022000906946754866
:1007700010F094FD4020009000208DF8050069469F
:100780006F4810F08BFD02208DF8070000208DF8D7
:10079000040001208DF8060048F207400090002078
:1007A0008DF805006946654810F078FD02208DF847
:1007B000070000208DF8040001208DF8060040F2AB
:1007C000BB70009000208DF8050069465C4810F071
:1007D00065FD02208DF8070000208DF8040001203F
:1007E0008DF806004FF46040009000208DF8050061
:1007F0006946554810F052FD02208DF80700002090
:100800008DF8040001208DF8060040F241100090A0
:1008100000208DF8050069464A4810F03FFD012090
:1008200046498861022088610120464918310860E4
:1008300043491831086002204149283108600420EA
:100840003E49886200023E492831086080103D49D7
:100850002831086080003949886240013A491831DE
:100860000860801038492831086040000860801115
:10087000334928310860400008608020086004F097
:10088000C5F940202F492831086001208DF8070064
:1008900000208DF8040002208DF806004FF4C650A9
:1008A000009000208DF805006946244810F0F6FC01
:1008B00008220C21214810F037FD08220B211F4887
:1008C00010F032FD072211461C4810F02DFD0822C1
:1008D00006211A4810F028FD03208DF80600042098
:1008E00000906946164810F0D9FC30200090032093
:1008F0008DF8060000208DF804008DF80500012019
:100900008DF8070069460D4810F0C8FC08200090DB
:1009100000208DF804008DF8050002208DF80600F7
:1009200001208DF807006946044810F0B7FC032247
:100930001146024810F0F8FC1CBD00000000024007
:1009400000040240001402400008024010B50024D8
:100950000121104810F0FAF802E00120F6F7F3FF49
:100960000D48006838B90D48006820B92046611C60
:10097000CCB21428F1DB0020084908600649086061
:10098000074800888000422190FBF1F0054908806B
:1009900010BD000000200140A4080020A008002095
:1009A0009C080020B008002001460E2903DC01F15C
:1009B0002100C0B27047152903DC01F12B00C0B241
:1009C000F8E71B2903DC01F14500C0B2F2E71F295B
:1009D00003DC01F15F00C0B2ECE72020EAE730B5AC
:1009E00003460C460020002107E06518C5F30B05FF
:1009F0005D5D0544E8B24D1CA9B29142F5DB30BD06
:100A000001464E2901DD03207047482901DD0220FF
:100A1000FAE7422901DD0120F6E70020F4E70000B3
:100A20000146044A505C3F2902DD00F5807290B215
:100A300070470000C02002080246002100BF08E005
:100A4000064830F81100904201DB08467047481C08
:100A5000C1B23229F4DB0020F8E700005C20020874
:100A600010B5002400201449088000BF13E04FF4A3
:100A7000931000EB44112022104810F0D5FE0F48CF
:100A80000078022805DA0C480088401C0A490880D2
:100A900000E004E0641C40F2E7308442E7D300BF8A
:100AA0000548008838B90648C08820B100200449AC
:100AB000C88009F033FF10BD0C0C0020C5A7002032
:100AC000BB2D002070B505460C46B5F5806F01DBE7
:100AD000002070BD2E4606EB46004FF4804101EB2E
:100AE000001604EB44011B4A02EB01103022314690
:100AF00010F09AFE04EB4400164901EB0010007858
:100B00000121B1EB901F01DA0020E2E704EB44027F
:100B1000104B03EB02121278910904EB440203EB31
:100B20000212D2F80500F4F715FF88B104EB440275
:100B3000084B03EB02121278910904EB440203EB19
:100B40000212D2F80900F4F705FF08B10120C0E74E
:100B50000020BEE7EA2D00201CB5002400200190F3
:100B60004FF48062D100C94810F05EFE2F22C849C0
:100B7000C84810F059FEC548808943F23332811AC3
:100B8000904224D00ADCA0F58850A0F11100A0B159
:100B9000A0F58850A0F1110018BB13E0A1F5885012
:100BA000A0F11100C0B1A0F5CE40A0F18900C0B9FC
:100BB0004FF00000B849087018E04FF00100B64946
:100BC000087013E04FF00200B34908700EE04FF0D8
:100BD0000300B149087009E04FF00400AE49087005
:100BE00004E04FF00500AC49087000BF00BFAA4800
:100BF0000078052854D10120A849087082024FF4DA
:100C00004051A24810F010FEA048808943F23332D0
:100C1000811A904224D00ADCA0F58850A0F111007E
:100C2000A0B1A0F58850A0F1110018BB13E0A1F508
:100C30008850A0F11100C0B1A0F5CE40A0F189000C
:100C4000C0B94FF000009449087018E04FF001005F
:100C50009149087013E04FF002008F4908700EE0D0
:100C60004FF003008C49087009E04FF004008A49F6
:100C7000087004E04FF005008749087000BF00BF0E
:100C80008548007805280BD102208449087043026A
:100C9000002283497D48F5F736FB00207E49087025
:100CA00009F034FA03F096FE09F03CFB7748007C2B
:100CB000A8B97648C07E90B97448007D78B9002004
:100CC000102378A2014600900220F7F7C1FE002011
:100CD000102379A2014600900420F7F7B9FE6B4873
:100CE000007C18B14FF4801002F01AFF6748C07EF4
:100CF00060B16648007C18B94FF4801002F010FF14
:100D000040F6B830F6F71FFEF5F7A4F85F4991F802
:100D1000620001F09DFB6D4908605C4991F85F003D
:100D200001F096FB6A490860584991F8650001F0A6
:100D30008FFB684908605749487901F01FFB6649F5
:100D400008605448007865498871504890F86700F9
:100D5000C8715048807888720020C8724B4890F85B
:100D60005D000873494890F80D01C873002048736E
:100D700001F02AF930224FF47021594810F054FD47
:100D80005848007817280BD056480078182807D004
:100D900054480078192803D000205349086074E0B3
:100DA00004221105514810F03FFD504800784E498B
:100DB000086008460068000208604C4840780968EE
:100DC000084449490860084600680002086047482E
:100DD00080780968084444490860084600680002B1
:100DE00008604248C078096808443F4908600846DE
:100DF0000068401C08B9002008603A4800781728AD
:100E000016D139480068B0F5400F04D94FF44000BE
:100E1000354908600CE033480078182808D132487A
:100E20000068B0F1E07F03D94FF0E0702E49086010
:100E30002D480068D0B1C82415E02B48006800F5A3
:100E40008000411E012201A810F0EEFC9DF8040074
:100E50000A2805D024480068401E2349086000E0A5
:100E600003E0601EC4B2002CE7DC00BF1E4800682F
:100E70001F49086000201F490860084600681C4997
:100E80000968084440081C4908601CBDBB290020B3
:100E900060C00100BB2D0020120C0020220C00209D
:100EA000C84802085374617274696E672075702EA9
:100EB0002E2E202000000000506C656173652077A5
:100EC000616974202020202000000000C80B002051
:100ED000BC0B0020C40B0020A00B0020C008002089
:100EE000E40F00201C0C0020B00B0020BE6E002080
:100EF000A80B0020AC0B0020A40B002070B504460A
:100F00002546C5EBC50000EB400000F5BC251522C9
:100F10002946024810F088FC70BD000028A300207C
:100F200030B587B0002500240020164908801649F6
:100F3000088000BF1FE02546C5EBC50000EB400060
:100F400000F5BC251522294601A810F06DFC9DF87E
:100F5000040002280DDC0B480088401C0949088069
:100F60009DF80400012804D107480088401C064968
:100F70000880601C84B242F210708442DBDB07B050
:100F800030BD0000FC0B0020FE0B002070B50546B4
:100F9000002400BF08E02046FFF742FDA84201DB25
:100FA000204670BD601CC4B2692CF4DB0020F8E759
:100FB00070B50446254605EB45004FF4502101EB82
:100FC000001530222946024810F02EFC70BD0000AA
:100FD00095A5002010B50748847C04EB44004FF42D
:100FE000702101EB001430222146034810F01CFC54
:100FF00010BD0000BB2D0020E40F00202DE9F041C2
:101000000446854884420DD3844884420AD8002689
:101010008348201A8349B0FBF1F0C5B20020824911
:101020000870ABE0814884420DD3814884420AD8DD
:1010300001267E48201A7B49B0FBF1F0C5B20120A1
:10104000794908709AE07B4884420DD37A488442FB
:101050000AD802267948201A7249B0FBF1F0C5B2CD
:1010600000207149087089E0734884420DD36A48B2
:1010700084420AD803267248201A6A49B0FBF1F06C
:10108000C5B200206849087078E0644884420DD3F6
:101090006C4884420AD804266B48201A6149B0FB88
:1010A000F1F0C5B200206049087067E065488442ED
:1010B0000DD3664884420AD805266248201A594949
:1010C000B0FBF1F0C5B201205749087056E05F4807
:1010D00084420DD3554884420AD806265B48201A1C
:1010E0005049B0FBF1F0C5B201204F49087045E00E
:1010F0004F4884420DD3564884420AD807264C48AC
:10110000201A4849B0FBF1F0C5B2012046490870E9
:1011100034E04F4884420DD34E4884420AD8082612
:101120004B48201A3F49B0FBF1F0C5B201203E49BF
:10113000087023E0484884420DD3484884420AD8C6
:1011400009264548201A3749B0FBF1F0C5B2012005
:101150003549087012E0414884420DD3404884422A
:101160000AD80A263D48201A2E49B0FBF1F0C5B234
:1011700001202D49087001E0BDE8F0813948007870
:10118000864225D0374806703746C7EBC7000701AF
:1011900020373548007828B970223946334810F096
:1011A00043FB15E030480078012806D1702207F58E
:1011B00080512E4810F038FB0AE02B4800780228B6
:1011C00006D12B48C119702300222848F5F79BF857
:1011D0000F2D00DD0F2525481030405D2549087092
:1011E00022482030405D2449087020483030405D5E
:1011F000224908701D484030405D214908701B4855
:101200005030405D1F49087018486030405D1E49ED
:10121000087000BFB0E700000085CF00C080090162
:1012200060FECD0020A107001A080020005A6202CB
:10123000006CDC0240771B0000A8610060E3160030
:10124000808D5B0000366E01406603010048E801B6
:10125000007E56038014EF0300BD010500CF7B051F
:1012600000E1F50513080020210C00203B2500209B
:10127000C8400208140800201508002016080020A5
:1012800018080020170800201908002070B504462F
:1012900025460748048005EB85004FF4462101EB05
:1012A000001550222946034810F0BEFA70BD000018
:1012B000000C00203DA30020014600200878000219
:1012C0004A78104400028A7810440002CA78104418
:1012D00070470146881E082815D2DFE800F0040692
:1012E000080A0C0E1012612070476420FCE767208A
:1012F000FAE76A20F8E76D20F6E77020F4E774203B
:10130000F2E77720F0E7FF20EEE700004048008892
:10131000012801D10B2070473D480088102801D1D9
:101320000C20F8E73A480088B0F5807F01D10D2005
:10133000F1E737480088B0F5805F01D11020EAE777
:1013400033480088022801D10120E4E730480088B2
:10135000202801D10220DEE72D480088B0F5007F6B
:1013600001D10320D7E72A480088B0F5005F01D1FA
:101370000E20D0E726480088042800D1CBE7244877
:101380000088402801D10520C5E721480088B0F534
:10139000806F01D10620BEE71D480088B0F5804F60
:1013A00001D10020B7E71A480088082801D107209A
:1013B000B1E717480088802801D10820ABE714481E
:1013C0000088B0F5006F01D10920A4E7104800881B
:1013D000B0F5004F01D10F209DE70D48008841F284
:1013E0001111884201D10A2095E70948008842F28C
:1013F0002221884201D111208DE70548008844F25E
:101400004441884201D1122085E7FF2083E7000094
:101410007C0B00202DE9FF5F04460D4690464FF0FF
:10142000000AD34600200390002602900027019076
:1014300000908146F8480078F8490877B8F1000F25
:1014400006D0B8F1010F3BD0B8F1020F37D16FE0F1
:1014500004EB4400F24901EB0010D0F805A004EBC6
:10146000440001EB0010D0F809B00CB9012000E0F5
:10147000002000EB4000EA4901EB0010D0F8050025
:10148000039004EB440001EB0010807B060904EBA1
:10149000440001EB0010007C070904EB440001EB61
:1014A0000010B0F80D00C0F30B00029004EB4400F4
:1014B00001EB0010B0F80F00C0F30B0001906FE0DB
:1014C00004EB4400D64901EB0010D0F805A004EB72
:1014D000440001EB0010D0F805B00CB9012000E089
:1014E000002000EB4000CE4901EB0010D0F80500D1
:1014F000039004EB440001EB0010807B060904EB31
:10150000440001EB0010807B070904EB440001EB71
:101510000010B0F80D00C0F30B00029004EB440083
:1015200001EB0010B0F80D00C0F30B00019037E0A4
:1015300004EB4400BA4901EB0010D0F809A004EB19
:10154000440001EB0010D0F805B00CB9012000E018
:10155000002000EB4000B24901EB0010D0F8090078
:10156000039004EB440001EB0010007C060904EB3F
:10157000440001EB0010807B070904EB440001EB01
:101580000010B0F80F00C0F30B00029004EB440011
:1015900001EB0010B0F80D00C0F30B00019000BF8C
:1015A00000BF9E4880F8424045779E48005D9B49B9
:1015B00088779C48801C005DC877102300229AA180
:1015C00096482030F4F792FE022D06D00723002221
:1015D0009AA192481530F4F789FE9048807F002840
:1015E00073D0012802D0022870D173E110230022A9
:1015F00094A18A48F4F77AFE8A49891D01EB4401D7
:101600000988481C042106F093FF04EB4400844938
:1016100001EB001000780121B1EB901F06D10623E9
:1016200000228DA18E48F4F761FE05E0062300221A
:101630008CA18B48F4F75AFE042302228B49884878
:10164000F4F754FE77481438C07870BB7348C07FF5
:1016500002280DD104EB4400714A02EB001000F1A6
:101660002001102300226D482030F4F73FFE8BE06C
:101670006A48C07F012819D1032D04D008215046A3
:1016800006F056FF03E00821584606F051FF0923F3
:1016900003222E21754801F087FF09230022734998
:1016A0005E482030F4F722FE6EE010E003230022B3
:1016B0006FA15A482030F4F719FE042303226B4926
:1016C00056482030F4F712FE5EE05EE0DDE155485A
:1016D000801C005D02280EDA0323002264A14F481B
:1016E0002030F4F703FE0423032260494B482030E6
:1016F000F4F7FCFD17E0032D04D00821504606F056
:1017000017FF03E00821584606F012FF09230322C1
:101710002E21564801F048FF0923002253493F4833
:101720002030F4F7E3FD1023002252A13B48433060
:10173000F4F7DCFD3B48801C005D68B104EB44001D
:10174000374A02EB001000F1200110230022334839
:101750004330F4F7CBFD17E0032D04D008215046A9
:1017600006F0E6FE03E00821584606F0E1FE0923F4
:1017700003222E213D4801F017FF092302223B4995
:1017800026484330F4F7B2FD7FE1102300223EA14A
:101790002248F4F7ABFD04EB4400214901EB0010B3
:1017A00000780121B1EB901F06D1062300223BA156
:1017B0002B48F4F79BFD05E00623002239A12848B9
:1017C000F4F794FD032D04D00821504606F0B0FE36
:1017D00003E00821584606F0ABFE092303222E2120
:1017E000224801F0E1FE0923002220490B48203065
:1017F000F4F77CFD3CB9102300222CA107484330AC
:10180000F4F774FD06E0102300222DA103484330B5
:10181000F4F76CFD39E10000760B0020C3090020CD
:10182000EA2D0020CF2D0020202020202020202065
:101830002020202020202020000000002020202028
:10184000202020004348204D4F44452020202020C8
:101850002020202000000000412D2020202000001A
:10186000280A0020442D202020200000D024002021
:1018700043482D0020202020202020202020202030
:10188000202020202000000056464F204D4F444588
:10189000202020202020202000000000414E412058
:1018A00020200000444D52202020000020205646D9
:1018B0004F204D4F44452D412020202000000000A6
:1018C000202056464F204D4F44452D4220202020B9
:1018D0000000000004EB8410FE4A02EBC000011D72
:1018E00010230022FC48F4F701FD04EB8410F949B1
:1018F00001EBC00000EB4400B0F80090042109F1B6
:10190000010006F015FE04EB4400F44901EB001061
:1019100000780121B1EB901F07D106230022AFF21E
:10192000C801EF48F4F7E2FC06E006230022AFF21C
:10193000CC01EB48F4F7DAFC04230222E949E84839
:10194000F4F7D4FCE848C078F0BBE348C07F022835
:101950000DD104EB4400E14A02EB001000F120013C
:1019600010230022DC482030F4F7C0FC8CE0DA4879
:10197000C07F012818D1032D04D00821504606F05D
:10198000D7FD03E00821584606F0D2FD09230322C3
:101990002E21D44801F008FE09230022D149CE4867
:1019A0002030F4F7A3FC6FE003230022AFF24011D4
:1019B000C9482030F4F79AFC04230322C949C648D9
:1019C0002030F4F793FC5FE0FFE7C7481630005D76
:1019D00002280FDA03230022AFF26C11BE48203038
:1019E000F4F784FC04230322BE49BB482030F4F7FB
:1019F0007DFC17E0032D04D00821504606F098FD29
:101A000003E00821584606F093FD092303222E2106
:101A1000B44801F0C9FD09230022B249AE48203084
:101A2000F4F764FC10230022AFF2B811AA48433047
:101A3000F4F75CFCAC481630005D68B104EB440080
:101A4000A64A02EB001000F1200110230022A24858
:101A50004330F4F74BFC17E0032D04D00821504627
:101A600006F066FD03E00821584606F061FD0923F3
:101A700003222E219B4801F097FD09230222994958
:101A800095484330F4F732FC00BF00BF0CB9012188
:101A900000E0002194481430405C8F4981F8300008
:101AA0000CB9012100E000218F481630405C8A49C2
:101AB00081F8310010230022AFF2942186483230A1
:101AC000F4F714FC844890F83000E0B3012802D009
:101AD00002284AD15CE0804890F83100022811D1F8
:101AE0000CB9012000E0002000EB40007B4A02EB33
:101AF000001000F120011023002277483230F4F763
:101B0000F5FB32E0744890F83100E8B90323002275
:101B1000AFF2A42170483230F4F7E8FB0CB901228F
:101B200000E0002270491A3101EB42010988481C8B
:101B3000042106F0FDFC042303226A496648323082
:101B4000F4F7D4FB11E011E00821039806F0F0FC53
:101B5000092303222E21634801F026FD09230022D8
:101B600060495D483230F4F7C1FB64E00821039816
:101B700006F0DEFC092303222E215A4801F014FD51
:101B800009230022574954483230F4F7AFFB52E0A2
:101B9000514890F83100022811D10CB9012000E021
:101BA000002000EB40004D4A02EB001000F1200144
:101BB0001023002248483230F4F798FB3AE04648B8
:101BC00090F8310028BB0CB9012000E0002000EBA8
:101BD0008010404901EBC0000CB9012100E0002158
:101BE00000EB4100B0F8009003230022AFF28031F7
:101BF00039483230F4F77AFB042109F1010006F08C
:101C000097FC04230322374933483230F4F76EFB44
:101C100010E00821039806F08BFC092303222E21F3
:101C2000304801F0C1FC092300222E492A483230F5
:101C3000F4F75CFB00BF00BF04EB4400274901EB55
:101C4000001000780121B1EB901F72D1032D2BD031
:101C500004EB4400214901EB00100079C0F30110AE
:101C6000012807D10323002220A11D48801DF4F77D
:101C70003DFB20E004EB4400184901EB0010007923
:101C8000C0F30110022807D10323002218A1144831
:101C9000801DF4F72BFB0EE00323002215A1104852
:101CA000801DF4F723FB06E00323002211A10C485A
:101CB000801DF4F71BFB04EB4400084901EB001006
:101CC00000798009E8B9012300220BA104480F30F4
:101CD00014E00000AB250020C3090020EA2D0020FD
:101CE000280A0020D0240020BB2D0020414D2000D8
:101CF00053534200464D200057000000F4F7F6FA17
:101D000005E001230022A1A1A148F4F7EFFA04EBBA
:101D10004400A04901EB00100079C0F34200042800
:101D200008D1052300229CA19948801FF4F7DEFA10
:101D300010E1B3E0032D58D147B905230022AFF2DB
:101D4000C0419348801FF4F7D1FA03E1012F17D166
:101D50000421019806F0ECFB9148C0789049087185
:101D60002E20C87008460078302801D12020087045
:101D7000052300228A498648801FF4F7B7FAE9E074
:101D800004EB4400834901EB00100079C0F34200EA
:101D900038B10523002283A17D48801FF4F7A6FAFD
:101DA000D8E0022F03D14E207D49087102E049207E
:101DB0007B4908710198F5F7A9FD0090032100986F
:101DC00006F0B6FB764880787549C87008464078BA
:101DD0008870084600784870442008700523002267
:101DE0006B48801FF4F782FAB4E046B9052300225D
:101DF000AFF274516648801FF4F778FAAAE0012E1A
:101E000017D10421029806F093FB6548C078644915
:101E100008712E20C87008460078302801D1202093
:101E20000870052300225E495948801FF4F75EFAC6
:101E300090E004EB4400574901EB00100079C0F337
:101E4000420038B10523002256A15148801FF4F703
:101E50004DFA7FE0022E03D14E205149087102E075
:101E600049204F4908710298F5F750FD0090032171
:101E7000009806F05DFB4A4880784949C8700846DA
:101E80004078887008460078487044200870052320
:101E900000223F48801FF4F729FA5BE004EB44007E
:101EA0003C4901EB00100078C0F3400038B903232F
:101EB00000223EA136480938F4F718FA06E0032359
:101EC00000223BA132480938F4F710FA04EB440031
:101ED000304901EB0010808A30B9012300222FA184
:101EE0002B48F4F703FA05E00123002231A128482A
:101EF000F4F7FCF905230022AFF27C612448801F2F
:101F0000F4F7F4F9012300222BA12148801FF4F7F4
:101F1000EDF904EB44011F4A02EB0111497808096D
:101F2000022106F005FB022301221D491848801FEB
:101F3000F4F7DCF904EB4400164901EB00100078DB
:101F400000F0010030B1022303221CA11048801FC1
:101F5000F4F7CCF904EB44000E4901EB0010807853
:101F60000121B1EB901F07D10123002214A10848E1
:101F7000401EF4F7BBF906E00123002211A104483A
:101F8000401EF4F7B3F9BDE8FF9F00004E000000CB
:101F9000370A0020EA2D00204D5554202000000073
:101FA000D0240020454E4320200000005431200062
:101FB0005432200045000000430000002D4D000079
:101FC000480000004C000000084890F87F0020B94D
:101FD0000020074981F8640004E00648407804497D
:101FE00081F864000120044908727047BB29002071
:101FF000C3090020BB2D0020EB2400202DE9F04F69
:10200000ADF5657D04468B46914600260025A84621
:1020100000270320E4904FF0FF0A6078C01EC0B292
:10202000E39004F1160000F809B0A07DFFF751F924
:10203000824600BF81E0A07D072802D0A07D09284C
:1020400002D10420E49001E00320E49000256FE039
:10205000E398A8BB0AEB050006EB8601994A12F843
:102060001110884262D14FF0000811E006EB8600A3
:10207000944901EB400010F8080007EB8701924AF1
:1020800002EB410101F8080008F101001FFA80F895
:10209000B8F1060FEADB07EB87008B4901EB400044
:1020A000C68006EB8600874901EB4000C08807EB3D
:1020B0008701854A02EB41010881781C87B235E02F
:1020C000FFE70AEB050006EB8601804A12F81110C3
:1020D00088422BD14FF0000811E006EB86007B49C7
:1020E00001EB400010F8080007EB8701764A02EB8D
:1020F000410101F8080008F101001FFA80F8B8F169
:10210000060FEADB07EB87006F4901EB4000C68052
:1021100006EB86006D4901EB4000C08807EB8701A4
:10212000694A02EB41010881781C87B2681C85B2BC
:10213000E49885428CDB701C86B2E39810B940F2BB
:10214000971001E040F28F10B0423FF774AFE78183
:1021500001268CE0002704F11601885DFFF7B9F82D
:10216000824604F11600805D072804D004F11600B1
:10217000805D092802D10420E49001E00320E4906E
:1021800000253CE04FF0000834E00AEB080005EBC6
:1021900085014D4A02EB4101895D884226D105EB5C
:1021A0008502494B03EB420107EB870202AB03EBCD
:1021B000420006230022F4F799F805EB8500424916
:1021C00001EB4000C08807EB870102AA02EB410146
:1021D000C88005EB85003C4901EB4000008907EB16
:1021E000870102EB41010881781C87B208F10100E8
:1021F0001FFA80F8E4988045C7DB681C85B2E08947
:10220000A842BFDC27B900200DF5657DBDE8F08F41
:10221000E781002526E005EB850202AB03EB4201D6
:1022200005EB8502284B03EB420006230022F4F75E
:102230005DF805EB850002A901EB4000C08805EBC5
:102240008501214A02EB4101C88005EB850002A906
:1022500001EB4000008905EB850102EB410108819B
:10226000681C85B2E089A842D5DC701C86B24E4558
:102270007FF770AF06230022134904F11C00F4F726
:1022800035F80020A08120820F480089608201205B
:10229000009009F10100C3B204F11C0200210620E4
:1022A000F6F7D6FB00200090C9F10500C3B209F192
:1022B0000100C0EBC000C1B205A20620F6F7C8FBC2
:1022C0000120A1E74A2102084C21002030310208F8
:1022D00020202020202000002DE9FF4105460E4649
:1022E00017460024A0461EA30FCB8DE80F00002048
:1022F0001F49088000BF1FE005EB0421102268463B
:102300000FF092FA9DF80000B84213D108F10100D5
:102310001FFA80F8B5F55E2F0DD19DF80C0001284D
:1023200009D013480088401C114908800120114938
:10233000487200E002E0641CB442DDD300BF0C48E8
:10234000008818B101200B49487202E000200949B9
:102350004872012008490871404604B0BDE8F08188
:10236000FFFFFFFFFFFFFFFFFFFFFFFFFFFFFFFF7D
:10237000020C0020C0080020E0240020014615299E
:1023800040D2DFE801F00B0D0F11131517191B1DBB
:10239000202326292C2F3235383B3D000120704761
:1023A0000220FCE70320FAE70520F8E70A20F6E719
:1023B0001920F4E73220F2E77D20F0E7FA20EEE77B
:1023C0004FF4FA70EBE740F27120E8E740F2413059
:1023D000E5E74FF47A70E2E740F2E240DFE74FF4DE
:1023E000FA60DCE740F6C410D9E741F28830D6E75E
:1023F00042F21070D3E74CF25030D0E70248CEE7FB
:102400000248CCE71920CAE7A086010020A10700F6
:1024100070B504460025002694F8000108B100209C
:1024200070BD94F8020100F00F0565B9B4F802011F
:1024300048B1B4F802112046F3F780F80646022EA0
:1024400001D17820ECE7C5EBC5000830C0B2E7E762
:1024500001460A4632B1012A06D0022A05D0032AD3
:1024600007D103E00020704700BF00BF02EB8200ED
:10247000F9E7901EC0EB0010F5E7000010B5002052
:1024800010490870202200210F480FF0CDF90E48A6
:1024900000789A2814D001200A49087020220103EC
:1024A00009480FF0C1F9084800789A2808D002209E
:1024B000044908702023002204490348F3F723FF4E
:1024C00010BD0000210C00201B250020C840020880
:1024D0002DE9F041044600250127264606EB46007B
:1024E0004FF4E03101EB001604EB4401484A02EBE3
:1024F0000110302231460FF097F904EB44004449B3
:1025000001EB001000780121B1EB901F01DA0027E8
:1025100021E004EB44023E4B03EB021212789109D6
:1025200004EB440203EB0212D2F80500F3F712FAAF
:1025300000B9002704EB4402354B03EB021212787A
:10254000910904EB440203EB0212D2F80900F3F7FD
:1025500001FA00B90027002F58D104EB44022D4B9B
:1025600003EB021104EB4402294B03EB021030236E
:102570000022F3F7C8FE04EB4402254B03EB0212E2
:102580001278910904EB440203EB0212D2F8050021
:10259000F3F7E0F9B8BB002515E005EB85011E480F
:1025A000405C02280DD105EB85011B480844B0F8BA
:1025B000010004EB4401164A02EB0111C1F80500C9
:1025C00003E0681CC5B2042DE7DB00BF04EB440048
:1025D0000F4901EB0010D0F805001049484304EB07
:1025E00044010B4A02EB0111C1F8050004EB440061
:1025F000114601EB0010D0F8050004EB440102EB9A
:102600000111C1F80900204608F02CFABDE8F0815C
:10261000EA2D0020F74C0208492A0020A08601007C
:102620002DE9F04704460E4617460025A846A94660
:102630001B4800EB440005881A4820F8145000BFDE
:1026400021462846FEF73EFA80464846411C1FFABE
:1026500081F9B0F5806F0BDAB8F1000F08D11FB91E
:10266000681CC0F3090502E0681EC0F30905E7E72E
:10267000B8F1000F02D10020BDE8F087084800EB58
:1026800044000088A84206D0054800EB44000580BD
:102690000EB108F043F9034820F814500120EBE78D
:1026A000D52D0020600B00202DE9F04104460025C7
:1026B00000273B48065D374607EB87104FF4F031A3
:1026C00001EBC00704EB8411364A02EBC1004FF462
:1026D000027239460FF0A8F804EB8411314A02EB7C
:1026E000C10101EB440108882146FEF7EBF90128FE
:1026F0000DD104EB84102B4901EBC00000EB44002A
:102700000088294921F814000120BDE8F081002546
:1027100041E004EB8410234901EBC000143000EBCE
:1027200045000088B0F5806F33DA04EB84111D4A50
:1027300002EBC101143101EB450108882146FEF787
:10274000C1F9012825D104EB8410164901EBC00022
:10275000143000EB45000088134921F8140004EB05
:102760008410104901EBC000143000EB45000088D4
:1027700004EB84110B4A02EBC10101EB4401088018
:1027800004EB841002EBC001304608F085F901200B
:10279000BBE7681CC5B2FA2DBBDB0020B5E7000023
:1027A000D32D0020AB250020600B002070B504461F
:1027B000254605EB85104FF4F03101EBC0054FF4D1
:1027C0000272294601480FF02FF870BD8DA300203A
:1027D00000BFFEE710B506F023FAFDF7ADFFF4F7F2
:1027E0008FFFF0F7BFFAFDF72BFAF3F799FDF3F738
:1027F000A1FD0BF0C5F94FF4E1300DF087FF4FF468
:10280000E1300DF065FF05F088FB00F03BF908E0D2
:10281000C820F5F798F8FEF799F8064800780649B9
:102820000870054800783C28F2DB02F0DFF902F07E
:10283000BDF910BDB0080020B60B002010B502464F
:102840000B460020002100BF21E00001545C302C29
:1028500006DB545C392C03DC545C303C204414E02F
:10286000545C412C06DB545C462C03DC545C373C46
:1028700020440AE0545C612C06DB545C662C03DCCB
:10288000545C573C204400E000BF4C1CE1B299422C
:10289000DBDB10BD2D48C07818382C49C8700846BD
:1028A0008078401C8870084640780D284CD2DFE8BC
:1028B00000F04B0723083C093D0A0B3E0C3F0D007E
:1028C00000BF00BF00BF00BF00BF00BF1F4880782F
:1028D0001F2810DD01201D49887008464078401CE3
:1028E0004870084640780C2805DD012048700846ED
:1028F0000078401C087027E01448007800F00300BE
:1029000048B9124880781D280EDD01200F498870D3
:102910000320487008E00D4880781C2804DD012061
:102920000A498870032048700EE000BF00BF00BF56
:10293000064880781E2806DD012004498870084674
:102940004078401C487000BF00BF7047400B00201B
:1029500070B50546002400BF0AE005EB0411074AE4
:1029600002EB041010230022F3F7CDFC601C84B2AC
:1029700003488088A042F0DC70BD0000F00C00200D
:10298000E80C00201FB5002438A30FCB8DE80F0002
:1029900000F0BAF83023002238493948F3F7B3FC85
:1029A000302300223549303135483030F3F7ABFC65
:1029B000002008F057F8012008F054F8FDF7C0FD9A
:1029C00000BF03E0201D0EF0ADFF641C0C2CF9D3FA
:1029D000002404E004F11E000EF0A4FF641C202C6F
:1029E000F8D3002404E004F15E000EF09BFF641CA9
:1029F000342CF8D30D224FF4BC2168460FF038F880
:102A0000002404E004F1C6000EF08CFF641C052CC9
:102A1000F8D3002404E004F1D0000EF083FF641C1E
:102A2000032CF8D3D6200EF07DFF00240CE004F137
:102A3000D7000EF077FF04F1DE000EF073FF04F113
:102A4000E7000EF06FFF641C082CF0D3F0200EF0AE
:102A500069FF002404E004F593700EF063FF641C2A
:102A6000082CF8D3FDF792FD1FBD000002AAAAAA08
:102A7000AA416C6C2043616C6C000000F74C0208AA
:102A8000EA2D0020002000BF04E00021194A115463
:102A9000411C88B240F214518842F6DB002004E069
:102AA0000021154A1154411C88B2B0F5805FF7DB54
:102AB000002004E00021114A1154411C88B2B0F5F5
:102AC000805FF7DB002004E000210D4A1154411C17
:102AD00088B240F21A418842F6DB002004E000216F
:102AE000084A1154411C88B240F21A418842F6DB70
:102AF00070470000DB7D0020EF820020EF92002075
:102B0000757500208F79002008B5002080230246CB
:102B10000821009000F010FE00200F230FA20146B4
:102B200000900220F5F794FF00200F230FA201462A
:102B300000900420F5F78CFF4FF4806300220F49CA
:102B40000F48F3F7E0FB07F0DBFE2F2300220D49CF
:102B50000D48F3F7D8FB07F0E1FE08BD5265636F3F
:102B6000766572696E672E2E2E202000506C65618E
:102B7000736520776169742020202000C84802080E
:102B8000BB290020C84C0208BB2D002010B540F224
:102B9000094200210148F3F74FFA10BD6E70002082
:102BA00010B5FF2200210248F3F746FA10BD0000DD
:102BB000767400202DE9F04104460D4616461F4666
:102BC000012020706570A670FF20607520750020C0
:102BD000A080A0712081A081E081208260820622F5
:102BE000002104F11600F3F727FA0622002104F170
:102BF0001C00F3F721FA0A22002104F12200F3F766
:102C00001BFA0648857417B101200549C8700122D6
:102C10000721062008F0C2F8BDE8F081830A0020F1
:102C2000F4240020FF2005490870487088700020B7
:102C3000C8700871A1F8050070470000570B00200C
:102C400070B504460D461023002221461948F3F7BB
:102C50004DFB11230022294616481630F3F746FB98
:102C60000223002214A113482730F3F73FFB02236D
:102C7000002211A10F482730F3F738FB062300226A
:102C80000EA10C482A30F3F731FB0A2300220DA1D4
:102C900008483030F3F72AFB00200649491E8874A3
:102CA000C874087501204875FF2081F82A0081F852
:102CB0003B0070BD840A002030310000202020201D
:102CC0002020000020202020202020202020000084
:102CD0002DE9F04104460E46174600254FF4807258
:102CE00000212046F3F7A8F900BF07E0705DFF2838
:102CF00000D105E0705D6055681C85B2BD42F5DB12
:102D000000BF04F580742781E58001202070002039
:102D1000608020716081A4F580742046F5F76EFF15
:102D2000BDE8F08108B5002080230246082100900C
:102D300000F002FD00200F2311A2014600900220A6
:102D4000F5F786FE00200F2311A201460090042013
:102D5000F5F77EFE4FF40063002211491148F3F7A6
:102D6000D2FAFDF7EDFB00200EF0DCFD4FF400621F
:102D700000210C480EF07CFEFDF708FC08BD0000A9
:102D80005265636F766572696E672E2E2E20200065
:102D9000506C656173652077616974202020200084
:102DA000C8400208BE2E002010B50446FF2C31D0CA
:102DB0003F480078D8B901220621104607F0EEFFFF
:102DC000012C0BDD042300223AA13C48F3F78EFAD4
:102DD00037480078401C3649087005E0042300227B
:102DE00037A13648F3F782FA00203749086004F12A
:102DF0003000C1B22E4802780078401C2C4B18706D
:102E00002E4881543048006800EB800004EB4000FD
:102E10002D4908602D480078022818D12C484078A8
:102E20002C490978884212D000202B4981F83100C2
:102E30001023002229A128483230F3F757FA04233F
:102E400003221E4924483230F3F750FA10E00020E4
:102E50002149C8771023002220A11F482030F3F712
:102E600045FA0423032215491B482030F3F73EFAA4
:102E70001F48007830B11F48007828B91C480078F6
:102E8000082801D1012000E0002038B901220621E4
:102E9000104607F083FF002015490870012007F055
:102EA0008DFF03480078042801D1F5F7EDFF10BD30
:102EB0008E0C0020302D2D2D00000000940C0020E1
:102EC0002D2D2D2D00000000900C00206D0B0020FA
:102ED000BB2D00205F0B0020C309002043482D2D8F
:102EE0002D2D2D202020202020202020000000003B
:102EF000B3080020B208002010B504461B48007833
:102F000008B9F2F7D5F819480078102806D16422DC
:102F100002214FF4DC7001F0CFFE10BD2046F2F725
:102F2000F6FA1349114A12788854104800780F288D
:102F300005DA5F210E4A0D480078401C1154102319
:102F400000220B490B48F3F7D1F9012007F0E0FE0E
:102F500006480078401C054908706422022140F2AE
:102F60005C6001F0A9FE00BFD7E70000AD0C0020B7
:102F7000AE0C00203509002010B504461F4800782B
:102F800008B9F2F7BDF81D480078082806D1642278
:102F900002214FF4DC7001F08FFE10BD04F130000F
:102FA000C1B21748154A127881541448007807288E
:102FB00005DA5F22124911480078401C0A54114872
:102FC000006800EB800004EB40000E4908600B48ED
:102FD0000078401C094908700823002208490A4863
:102FE000F3F784F9012007F0AFFE6422022140F2DA
:102FF0005C6001F061FE00BFCFE700009D0C002087
:103000009F0C0020A80C00205F09002010B504468A
:103010001748007840B90323002216A11648F3F799
:1030200065F900201549088004F13000C1B210484C
:1030300002780078401C0E4B18700F4881540F48DE
:10304000008800EB800004EB40000C49088002235C
:10305000032209490A48F3F749F901200949887010
:1030600003480078022801D1F5F790FF10BD000059
:10307000BF0C00202D2D0000C20C0020C00C002031
:10308000FA0800201409002010B5044623480078EF
:10309000B8B90523002222A12348F3F727F9F2F754
:1030A00057F8012C02DD062C00DA10BD062C08DBD7
:1030B00030211A4802780078401C184B18701A48C2
:1030C000815404F13000C1B2144802780078401CE9
:1030D000124B18701448815418460078032804D104
:1030E00018460078401C194608701048008800EB0C
:1030F000800004EB40000D490880052300220A49A6
:103100000B48F3F7F3F801200A49C8700348007828
:10311000052801D1F5F786FF00BFC6E7BF0C0020E8
:103120002D2D2D2E2D000000C20C0020C00C0020E3
:10313000FF0800201409002010B50446FF2C20D001
:103140002F48007808B9F2F745F804F13000C1B211
:103150002B4802780078401C294B1870294881546C
:1031600018460078032804D118460078401C1946F8
:1031700008702548006800EB800004EB40002249FD
:10318000086022480078022815D12148407821495A
:10319000097888420FD0102300221FA12348F3F79B
:1031A000A5F80923002217492048F3F79FF80120CA
:1031B0001F49487110E01023002217A11B48123844
:1031C000F3F794F8092300220E4918481238F3F750
:1031D0008DF8012016490871164890F8EA0018B9D0
:1031E00007480078072807D0124890F8EA0028B16D
:1031F00003480078092801D1F5F758FF10BD0000F9
:103200008E0C0020940C0020900C00206D0B0020F0
:10321000BB2D00205F0B00202D2D2D2E2D2D2D2DB3
:103220002D2020202020202000000000F509002073
:10323000EB240020BB29002010B50446304800785C
:1032400040B9042300222FA13048F3F74FF80020A3
:103250002F49086004F13000C1B229480278007893
:10326000401C274B1870294881542948006800EBFE
:10327000800004EB40002649086004230022234913
:103280002448F3F733F824488088214909688842A4
:1032900003D31B48007804280EDD0020184908706D
:1032A0001B4908600423002216A11A48F3F71EF8F0
:1032B00001201A4988701EE015480068D8B11449E9
:1032C0000968481EF5F742FF1348808810490968CD
:1032D00001EB8101B0EB410F0DD8002008490870C7
:1032E0000B4908600423002206A10A48F2F7FEFFFA
:1032F00001200A49887001200849C87110BD0000EA
:103300008E0C00202020202000000000940C0020C3
:10331000900C0020770A0020E80C00207B0A002097
:1033200010B504461748007840B90323002216A1BF
:103330001648F2F7DBFF00201549086004F1300061
:10334000C1B2104802780078401C0E4B18700F482C
:1033500081540F48006800EB800004EB40000C49EA
:10336000086003231A4609490A48F2F7BFFF012003
:103370000949C87003480078032801D1F5F7B4FF64
:1033800010BD00008E0C00202D2D2D00940C00206F
:10339000900C0020150B00200925002010B50446D4
:1033A0002148007840B90923002220A12248F2F7E1
:1033B0009DFF00202149086004F13000C1B21A4885
:1033C00002780078401C184B18701B48815418462E
:1033D0000078032804D118460078401C194608706C
:1033E0001648006800EB800004EB400013490860B9
:1033F0000923002210491248F2F778FF01201149F1
:103400008870114890F8EA0030B90748007807281A
:1034100008D1F5F799FF05E003480078092801D1A4
:10342000F5F792FF10BD00008E0C00202D2D2D2EE3
:103430002D2D2D2D2D000000940C0020900C00202F
:10344000020B002009250020BB29002010B50446EE
:103450002148007840B90723002220A12148F2F733
:1034600045FF00202049086004F13000C1B21A482D
:1034700002780078401C184B18701A48815418467E
:103480000078012804D118460078401C19460870BD
:103490001548006800EB800004EB4000124908600A
:1034A000072303220F491148F2F720FF012010499A
:1034B0004870104890F8EA0030B9074800780528AD
:1034C00008D1F5F775FF05E003480078072801D11A
:1034D000F5F76EFF10BD00008E0C00202D2E2D2D57
:1034E0002D2D2D00940C0020900C00200B0B0020A3
:1034F00009250020BB2900202DE9F04704460E468F
:1035000017460025A846A946AA46B4F80601B4F80D
:103510000811884206DBB4F80801A4F8060100206F
:10352000BDE8F08794F8000158B1B4F8065104E002
:10353000681E205C6055681E85B2002DF8DC267080
:1035400010E0B4F80201401C1FFA80F8B4F80651EC
:1035500004E0681E205C6055681E85B24545F8DCB5
:1035600004F80860B4F80601401CA4F8060184F8C9
:1035700004710D21204604F0D3FB8146B9F1000F00
:103580000CD12046F5F73AFB2046FEF741FF824674
:10359000012003494871034880F814A00120BFE7C7
:1035A000F4240020830A002030B50C46002119467F
:1035B00004E04D1E455D45544D1EA9B29142F8DC14
:1035C000845430BD2DE9F04104460E460025002705
:1035D000A846B4F80601401CB4F80811884202DB82
:1035E0000020BDE8F08194F8000180B1B4F8060134
:1035F000401C85B204E0A81E205C6055681E85B2A0
:10360000012DF8DC307820707078607017E0B4F825
:103610000601401C85B204E0A81E205C6055681EAF
:1036200085B2B4F80201A842F6DB3178B4F80201A1
:10363000401C21547178B4F80201801C2154B4F864
:103640000601801CA4F80601002084F804010D2165
:10365000204604F065FB8046B8F1000F0BD12046F0
:10366000F5F7CCFA2046FEF7D3FE074601200349C2
:103670004871034807750120B3E70000F4240020D7
:10368000830A002010B50022074908480EF0BCFC50
:103690000022012106480EF0EAFA002201218807E3
:1036A0000EF0E5FA10BD000005000C00001401400A
:1036B0000000014010B50122074908480EF0A4FCA3
:1036C0000122114606480EF0D2FA01221146900757
:1036D0000EF0CDFA10BD000005000C0000140140F2
:1036E0000000014038B5002400BF0CE01148005D27
:1036F00038B100208023024601210090204600F0CE
:103700001BF8601CC4B2082CF0DB0A48007A0128C0
:1037100009D10020702302460121009000F00CF82E
:1037200000200449087200220721104607F036FBEA
:1037300038BD0000122500202DE9F04705460E4651
:1037400017469846DDF820A0002412E02919C8B2D7
:10375000394601F093F94FF0000906E0504601F0B8
:10376000E3F909F1010000F0FF09C145F6DB601C37
:10377000C4B2B442EADBBDE8F087000008B51F48D8
:10378000007838B101201E4B06220021009007204E
:10379000F5F719FA1948407840B10120184B9B1DE4
:1037A0000322302100900720F5F70DFA13488078A6
:1037B00040B10120124B093305224421009007201B
:1037C000F5F701FA0D48C07840B101200C4B0E33DB
:1037D0000246682100900720F5F7F5F907480079BF
:1037E00040B10120064B0F3302467821009007209C
:1037F000F5F7E9F9002007F06FFA08BD380A002054
:10380000280A002008B54A48007838B1002008236B
:10381000484A014600900120F5F71AF944484078DB
:1038200040B100200723434A08323C210090012088
:10383000F5F70EF93E48807840B1002012233D4A4A
:103840001032014600900320F5F702F9394890F84C
:103850003F0090BB3648C07840B100200A23354A6B
:103860003532014600900520F5F7F2F8304800792E
:10387000A8B1304991F83F00F4F778FD002001230A
:103880002DA2712100901846F5F7E2F800200123DF
:10389000284A4032782100901846F5F7D9F8244894
:1038A000407900283FD000200123224A4032742171
:1038B00000900520F5F7CCF835E0FFE71C480079CB
:1038C00038B3002001231DA2712100901846F5F79E
:1038D000BFF800200123174A403278210090184693
:1038E000F5F7B6F8134890F85200012812D10020DD
:1038F0000C23104A4132014600900520F5F7A8F844
:10390000002005230B4A4D325C2100901846F5F744
:103910009FF808E000201223064A22320146009058
:103920000520F5F795F8002007F0E4F908BD000040
:10393000BD0900206A0900203E0000003C00000094
:1039400008B50D48007838B100200C230B4A014619
:1039500000900120F5F77CF80748407840B100203E
:103960001023064A0C32014600900420F5F770F847
:10397000002007F0CDF908BD4509002029090020E5
:1039800008B51848007838B100200F23164A0821DE
:1039900000900120F5F75CF81248407888B10020CB
:1039A0000723114A1032082100900320F5F7F0F8A0
:1039B000002002230C4A17325D2100900320F5F706
:1039C00047F80848807840B100200C23064A193295
:1039D000082100900620F5F73BF8002007F0A6F933
:1039E00008BD0000F5080020D008002008B51348E5
:1039F000007838B100200E23114A014600900120C2
:103A0000F5F726F80D48407840B100200A230C4A0B
:103A10000E32014600900320F5F71AF80748807827
:103A200040B100200823064A1832014600900520C4
:103A3000F5F70EF8002007F087F908BD67090020A8
:103A40004709002008B53348007838B132482523AB
:103A50000522082100900120F5F783F92D484078D0
:103A600078B32E48407820B101280FD0022827D102
:103A700019E001210846F4F749FE00210320F4F77C
:103A800045FE00210620F4F741FE19E00021012047
:103A9000F4F73CFE01210320F4F738FE0021062054
:103AA000F4F734FE0CE000210120F4F72FFE002192
:103AB0000320F4F72BFE01210620F4F727FE00BFB8
:103AC00000BF1448807840B100200523134A921C9F
:103AD000382100900120F4F7BBFF0E48C07840B1B8
:103AE000002005230D4AD21D382100900320F5F750
:103AF0004FF80848007940B100201023074A0C32E3
:103B0000082100900620F4F7A3FF002007F02AF90F
:103B100008BD0000140900205C500208F8080020CD
:103B200070B50646002400254FF4806231460E48E9
:103B30000DF07AFE00BF13E0E0B2002100F09EFF1E
:103B4000002509E0C4F1070105EBC111064A505CEC
:103B500000F0EAFF681CC5B2802DF3DB601C84B264
:103B6000082CE9DB70BD0000BE2E002008B5184807
:103B7000007808B1F4F72FFD1648007860B91448B2
:103B8000407808B300201023124A521C08210090EC
:103B90000320F4F75DFF17E00D48407840B10020A6
:103BA00010230C4A521C082100900220F4F750FF09
:103BB0000748807840B100201023064A11320821BE
:103BC00000900420F4F744FF002007F0D9F808BD66
:103BD000FF240020E00A0020F8B59E4890F842003B
:103BE00008B1032000E0012004469A4890F8420002
:103BF00008B1042000E002200546964890F84200F3
:103C000008B1012000E0052006469348C07828B19D
:103C1000904A92F84210507FF4F704FB8E48C07926
:103C200010B38C4890F8630010B1012812D108E05D
:103C300001210220F4F76AFD00210520F4F766FD5A
:103C400011E000210220F4F761FD01210520F4F7C5
:103C50005DFD08E000210220F4F758FD0021052059
:103C6000F4F754FD00BF00BF7B480079002848D01E
:103C70007848807F80B3012802D0022840D100BF5D
:103C80007448C07F022807D11023724A20320A21CB
:103C90002846F4F73DFF1EE06E48C07F48B900207B
:103CA00008236C4A2032142100902846F4F770FF54
:103CB00011E000200723674A20320F210090284698
:103CC000F4F766FF00200223624A27326421009045
:103CD0002846F4F7BDFE13E0FFE7002007235D4A06
:103CE00020320F2100902846F4F752FF00200223D3
:103CF000584A2732642100902846F4F7A9FE00BFF5
:103D000000BF5548407978B3524890F8300060B30E
:103D1000012802D0022833D100BF4E4890F831006C
:103D2000022809D1002010234A4A32320A21009089
:103D30003046F4F78DFE16E0464890F8310048B959
:103D400000200723434A3232272100903046F4F7FF
:103D50007FFE08E0002009233E4A32321C210090F9
:103D60003046F4F775FE0BE00BE0FFE70020092377
:103D7000384A32321C2100903046F4F769FE00BF09
:103D800000BF3548007838B10020324B1022014680
:103D900000902046F4F717FF2F48807940B10020AB
:103DA0002C4B15330422682100902046F4F70BFFBA
:103DB0002948007A90B3274890F8640010B1012890
:103DC0002BD11DE0234890F8420060B90121032067
:103DD000F4F750FD00210120F4F74CFD00210620EE
:103DE000F4F748FD0BE001210846F4F743FD0021FC
:103DF0000320F4F73FFD00210620F4F73BFD0CE023
:103E000000210320F4F736FD00210120F4F732FDF4
:103E100001210620F4F72EFD00BF00BF0E48807878
:103E200098B10C48007F40B100200CA302227421FD
:103E300000902046F4F7C7FE07E0002008A3022206
:103E4000742100902046F4F7BEFE002006F0B6FF75
:103E5000F8BD0000C3090020EB2400204844000006
:103E600020200000F8B50124022505263F480079EE
:103E7000002846D0002010233D4A0F2100903046F4
:103E8000F4F7E6FD3A484338807F30B3012802D08A
:103E9000022835D100BF36484338C07F022809DAEE
:103EA00000200823324A233A142100902846F4F7D0
:103EB0006FFE11E0002007232D4A233A0F210090C6
:103EC0002846F4F765FE00200223294A1C3A6421A3
:103ED00000902846F4F7BCFD12E000200723244A96
:103EE000233A0F2100902846F4F752FE00200223C7
:103EF0001F4A1C3A642100902846F4F7A9FD00BF30
:103F000000BF1A48007840B10020194B433B1022F3
:103F1000014600902046F4F756FE1448807940B1DF
:103F20000020134B2E3B0422682100902046F4F71A
:103F30004AFE0E488078A0B10D484338007F40B15A
:103F400000200CA30222742100902046F4F73BFECF
:103F500007E0002008A30222742100902046F4F715
:103F600032FE002006F02AFFF8BD0000EB240020FE
:103F7000060A0020484400002020000038B5002434
:103F80003A4890F8390030B139484079002869D072
:103F9000F4F79CFB66E03648C07810B1FF20F4F7D8
:103FA0004BFB3348007808B1F4F7F6FB3048C07992
:103FB000A8B1682408E02146032000F05FFD00203E
:103FC00000F0B2FD601CC4B2802CF4DB0120274B52
:103FD0003A330422692100900320F4F7F4FD2448C9
:103FE000407840B100201023204A521C0E2100903E
:103FF0000120F4F72DFD1E48807808B1F4F7ECFBA2
:104000001B48007918B11949C87CF4F7F5FB18482A
:10401000407948B11548007D1023144A15320E210D
:1040200000900420F4F714FD11488079D0B10F48B6
:1040300090F8380058B100200C49C874112301F1E0
:104040002702014600900620F4F702FD0AE0074827
:1040500090F825001023054A27320E2100900620F3
:10406000F4F7F6FC002006F0B7FE38BD3D0A00204C
:104070007B0A002038B5224890F82A00112809DB75
:10408000002011231E4A1732012100900420F4F76A
:10409000DFFC34E000200090194890F82A3000F14D
:1040A000170201210420F4F7D3FC012000901448EA
:1040B00090F82A3017301A18173890F82A00C0EBF9
:1040C000C000401CC1B201230420F4F7C1FC002051
:1040D00000900B4890F82A00C0F11000C3B20848C5
:1040E00090F82A4017302044421C054890F82A00D6
:1040F000C0EBC0000830C1B20420F4F7A9FC38BD01
:10410000830A002038B500246B48007878B3002378
:10411000202237210120F4F749FC002320227B21B3
:104120000120F4F743FC0023202263210220F4F74E
:104130003DFC6248007820B1012809D0022815D141
:104140000DE000237F2237210120F4F72FFC0DE042
:1041500000237F227B210120F4F728FC06E00023C6
:104160007F2263210220F4F721FC00BF00BF5248E8
:10417000807840B10020514B5B1C09220146009021
:104180000120F4F720FD4C48407840B100204B4B13
:104190000A330A223E2100900120F4F714FD46481C
:1041A000C07840B10020454B143306223E210090D8
:1041B0000220F4F708FD40480079D0B100203F4BC1
:1041C00026330322014600900420F4F7FCFC002073
:1041D0003A4B29330322014600900520F4F7F3FC03
:1041E0000020364B2C330322014600900620F4F7C2
:1041F000EAFC3148407940B10020304B1D330922A0
:10420000014600900220F4F7DEFC2B48C07988B10B
:104210002A4991F832000021F4F7F4FB274991F87C
:1042200031000121F4F7EEFB244890F831002349D6
:1042300081F832002048807968B3204890F8300037
:104240000F2801DC002404E01C4890F830000F38EF
:10425000C4B21A4890F82F006830692190FBF1F23F
:1042600001FB12001730C5B2002320222946062088
:10427000F3F796FF114890F82F006830692190FB02
:10428000F1F201FB12001730C5B201232246294684
:104290000620F3F785FF0848007A40B10020074B5D
:1042A0001A3303226E2100900220F4F78CFC0020C8
:1042B00006F0A0FD38BD000009250020010B0020FC
:1042C00038B50024F048007808B1F4F765FAEE48F4
:1042D000407838B100201023EC4A0E2100900120D4
:1042E000F4F7B6FBE848807808B1F4F775FAE648C9
:1042F000C07820B1E549491E887CF4F79DF9E34870
:10430000401E807C052816D0DF48007928B1DF499F
:10431000491EC87C0021F4F7EBFCDB48407950B122
:10432000DA48401E007DD949491EC8740A46517DAD
:10433000107DF4F7DDFCD448807900287DD0D34887
:10434000401E807D072807D2DFE800F0042A4D7B5D
:10435000C9E40700FFF78EFE07E100200323CB4AE4
:104360001632012100900420F4F772FB0020012393
:10437000C7A2162100900420F4F76AFB0020032353
:10438000C24A19321D2100900420F4F761FB00207D
:104390000323C0A2322100900420F4F759FBE4E08B
:1043A00000200323B94A1632012100900420F4F7BB
:1043B0004FFB00200123B6A2162100900420F4F741
:1043C00047FB00200523B14A19321D21009004202B
:1043D000F4F73EFB00200323AEA24021009004200E
:1043E000F4F736FBC1E000200423A84A163201216D
:1043F00000901846F4F72CFB00200123A6A21D21F3
